:020000040000FA
:06000000F1EF7DF012009B
:0600080004EF0CF01200F1
:060018000CEF0CF01200D9
:06180000F1EF7DF0120083
:0618080069EF2DF0120053
:021818001200BC
:06182A000001FA6B120040
:10183000060E0B019C5D01E2B3D06550020B01E086
:10184000120052EC19F001E1ABD003EC18F00009E2
:1018500001E1A1D051EC18F01E0A01E192D0030A77
:1018600001E18CD0010A01E186D0070A01E180D0B4
:10187000010A01E17AD0030A75E0010A70E00F0A5B
:101880006BE0010A66E0030A61E0010A5CE0070A16
:1018900057E0010A52E0030A4DE0010A48E01F0A3E
:1018A00043E0010A3EE0030A39E0010A34E0070A96
:1018B00030E0010A29E0030A25E0010A21E00F0ACD
:1018C0001DE0010A19E0030A15E0010A11E0070A08
:1018D0000CE0010A08E0030A04E0010A55E161D8BE
:1018E00058D07AD856D0B6D854D02FEC13F051D067
:1018F000C3D84FD028D94DD088D94BD0D3D949D0CF
:1019000056DA47D063DA45D0010EE66E99DA41E93E
:1019100040D0D6DB3ED099EC10F03BD0C0EC10F0BC
:1019200038D0E1EC10F035D002EC11F032D06FEC91
:1019300011F02FD029EC11F02CD04CEC11F029D063
:1019400096EC11F026D0BDEC11F023D0E0EC11F0B4
:1019500020D003EC12F01DD011EC14F01AD089EC59
:1019600016F017D09EEC16F014D082EC17F011D0C0
:10197000D1EC16F00ED014EC17F00BD069EC17F088
:1019800008D0E8EC16F005D0500EE66E660EDFECDF
:1019900018F03BEC1AF04B0EE66E660EDFEC18F01A
:1019A0001200490EE66E660EDFEC18F0390EE66E98
:1019B000660E7EEC1AF0270EE66E660E7EEC1AF0CE
:1019C000160EE66E660E7EEC1AF0080EE66E660ED9
:1019D000DFEC18F07FEF4BF00001010EFB6F15D923
:1019E0003BEC1AF0F3D93BEC1AF06ADB3BEC1AF053
:1019F000A0DB68EC1AF0C4DB68EC1AF0E2DB3BEC2D
:101A00001AF002EC11F068EC1AF06FEC11F03BECFC
:101A10001AF029EC11F068EC1AF04CEC11F03BECE8
:101A20001AF096EC11F068EC1AF0BDEC11F068ECCD
:101A30001AF0E0EC11F03BEC1AF09EEC16F068ECBA
:101A40001AF082EC17F07FEC4BF0FF0EE66E650E9D
:101A500038EF1BF0F3EC18F041E8010E016E19ECC1
:101A600019F003E20CEC19F0016E01EBE6FF1FEC3C
:101A700064F041E960EF19F0F3EC18F046E8026A0F
:101A800019EC19F00AE2F1EC1AF007E2013402E273
:101A90000150050802E381EB02F0EA6A0234FE0B12
:101AA000E96EEA360D0EE926000EEA22EE50056ECA
:101AB000ED50066E055006103BE0036A046A0550BF
:101AC00006103BE005500408000E06541EE230EC00
:101AD0001BF019EC1AF0E66A0401032811EC1BF064
:101AE000E66A020E0401032411EC1BF0E66A030E01
:101AF0000401032411EC1BF0CBEC19F00326000EBB
:101B00000422040E055E000E11D030EC1BF0EFEC49
:101B100018F005500108000E065402E23EEC1BF0DE
:101B20001CEC1AF0032A000E04220506065AC7D739
:101B3000EC0EE66E650EDFEC18F07FEC4BF047E93B
:101B4000E7CFD9FF1200F3EC18F044E800013E5152
:101B5000036E3F51046E035004104CE0016A026AA8
:101B60007FEC4BF0D70EE66E650E03EC19F0B40E69
:101B700019EC1AF01CEC1AF0CE0EE66E650EDFECD6
:101B800018F0035004103BE003500408000E045406
:101B90001EE223EC1BF019EC1AF0E66A040101289E
:101BA00000EC1BF0E66A020E0401012400EC1BF0BD
:101BB000E66A030E0401012400EC1BF0CBEC19F0E3
:101BC0000126000E0222040E035E000E11D023EC4B
:101BD0001BF0EFEC18F003500108000E045402E271
:101BE0003EEC1BF01CEC1AF0012A000E0222030648
:101BF000045AC7D7EC0EE66E650EDFEC18F07FECEA
:101C00004BF045E9E7CFD9FF120055EC1BF000017E
:101C1000FB5102082BE20CEC19F0026E010E025C83
:101C200025E30250050822E3F4C0E6FFF5C0E6FF15
:101C300062EC4EF042E9016E013401E3016A0134C5
:101C400005E20150640802E2640E016E020403E042
:101C5000020E025C05E101EB0CFF01EB0DFF04D06D
:101C600001EC1AF001EBEFFF54EC46F0C80EE66E03
:101C7000650E6BEC1AF0026A025005080FE3E66A83
:101C800001EC1AF0EF50EFEC18F0050E025C04E0E6
:101C900055EC19F0FEEC18F0022AEED799EC18F08A
:101CA00011EF19F0F3EC18F046E819EC19F033E2F3
:101CB00056EC1AF0056EF450066E05EBE4F406EBF4
:101CC000E5F40401E66BE76BE5AF02D0E669E7698E
:101CD000BFEC19F003E6390EF5EC1AF01CE305EB46
:101CE000E8F406EBE9F4EA6BEB6BE9AF02D0EA69E2
:101CF000EB69C3EC19F006E6D880400EE855090EF2
:101D000023EC19F008E305EB01FF06EB02FF54ECAE
:101D100046F01DEC28F07FEC4BF0B70EE66E650E3A
:101D200003EC19F001CFE6FF02CFE6FF1FEC1BF03A
:101D3000B10EE66E650EFEEC18F01CEC1AF0000118
:101D4000625129EC19F006E00401D890E533E43340
:101D5000E804FBE1E9EC19F0E5AF02D0E669E769D8
:101D6000A0EC19F0A20EE66E650EAAEC1AF01CECBF
:101D70001AF00001635129EC19F006E00401D89033
:101D8000E533E433E804FBE1E9EC19F0E5AF02D018
:101D9000E669E769A0EC19F0930EE66E650EAAEC11
:101DA0001AF099EC18F047E9E7CFD9FF1200BDEC23
:101DB00028F0000906E00001010EFB6F73DF54EF0D
:101DC00046F0770EE66E650EDFEF18F040EC1AF085
:101DD00023E2F9EC1AF0E5AF02D0E669E769BFEC5F
:101DE00019F003E6FA0EA3EC1AF016E3A4EC19F0CE
:101DF000E9AF02D0EA69EB69C3EC19F006E6D880D6
:101E0000EE0EE855020E23EC19F006E301EB03FF9A
:101E100002EB04FF54EC46F07FEC4BF0720EE66EE2
:101E2000650E03EC19F003CFE6FF04CFE6FF1FECCD
:101E30001BF06C0EE66E650E2DEC1BF011EF19F029
:101E4000D9CFE6FFE1CFD9FF82E95DE8136A146AD2
:101E5000156A166A176A186A196A1A6A1B6A1C6A6E
:101E60001D6A1E6A096A0A6A0B6A0C6A0D6A0E6AA2
:101E70000EEC27F008EC1AF0F350036EF450046EE9
:101E800003CFE6FF04CFE6FF52EC2AF042E9B5ECBF
:101E900019F0D00EE45D070EE55955E200016551D9
:101EA0002DE0656BF29E6451026E020406E16A51F8
:101EB000685D076E69516B5505D068516A5D076EA4
:101EC0006B516955086EF28EB5EC19F0E451F408C7
:101ED000010EE55513E2020409E1F1EC19F01B0FC4
:101EE0003FEC19F00D2A000E0E2208D0F1EC19F08B
:101EF000170F3FEC19F00B2A000E0C22AEEC2AF063
:101F00008FEC2BF004010550F35CE46F0650F4589D
:101F1000E56FE4510208000EE555B9E208EC1AF04D
:101F200086C0E4F487C0E5F40401E66BE76BE5AF37
:101F300002D0E669E769D950130F3FEC19F0092A7E
:101F4000000E0A22A4D7000EE66EE66A52EC2AF0D2
:101F500042E9005001E1B0D009EBE6FF0AEBE6FFF1
:101F6000E66AE66A13EBE6FF14EBE6FF15EBE6FF25
:101F700016EBE6FF0FEC1AF0166EE550156EE55005
:101F8000146EE750136E0BEBE6FF0CEBE6FFE66A10
:101F9000E66ACEEC19F00FEC1AF01A6EE550196EE5
:101FA000E550186EE750176EABEC19F0E66AE66A7A
:101FB000D7EC19F00FEC1AF01E6EE5501D6EE550CF
:101FC0001C6EE7501B6E7FEC4BF05E0EE66E650EEE
:101FD00003EC19F076EC19F0CEEC19F049EC1AF09C
:101FE00099EC18F04A0EE66E650E03EC19F076ECEB
:101FF00019F0D7EC19F049EC1AF01CEC1AF0175054
:10200000181019101A1005E11B501C101D101E107D
:1020100030E01BEBE8F41CEBE9F41DEBEAF41EEBFB
:10202000EBF4D950170FE96EDACFEAFFEE50040156
:10203000E827EE50E923EE50EA23EE50EB23E8C404
:10204000E6FFE9C4E6FFEAC4E6FFEBC4E6FF1B0EC9
:10205000E66EB70EE66EE66AE66A4BEC19F004012E
:10206000E4510F6EE551106EE651116EE751126E9C
:1020700004D00F6A106A116A126A7FEC4BF03C0EB2
:10208000E66E650E03EC19F00FEBE6FF10EBE6FFD2
:102090001FEC1BF0340EE66E650E2DEC1BF0280EC7
:1020A000E66E650E03EC19F013EBE6FF14EBE6FFAA
:1020B0001FEC1BF084EC1AF05EE9E7CFD9FF1200A9
:1020C00040EC1AF025E2F9EC1AF0E5AF02D0E6692F
:1020D000E769BFEC19F003E6640EA3EC1AF018E30D
:1020E000A4EC19F0E9AF02D0EA69EB69C3EC19F08E
:1020F00006E6D880E80EE855030E23EC19F008E355
:1021000001EB05FF02EB06FF54EC46F004EC3AF05D
:102110007FEC4BF0200EE66E650E03EC19F005CF58
:10212000E6FF06CFE6FF1FEC1BF099EC18F011EF6D
:1021300019F091EC1AF017E29CEC18F005E6100E7D
:10214000055C270E88EC19F00EE3083405E2055013
:102150005008460E8EEC19F006E305EB07FF06EB80
:1021600008FF54EC46F07FEC4BF01B0EE66E650E5C
:102170006BEC1AF007CFE6FF08CFE6FF35EF1AF059
:1021800095EC1AF00FE2F1EC1AF001E3016A013468
:1021900005E20150640802E2640E016E01EB09FFE2
:1021A00054EC46F07FEC4BF0120EE66E650E03EC3D
:1021B00019F00F010951EFEC18F084EC1AF060EF00
:1021C00019F095EC1AF00FE2F1EC1AF001E3016A54
:1021D000013405E20150640802E2640E016E01EB75
:1021E0000AFF54EC46F07FEC4BF00D0EE66E650EE8
:1021F00003EC19F00F010A51EFEC18F084EC1AF01F
:1022000060EF19F091EC1AF017E29CEC18F005E67B
:10221000C80E055C000E88EC19F00EE3083405E2E8
:102220000550C208010E8EEC19F006E305EB2FFFF6
:1022300006EB30FF54EC46F07FEC4BF0050EE66EFB
:10224000650E6BEC1AF02FCFE6FF30CFE6FF35EFCF
:102250001AF040EC1AF015E2F9EC18F0140ED890D0
:1022600002BE03D0015C000E02580BE3023404E20C
:1022700001506408000E025404E301EB33FF54ECF8
:1022800046F07FEC4BF0FD0EE66E640E03EC19F0A9
:102290000F01335143EF1AF040EC1AF015E2F9EC5C
:1022A00018F0040ED89002BE03D0015C000E025854
:1022B0000BE3023404E201501408000E025404E35C
:1022C00001EB34FF54EC46F07FEC4BF0F50EE66E7C
:1022D000640E03EC19F00F01345143EF1AF091EC46
:1022E0001AF017E29CEC18F005E6640E055C000E8F
:1022F00088EC19F00EE3083405E205502C08010EB5
:102300008EEC19F006E305EB31FF06EB32FF54ECDF
:1023100046F07FEC4BF0EE0EE66E640E6BEC1AF0BE
:1023200031CFE6FF32CFE6FF35EF1AF091EC1AF02D
:1023300017E29CEC18F005E62C0E055C010E88EC0B
:1023400019F00EE3083405E205505808020E8EEC31
:1023500019F006E305EB36FF06EB37FF54EC46F0C9
:102360007FEC4BF0E70EE66E640E6BEC1AF036CFA6
:10237000E6FF37CFE6FF35EF1AF040EC1AF015E232
:10238000F9EC18F00A0ED89002BE03D0015C000EE2
:1023900002580BE3023404E20150FF08000E02541D
:1023A00004E301EB35FF54EC46F07FEC4BF0E10E1B
:1023B000E66E640E03EC19F00F01355143EF1AF08D
:1023C00040EC1AF015E2F9EC18F0280ED89002BE95
:1023D00003D0015C000E02580BE3023404E201500A
:1023E0005A08000E025404E301EB38FF54EC46F0A7
:1023F0007FEC4BF0D90EE66E640E03EC19F00F0182
:10240000385143EF1AF0F3EC18F051E8540E016E16
:10241000520E026E550E036E450E046E056A460E90
:10242000066E410E076E4C0E086E530E096E450E79
:102430000A6E0B6A19EC19F051E256EC1AF00F6EA5
:10244000F450106E0F0E0F140F01396F7FEC4BF02C
:10245000D30EE66E640E38EC1BF09C0EE66E640E36
:10246000A7EC1AF039A104D0950EE66E640E03D0E5
:102470008D0EE66E640EDFEC18F0560EE66E640EFE
:10248000A7EC1AF039A304D0950EE66E640E03D0C3
:102490008D0EE66E640EDFEC18F01F0EE66E640E15
:1024A000A7EC1AF039A504D0950EE66E640E03D0A1
:1024B0008D0EE66E640EDFEC18F0E80EE66E630E2D
:1024C000A7EC1AF039A704D0950EE66E640E03D07F
:1024D0008D0EE66E640EDFEC18F0BBD0CF0EE66E0C
:1024E000630EA7EC1AF03951116E9C0EE66E640E65
:1024F000A7EC1AF039A103D0D950010F02D0D9505E
:10250000060F21EC1AF052EC19F003E1C0EC47F091
:10251000FAD794EC19F006E0540E0C5C03E0740E4C
:102520000C5C01E11180300E0C5C06E0460E0C5C88
:1025300003E0660E0C5C01E11190560EE66E640E2F
:10254000A7EC1AF039A303D0D950010F02D0D9500B
:10255000060F21EC1AF052EC19F003E1C0EC47F041
:10256000FAD794EC19F006E0540E0C5C03E0740EFC
:102570000C5C01E11182300E0C5C06E0460E0C5C36
:1025800003E0660E0C5C01E111921F0EE66E640E14
:10259000A7EC1AF039A503D0D950010F02D0D950B9
:1025A000060F21EC1AF052EC19F003E1C0EC47F0F1
:1025B000FAD794EC19F006E0540E0C5C03E0740EAC
:1025C0000C5C01E11184300E0C5C06E0460E0C5CE4
:1025D00003E0660E0C5C01E11194E80EE66E630EFA
:1025E000A7EC1AF039A703D0D950010F02D0D95067
:1025F000060F21EC1AF052EC19F003E1C0EC47F0A1
:10260000FAD794EC19F006E0540E0C5C03E0740E5B
:102610000C5C01E11186300E0C5C06E0460E0C5C91
:1026200003E0660E0C5C01E11196BF0EE66E630ED0
:10263000DFEC18F052EC19F003E1C0EC47F0FAD7E8
:10264000590E0001E05D03E0790EE05D04E111EB5D
:1026500039FF54EC46F052E9E7CFD9FF1200F3EC12
:1026600018F041E8AD0EE66E630EDFEC18F07FEC7B
:102670004BF0A60EE66E630E4FEC19F00150050804
:1026800011E3010EE66E0150EFEC18F0050E015C4F
:1026900003E055EC19F003D04D0EE66E660ED5EC56
:1026A0001AF0ECD799EC18F09F0EE66E630E4FEC23
:1026B00019F00150050811E3B0EC19F0130FE96EA1
:1026C0000F0E9DEC1AF003E055EC19F003D04D0EFF
:1026D000E66E660ED5EC1AF0ECD799EC18F0980E71
:1026E000E66E630E4FEC19F00150050811E3B0ECF3
:1026F00019F01B0FE96E0F0E9DEC1AF003E055EC7C
:1027000019F003D04D0EE66E660ED5EC1AF0ECD73C
:1027100099EC18F0910EE66E630E4FEC19F0015033
:10272000050811E3B0EC19F00B0FE96E0F0E9DECEC
:102730001AF003E055EC19F003D04D0EE66E660E6C
:10274000D5EC1AF0ECD71CEC1AF00001435103E170
:102750000001475138E07FEC4BF0770EE66E630ED8
:102760004FEC19F0040E015C11E2B0EC19F0430FCC
:10277000E96E000ED8EC1AF003E055EC19F003D026
:102780004D0EE66E660ED5EC1AF0ECD799EC18F00B
:102790005E0EE66E630E4FEC19F0040E015C11E262
:1027A000B0EC19F0470FE96E000ED8EC1AF003E018
:1027B00055EC19F003D04D0EE66E660ED5EC1AF00E
:1027C000ECD71CEC1AF07FEC4BF04A0EE66E630E71
:1027D00003EC19F00F012B51EFEC18F055EC19F048
:1027E000FEEC18F0E66A0F012C5143EC1BF03D0E95
:1027F000E66E630E03EC19F08150020B01E0010E4E
:1028000043EC1BF0300EE66E630E03EC19F08150C2
:10281000040B01E0010E19EC1AF099EC18F060EFCE
:1028200019F0F3EC18F04FE80B680C680001015147
:10283000086E0251096E0D6B0E6B01C0E6FF02C0FF
:10284000E6FF66EC46F042E919EC19F003E246ECCB
:102850001BF00DD0F50EE66E620EDFEC18F052ECB8
:1028600019F003E1C0EC47F0FAD789EC1AF0C5EC97
:102870001AF006EBF3FF07EBF4FFF40EF31802E196
:10288000010EF4182AE0C80EF31801E1F45023E019
:10289000640EF31801E1F4501CE0320EF31801E16C
:1028A000F45015E0140EF31801E1F4500EE00A0E96
:1028B000F31801E1F45007E0050EF31810E1F450AD
:1028C0000EE10B6A0CD0010E09D0020E07D0030EE8
:1028D00005D0040E03D0050E01D0060E0B6EFF0EC0
:1028E0000B5C04E1D60EE66E620E62D00001FB5175
:1028F000020806E2F4C0E9FFF5C0EAFFEF5026D077
:10290000C90EE66E620EDFEC18F0B80EE66E620ECF
:10291000DFEC18F0A60EE66E620EDFEC18F08E0EFD
:10292000E66E620EDFEC18F0750EE66E620EDFECFE
:1029300018F0690EE66E620EDFEC18F052EC19F03A
:1029400003E1C0EC47F0FAD70001E051016E690ED7
:10295000015C06E0490E015C03E0300E015C01E120
:102960000C6A680E015C06E0480E015C03E0310E63
:10297000015C02E1010E0C6E740E015C06E0540E67
:10298000015C03E0320E015C02E1020E0C6E6D0E82
:10299000015C06E04D0E015C03E0330E015C02E1D8
:1029A000030E0C6EFF0E0C5C07E1580EE66E620E15
:1029B000E66EF4EC4BF0A8D1040E0B02F3500C249D
:1029C0000A6E0B5005E14E0EE66E620EDFEC18F05B
:1029D0000B0405E1430EE66E620EDFEC18F0020E0A
:1029E0000B5C04E1380EE66E620EE9DB030E0B5C55
:1029F00004E12D0EE66E620EE2DB040E0B5C04E1D8
:102A0000210EE66E620EDBDB050E0B5C04E1150E9B
:102A1000E66E620ED4DB060E0B5C04E1090EE66E78
:102A2000620ECDDB0C5004E1FD0EE66E610EC7DBDD
:102A30000C0404E1F00EE66E610EC1DB020E0C5CCC
:102A400004E1DD0EE66E610EBADB030E0C5C04E100
:102A5000C90EE66E610EB3DB0001886B87DB2DECDF
:102A60001AF0B50EE66E610E8EEC1AF052EC19F00B
:102A700003E1C0EC47F0FAD782DBE5AF02D0E669AC
:102A8000E769BFEC19F003E6E80EF5EC1AF00FE386
:102A900059EC19F0E9AF02D0EA69EB69C3EC19F01F
:102AA00002E6DEEC1AF003E361DBE4EC19F000016E
:102AB000886B5CEC1AF02DEC1AF0A10EE66E610E3C
:102AC0008EEC1AF0EFDB03E1C0EC47F0FBD757DBED
:102AD000E5AF02D0E669E769BFEC19F003E6E80E5E
:102AE000F5EC1AF00FE3E5DBE9AF02D0EA69EB6938
:102AF000C3EC19F002E6DEEC1AF004E35CEC1AF029
:102B0000E4EC19F00001886B45EC1AF02DEC1AF09A
:102B1000900EE66E610E8EEC1AF0C4DB03E1C0ECA1
:102B200047F0FBD72CDBE5AF02D0E669E769BFECE5
:102B300019F003E6190EA3EC1AF00FE3BADBE9AFC4
:102B400002D0EA69EB69C3EC19F002E6E4EC1AF092
:102B500004E345EC1AF0E4EC19F00001886B60EC3A
:102B60001AF02DEC1AF07F0EE66E610E8EEC1AF064
:102B700099DB03E1C0EC47F0FBD701DBE5AF02D006
:102B8000E669E769BFEC19F003E6190EA3EC1AF049
:102B90000EE38FDBE9AF02D0EA69EB69F4DB02E612
:102BA000E4EC1AF004E360EC1AF0E4EC19F0000134
:102BB000886BE66A99EC1AF0B1EC1AF06A0EE66ED0
:102BC000610E8EEC1AF06EDB03E1C0EC47F0FBD730
:102BD0007BDB0BE2073404E20650FF08000E0754CB
:102BE00004E399EC1AF006EBEFFF0001886BE66A4C
:102BF00064EC1AF0B1EC1AF0550EE66E610E8EEC34
:102C00001AF050DB03E1C0EC47F0FBD75DDB0BE2D1
:102C1000073404E20650FF08000E075404E364EC96
:102C20001AF006EBEFFFA2DA4BEC1BF05CEC1AF0AB
:102C3000EECFE6F4EFCFE7F40401E651E45DE751AF
:102C4000E55911E293DAEE500D6EED500E6E5CEC2C
:102C50001AF04BEC1BF08ADAE7DB5CEC1AF00DEBB8
:102C6000EEFF0EEBEDFF45EC1AF04BEC1BF060ECC9
:102C70001AF0EECFE6F4EFCFE7F4E651E45DE7516A
:102C8000E55913E245EC1AF0EE500D6EED500E6E64
:102C900060EC1AF04BEC1BF045EC1AF0C5DB60EC75
:102CA0001AF00DEBEEFF0EEBEDFF99EC1AF0EFCF03
:102CB000E4F464EC1AF0EF50E45D10E2E6DBEF5070
:102CC0000F6E64EC1AF0EF50E66E99EC1AF0E552D4
:102CD000E750EF6E64EC1AF00FEBEFFFBF0EE66EFD
:102CE000630E6DDADFDA03E1C0EC47F0FBD7590E73
:102CF0000001E05D03E0790EE05D07E101C0E6FF61
:102D000002C0E6FF71EC46F042E950E9E7CFD9FF97
:102D1000120095EC1AF007E27FDA016E0150040808
:102D200002E301EB97FB7FEC4BF0470EE66E610E82
:102D30006ADA0B01975143EC1BF0C2D2A1DB1FE210
:102D4000F9EC1AF0E5AF02D0E669E76918DB03E6B3
:102D5000010EA3EC1AF013E3F7DAE9AF02D0EA6947
:102D6000EB6911DB05E6D8802C0EE855010E6BDA15
:102D700006E301EB3AFF02EB3BFF54EC46F07FEC3D
:102D80004BF03F0EE66E610E3EDA3ACFE6FF3BCFE8
:102D9000E6FF1FEC1BF03C0EE66E610E2DEC1BF007
:102DA00040D26EDB0CE2FCEC1AF005E0010E0118DB
:102DB00006E1025004E101EB3DFF54EC46F07FECEC
:102DC0004BF0340EE66E610E1EDA0F013D515BD3FF
:102DD00055EC1BF0DF0EE66EE1EC59F041E92EEC0C
:102DE0005AF028EC5AF00009FCE10AEC5AF0F350D2
:102DF000016EF450026E2B0EE66E610E04DA68DA94
:102E0000240EE66E610EFAD9E66A8350800B01E06B
:102E1000010EE5D91A0EE66E610EF0D9E66A84500D
:102E2000040B01E0010E2FD355EC1BF0030E016ED5
:102E3000026AFFD90EE2E0DB05E0010E011809E1AC
:102E4000025007E101EB3EFF54EC46F00001010E99
:102E5000576F7FEC4BF0020E01180FE102500DE1AD
:102E600000015C6B5D6B0001586B596B5A6B5B6BBF
:102E70000E0108690001010E576F120EE66E610E19
:102E8000C2D90F013E51ABD9020E011801E1025027
:102E900005E0030E01181BE1025019E10E0EE66E6B
:102EA000610EACD9E66A5CC0E6FF5DC0E6FFC7DB39
:102EB0000A0EE66E610EA2D958C0E6FF59C0E6FFC1
:102EC0005AC0E6FF5BC0E6FF06EC2DF044E931D9BD
:102ED000A8D1D6DA0EE290DB05E0010E011809E177
:102EE000025007E101EB3FFF0001010E576F54EC68
:102EF00046F07FEC4BF0020EE66E610E84D90F01B6
:102F00003F51C1D212DB1FE2F2C0E9FFF3C0EAFF7A
:102F1000EF50016E300E015C06E0470E015C03E0ED
:102F2000670E015C02E10F013C6B310E015C06E0B3
:102F3000460E015C03E0660E015C03E10F01010E29
:102F40003C6F54EC46F00F013C5104E1F80EE66E84
:102F5000600E35D90F013C0504E1EE0EE66E600E01
:102F60002ED9AED140D941E8040118BF4AD05EEC59
:102F70004BF0F350016E080E015C0CE10001FA51B8
:102F80000008F2E2FA07EA0EE66E600EE66EF4EC76
:102F90004BF035D00A0E015C03E00D0E015C08E138
:102FA0000001FA51C7D9EF6AFA6B65DA010E2AD02F
:102FB0000F0E0001FA5DD8E201EBE6F40401E76BC5
:102FC000E6BFE769E6C4E6FFE7C4E6FF23EC58F096
:102FD00042E9F3CFE4F4F4CFE5F4F350F410C4E0A5
:102FE0000001FA51FA2BA6D901EBEFFF7FEC4BF071
:102FF00001EB88F00001896B53DBCAEC4BF042E92E
:10300000B3D7000E5DD1EFD843E8026A036A00012E
:10301000FB6B02508FD9EF50016E01503DE0200E46
:10302000015C32E02C0E015C2FE00A0E015C2CE00A
:103030000D0E015C29E05B0E015C26E05D0E015C7B
:1030400023E03A0E015C20E03D0E015C1DE00350E0
:1030500021E1050E0001FB5D1DE2010E036E025031
:103060000401E56BE00FE46F000EE5230001FB5166
:10307000FB2BE96EEA6AD890E936EA36F00EE926CB
:10308000000EEA22D1D906D0035004E0036A0250B0
:1030900051D9EF6A022ABDD7025044E9E7CFD9FFE0
:1030A000120003DB02680001FB51000840E2026AE3
:1030B0001F0E025C3CE2016A100E015C36E299D9F7
:1030C000EFCFE6F40401E76BE6BFE769E6C4E6FF8D
:1030D000E7C4E6FF35EC58F042E9F3CFE4F4F4CF6F
:1030E000E5F40250060DF3CFEAF4F4CFEBF42C0E26
:1030F0000401EA27AD0EEB230150F76AEA25F66ECC
:10310000EB51F7220800F5CFE8F4E96BE8BFE96975
:10311000E851E4190AE1E951E51907E16AD9EF50EC
:1031200002E1025005D0012AC7D7022AC1D70250B6
:1031300078D082D97FEF4BF0A9DAD2D92EDA4ADAE9
:1031400001EBE6FF02EBE6FF1BDAEAEC7BF0B4EC06
:1031500079F00CDA0401E451056EE551066EE65192
:10316000076EE751086ED890085012000A500A0DF9
:103170000850F324E96E0950F420EA6E1200C9D910
:10318000AFD9026EE551036EE651046EE751056E4C
:1031900021DA02EBE6FFF4D905EBE6FFEAEC7BF07F
:1031A00043EC79F0E552E550076EE750066E06EB0A
:1031B000E4F407EBE5F40401E66BE76B1200E66E5E
:1031C000F4EC4BF042E91200A4D9CAEC57F044E900
:1031D000A0D9EBEC57F042E9F3CFFAF01200E66E1B
:1031E000E66A1FEF1BF0D9CFE6FFE1CFD9FF81E9F7
:1031F00012005CD9016EF450026E1200E66E5BECB8
:103200002DF042E9120067D9E66A120082D9CAECB1
:103210004BF042E97FEF4BF039DA62EC4EF042E9D5
:10322000120043E9E7CFD9FF1200E926000EEA2297
:1032300012000001FB5101081200E559000EE65989
:10324000000EE7591200E955000EEA55000EEB5545
:103250001200E66EE66A720EE66E060EE66E65EC2B
:103260007BF0E552E5CFE9F4E7CFE8F40401040E82
:10327000EA6FEA51E8C4E4F4E9C4E5F41200E96E47
:10328000DACFEAFFE451EE26E551EE22E651EE22D6
:10329000E751EE2212001FEC7BF0B6EF1AF01BD9BB
:1032A000016A12005FDE00091200060EE66E660E6D
:1032B000120006EBE8F407EBE9F4EA6BEB6B1200A3
:1032C00042E9E7CFD9FF120024D95FD907341200B1
:1032D00001EBE6FF02EBE6FF1FEF1BF001EBE4F46E
:1032E00002EBE5F40401E66BE76B1200640EE66E98
:1032F000E66AE66AE66A550EE66E080EE66EE66A6D
:10330000E66A12007FEC4BF00001886BE66A12005F
:103310000658000E0758000E085812000654000EFA
:103320000754000E085412000001E0510C6E310EDB
:103330000C5C1200EA6AE00FE96E000EEA2212004D
:10334000E4512BD97FEF4BF001EBE8F402EBE9F409
:10335000EA6BEB6B12000DEBE6FF0EEBE6FF1200E3
:10336000010EE66E0150EA6A12008FEC2BF00401A8
:103370000350F35CE46F0450F458E56F1200D890EA
:10338000E751000A1200EB35000EEB19120002ECB7
:103390002CF042E9120050D8040E120017EBE6FFA1
:1033A00018EBE6FF19EBE6FF1AEBE6FF12001BEB4A
:1033B000E6FF1CEBE6FF1DEBE6FF1EEBE6FF12004F
:1033C00049E9E7CFD9FF120006EBEEFF07EBEDFF6F
:1033D0001200390E0401E427030EE523E66BE76BC8
:1033E000120007EBE4F408EBE5F4E66BE76BD95069
:1033F000120001500001EA6AF025E96EF151EA225B
:1034000012000250EA6A0B0FE96E0F0EEA22120058
:103410008FEC2BF0F350056EF450066E12001FEC8B
:103420007BF0E552E5501200E4C4EEFFE5C4EDFF89
:103430001200D5DE3EEF1BF033D9CAEC4BF042E967
:103440001200E66EDACFE6FFE552E5500E6EE75069
:103450000D6E81DFB9DE06EF19F0EECFE6FFEECF9D
:10346000E6FF95DF1DD9E4EF18F091DF170EE66E49
:10347000650EF3D8A5D74D0EE66E660EDFEF18F099
:1034800014D919EF19F0FFD8CCD670DE040E15EF61
:1034900019F099EC7BF0FFDEE4C4E6FFE5C4E6FF3B
:1034A000CED8580EE66E650EFEEF18F0EFD8BBECE6
:1034B0004EF042E9F350120059DE020E15EF19F0FA
:1034C00055DE060E15EF19F051DE090E15EF19F055
:1034D000ECDEDFEF18F0E66E54EC2DF042E912005E
:1034E0004EEC55F042E9FCC0E4F4FDC0E5F4FEC04A
:1034F000E6F4FFC0E7F40401E451120060DE350E8B
:10350000E66E660EDFEF18F0250EE66E650E2DEF07
:103510001BF0E00EE66E000EE66E120050DE06EFC7
:1035200019F061DE48E819EF19F05DDE41E819EFA6
:1035300019F01CDE080E15EF19F0EA22EF504FDEED
:10354000050E015C1200E45D000E1DEF19F037DE80
:103550000F01120058DEBCDEB10EE66E650EFEEF06
:1035600018F0EF503CDE9CD8E4EF18F0E552E5CFC0
:10357000E7F4E5CFE6F4E5CFE5F4E7CFE4F41200B5
:1035800003EBE6FF04EBE6FF1200BBEC4EF042E972
:10359000F350066EF450076E1200016EE551026E94
:1035A000E651036EE751046E120028DE012A120074
:1035B000EA22EF5014DE030E015C1200D880200EC8
:1035C000E8554E0E23EF19F0D880880EE855130EFB
:1035D00023EF19F0E66AE66AC80EE66E420EE66E62
:1035E00012001ADE016E01341200E45D030E1DEFBD
:1035F00019F0FFDD6EEF19F0FCDD01500210120032
:10360000E46F000E0220E56F00013C510401E42547
:10361000E96E00013D510401E521EA6EEF5019EF1A
:103620001AF0E46F000E0420E56FE4C4E6FFE66ED6
:1036300002EBE6FF36EC3BF043E919EF1AF05DECE4
:103640002CF043E912005EDE000101503C25E96EDA
:1036500002503D21EA6EEF501200D0DD99EF18F0D4
:1036600051DE8EDF02EBE6FF36EC3BF043E9120061
:10367000CADD0F013951DDDE99EF18F04D0EE66E0F
:10368000660EFEEF18F0ABDD99EF18F0F2C0E6FF22
:10369000F3C0E6FF1200EECFE4F4EFCFE5F4120042
:1036A000880EE66E000EE66E12009DDD42E8120006
:1036B000D6EC23F045E8026A036AD0EC26F07CECF5
:1036C00039F00BEC28F0320EB8EC23F030EC27F098
:1036D0004DEC42F0C1EC46F0EBEC66F0010EE66E0C
:1036E000080E34EC23F0010EE66E090E34EC23F0E4
:1036F000E66A010E75EC23F0A0EC44F015EC0CF03A
:10370000800EE66EE66A000EE66E0B0EE66E010EA9
:10371000E66E7C0EE66E380EE66EDCEC46F047E9AF
:1037200022EC47F00B01976B0B01966B0F010051D8
:1037300003E0A1EC25F002D00B01956B16EC27F00D
:1037400067EC42F0016E025009E070EC24F0E808EA
:10375000030EE55503E2015001E1026A035016E051
:1037600070EC24F0D008070EE55502E2036A0ED093
:103770008150020B0BE18150040B08E1036A0B013D
:10378000020E956FE66A0C0E75EC23F0010411E150
:10379000026A036A0B01950505E1956BA0EC44F004
:1037A00089EC25F0020E0B01955D03E1956B89EC28
:1037B00025F0020E015C21E10B01955116E100019B
:1037C000586B596B5A6B5B6B00015C6B5D6B0E0148
:1037D000086989EC25F093EC24F0022A030E025CC0
:1037E0000CE3026AA1EC25F008D0950506E1026A17
:1037F000956BA0EC44F089EC25F0030E015C07E129
:103800000B01955104E193EC24F0010E036E64EC7E
:1038100027F0016E0B0195510BE1015002E089EC9C
:1038200025F01DEC21F063EC22F04DEC22F01FD0CE
:1038300095050AE1E9D892EC20F0000902E00B01BD
:10384000956B7CEC20F013D0020E955D10E1C7EC77
:1038500025F0BEEC23F006E6D880880EE455130E62
:103860006AEC24F004E2BDEC22F093EC24F0BAEC14
:1038700043F018EC0CF0C0EC47F062D765EC54F064
:103880000F015FBF02D08BEC54F01FEC4CF0C0EC8A
:1038900047F0F4D7D6EC23F04BE842EC26F0020ECA
:1038A000B8EC23F0010E026E0250050813E3046A1F
:1038B000056A016A100E015C03E2FEEC23F0FAD700
:1038C0003AEC24F0130FE96E0F0EEA22E4C4EFFF86
:1038D000022AEAD774EC25F0020EB8EC23F0030EAE
:1038E000026E0250050837E3046A056A016A100E89
:1038F000015C03E2FEEC23F0FAD73AEC24F01B0F54
:10390000E96E0F0EEA22E4C4EFFF0250EA6A130FD9
:10391000E96E0F0EEA22EF50066E076A0250EA6A5D
:103920001B0FE96E0F0EEA22EF50086E096A0F01B5
:103930000A510A6E0B6A2CEC26F00AEBE6FF0BEB41
:10394000E6FF08EC24F026EC26F0DFEC24F0E4C4DB
:10395000EFFF022AC6D716CF19FF18CF1AFF1ECFC6
:1039600021FF20CF22FF0F011951066E076A215156
:1039700055EC25F0E4C429FF0F011A51066E076AC1
:10398000225155EC25F0E4C42AFF060E026E0250C7
:10399000070834E3010E036E0350640822E303EBCF
:1039A000E6FF02EBE6FFBCEC3BF042E9020EB8ECAE
:1039B00023F0046A056A016A100E015C03E2FEEC62
:1039C00023F0FAD7040ED89005320432E804FBE164
:1039D000DFEC24F00450EF5C000E055402E2032AF1
:1039E000DBD70328E66E0250EA6A0B0FE96E0F0E72
:1039F000EA22E552E750EF6E022AC9D71BEC26F007
:103A00004CE9E7CFD9FF1200D6EC23F05AE80B01BE
:103A1000965101E0C3D08150020B01E0BFD081502C
:103A2000040B01E0BBD063EC42F0E66A070E75ECD4
:103A300023F00EEC27F02EDFE2EC24F0016A026A9C
:103A4000036A046AB9EC39F0EBEC66F011CFE6FFDB
:103A50004AEC26F012CFE6FF050E34EC23F0320ECE
:103A6000B8EC23F02C0EE66E010EE66E52EC2AF056
:103A700042E9E2EC25F0F00E0B01961501E084D04E
:103A80000001655171E0656BC7EC24F002E1F45070
:103A90000C1802E00B01968F7BEC3AF00B0196516B
:103AA0000EE1000125510B185FE126510C185CE175
:103AB00000010087008B4FEC23F0010E36D09605F5
:103AC0000BE1A1EC24F075EC24F04EE1E5510C186B
:103AD0004BE10EEC25F029D0020E965D16E1DCECF0
:103AE00023F003E3EDEC23F003E2CFEC25F01DD04F
:103AF00000011307000E145B1707185B8150020BBF
:103B000033E08150040B30E02DD0030E965D0FE1C1
:103B1000AAEC23F08150020B27E08150040B24E033
:103B20001CEC24F021E2D6EC25F0966F1DD0040E9B
:103B3000965D1AE1AAEC23F0ABEC24F000013651BB
:103B4000091806E137510A1803E1C70E00010017F2
:103B50002BEC24F009E30001005104E14FEC23F0C9
:103B6000050E966F0B019689AEEC2AF0000902E172
:103B70000B01968BA9EC25F002E6E9EC25F001E3B8
:103B80007AD70B01968D77D701EC25F0150E0B0136
:103B9000965D02E0B9EC39F063EC42F05BE9E7CF07
:103BA000D9FF1200D9CFE6FFE1CFD9FF85E94FE871
:103BB000140E00013025056E000E3121066E0550F1
:103BC000021810E1065003180DE100010083008582
:103BD0000089640E03EC26F074EC25F0030EE66E0B
:103BE000E66E40D0020E04018DEC25F007E3120EC4
:103BF00093EC23F003E239EC25F008D2120E18EC16
:103C000026F036E1E551031833E1DDEC25F004E060
:103C10000401C2EC24F0FDE192EC25F004E0040183
:103C2000C2EC24F0FDE1E4C41DFF0F0109510B6E4D
:103C30000C6A1451076E086A1C5123EC25F0E4C489
:103C400024FF0F011551076E086A1D5123EC25F062
:103C5000E4C425FF1E0E03EC26F00F012B6B2C6B2A
:103C6000E66AE66A8EEC3BF042E961EC25F040D270
:103C7000140E8DEC25F05AE3240E93EC23F056E25B
:103C800039EC25F0ED22170E040118EC26F002E1C4
:103C9000E551031822E01B0EEFEC25F0021802E1BB
:103CA000E75103181AE01F0E0524E86F000E0620E6
:103CB000E96FE851021802E1E95103180EE0230E02
:103CC0000524EA6F000E0620EB6FEA51021801E0AE
:103CD0000FD2EB51031801E00BD2020EF6EC25F0E7
:103CE0009AEC25F00F012B5107EC26F0EA22E4C4F0
:103CF000EFFF040EF6EC25F004019AEC25F00F011D
:103D00002C518DEC23F0E4C4EFFF61EC25F0230E81
:103D1000040118EC26F002E1E551031801E1E8D1B5
:103D20000F012B2B2C2BCEEC23F0E2D1240E18EC20
:103D300026F001E0ECD0E551031801E0E8D0B30E25
:103D4000076E086A00014651075C000E085806E23B
:103D5000456945C044F045C043F010D00F6A040ED9
:103D60000F5C0CE283EC23F0EF50075C000E085868
:103D700003E283EC23F0EF680F2AF1D700014A51E8
:103D8000075C000E085806E2496949C048F049C07E
:103D900047F012D00F6A040E0F5C0EE20F508DEC4C
:103DA00023F0EF50075C000E085804E20F508DEC32
:103DB00023F0EF680F2AEFD70F0124510001435D74
:103DC00006E2466B46C045F046C044F010D00F6A8C
:103DD000040E0F5C0CE20CEC26F00F0124510401E0
:103DE000E45D03E283EC23F0EF6A0F2AF1D70F01C1
:103DF00025510001475D06E24A6B4AC049F04AC0BE
:103E000048F014D00F6A040E0F5C10E20F508DECD6
:103E100023F0EFCFE4F40F0125510401E45D04E247
:103E20000F508DEC23F0EF6A0F2AEDD713680F6A5D
:103E3000040E0F5C46E283EC23F0EF5040E083EC8D
:103E400023F0E9EC24F001E1E55139E0106A040EB9
:103E5000105C35E210508DEC23F0EF502EE0105046
:103E60008DEC23F0E9EC24F001E1E55126E00CECC7
:103E700026F010508DEC23F0EF50D880E45508E286
:103E80000CEC26F01050EA6A470FE96E000E08D0DD
:103E900010508DEC23F0EFCFE4F40F5007EC26F038
:103EA000EA22EF50E45D116E1350115C06E291EBD3
:103EB00013F00FEB2BFF10EB2CFF102AC8D70F2AA3
:103EC000B7D7CEEC23F00F01320E0C6F0D6F0E6FD3
:103ED0000F6F106F03EC26F0320EE66E4AEC26F000
:103EE000320EE66E040EC0DB320EE66E050EBCDB53
:103EF00061EC25F0060E22EC26F0080E22EC26F0EE
:103F00000A0E22EC26F000010D6B0E6BF1D0280E8C
:103F10008DEC25F060E3780E93EC23F05CE2000179
:103F20001D511B5D1E511C5902E2010E01D0020EF3
:103F3000126EA5DBCFEC24F00CE266EC25F004E277
:103F400011500F010C2703D00F01640E0C6F0CCF22
:103F50000DFF95DB0401F0EC24F00BE27EEC25F084
:103F600004E211500F010C5F02D00F010C6B0CCF5B
:103F70000DFF0CCFE6FF12EBE6FFBCEC3BF042E995
:103F8000030E126E1250050801E2B2D078DBCFECBE
:103F900024F00AE266EC25F004E2A0DB1150EF26E3
:103FA00003D09CDB640EEF6E6ADBF0EC24F009E2D8
:103FB0007EEC25F004E292DB1150EF5E02D08EDB46
:103FC000EF6A8CDBEFCFE6FF12EBE6FFBCEC3BF0D9
:103FD00042E9122AD7D7780E8DEC25F019E3880E26
:103FE000A2DB16E239EC25F0ED22060E42DB1F5172
:103FF000EE262051ED22080E3CDB2151EE26225107
:10400000ED220A0E36DB2351EE262451ED2270D02C
:10401000880E18EC26F06CE1E551031869E1DDEC3F
:1040200025F004E00401C2EC24F0FDE192EC25F05F
:1040300004E00401C2EC24F0FDE1E4C41DFF1CCF48
:1040400024FFE4C425FF0F010A510B6E0C6A0E51C8
:104050005A0816E21651E6DB060E10EC26F004E0D4
:104060000401F7EC24F0FDE11DDB0AE29AEC24F0F8
:104070000F0109501E5D000E0A5402E209EB1EFFFB
:104080000F010F515A0816E21751CCDB080E10EC45
:1040900026F004E00401F7EC24F0FDE103DB0AE282
:1040A0009AEC24F00F0109501F5D000E0A5402E241
:1040B00009EB1FFF0F0110515A0816E21851B2DB2D
:1040C0000A0E10EC26F004E00401F7EC24F0FDE108
:1040D000E9DA0AE29AEC24F00F010950205D000EA3
:1040E0000A5402E209EB20FF0001009300950099B9
:1040F00050E9E7CFD9FF1200420E0B01965D08E1AF
:104100008150020B0EE08150040B0BE0966B120005
:10411000E00E961506E0E66A0B0EE7DA0B01420E9A
:10412000966F120043DB46E80B0196A981D0150E6D
:10413000965D75E10F01F40E056F010E066FB0EC90
:1041400024F00E01070E086FA2DBC40EE66E600EAF
:1041500013EC26F00E0104510511061107115FE161
:104160000A0ECEDBC1EC7AF0A9DB056EE551066ED6
:1041700005500F01075D0401E46F06500F01085957
:104180000401E56FE4510E010A5D0401E5510E01E1
:104190000B5945E3070EE96E0F0EEA6E0401EE506F
:1041A0000524E66FED500620E76F0E010A51040169
:1041B000E65D0E010B510401E75931E30CCEE6FF39
:1041C0000DCEE6FFE66AE66A140E9ADB99EC7BF008
:1041D0001FEC7BF073DBEBDB01EBE4F402EBE5F4CB
:1041E00003EBE6F404EBE7F4E42B000EE523E6230F
:1041F000E723D890E733E633E533E433E451D7DB04
:1042000001EB05FF02EB06FF0F01006B54EC46F0DB
:10421000E66A090E6ADA0B01966B010E0AD0120EDD
:104220000B01965D03E0E66A0A0E5FDA0B01966BFE
:10423000000E47E9E7CFD9FF1200B8DA57E80B01C3
:10424000965101E026D181B424D163EC42F081B2D1
:1042500020D10EEC27F089EC25F0B4DB106A016A5E
:10426000026A036A046A176AB9EC39F0EBEC66F08B
:1042700046EC25F00001C0DB320E7ADA49DB0D6E28
:10428000F4500E6EF00E0B01961501E0DFD01750C2
:104290001FE0F29ED650156ED750166EF28E0401B6
:1042A0001350155CE46F14501658E56FD890123017
:1042B000E76F1130E66FD890E733E633E451E65DFF
:1042C000E551E75905E2176AE66ACBEC3AF041E9B5
:1042D0000001655101E1ACD0F29E656B6651136E31
:1042E0006751146E7451116E7551126EF28E010E7B
:1042F000176E4DDB02E1F4500C1802E00B01968FB3
:10430000010EE66ECBEC3AF041E97BEC3AF00B01A2
:10431000965110E1000125510B1801E089D026517A
:104320000C1801E085D000010083380E0013B7D9C6
:10433000010E49D096050CE104DBB3DA01E3106A03
:104340005BDBD3DA75E1E5510C1872E167DB3BD03A
:10435000020E965D19E130DA02E33FDA03E2CFECB8
:1043600025F031D09EDA01E3106A46DB1307000E18
:10437000145B1507165B1707185B8150020B58E09A
:104380008150040B55E052D0030E965D1EE1EADB2E
:1043900000012951091805E12A510A1802E100011A
:1043A000008100013051091805E131510A1802E17C
:1043B000000100858150020B3BE08150040B38E086
:1043C0003BDA36E2F3DB966F33D0040E965D30E1D4
:1043D000C2DA00012B51091805E12C510A1802E13B
:1043E0000001009100012E51091805E12F510A1812
:1043F00002E10001009300013251091805E1335137
:104400000A1802E10001009500013651091806E181
:1044100037510A1803E1C70E000100171CDA08E340
:104420000001005103E13BD9050E966F0B019689FF
:10443000AEEC2AF0000902E10B01968B8ADB01E663
:10444000C8DB01E31FD70B01968D1CD7DADA150EF6
:104450000B01965D1AE10F6A00012D510F5C17E206
:10446000CBDBEF50E66E0F500001EA6A0325E96EE0
:104470000451EA22E552E750EF6E102A00012D5157
:10448000105C01E3106A0F2AE7D7B9EC39F063EC4E
:1044900042F058E9E7CFD9FF1200420E0B01965DBA
:1044A00008E18150020B0EE08150040B0BE0966B8B
:1044B0001200E00E961506E0E66A060E16D90B010C
:1044C000420E966F12000B0196A956D0150E965DFE
:1044D00051E146DA91EC68F033EC69F050EC6AF0A7
:1044E00017EC6BF031EC36F02AEC40F0E0EC3CF0ED
:1044F000CED9C20EE66E600E96DBD0EC6BF0F3CF39
:10450000E4F4F4CFE5F40401F350F41004E008CE31
:10451000E6FF030E2ED0EED8FC0EE417CAD903E155
:10452000E66A050E26D0E6D8F00EE517C2D902E1FC
:10453000010E1DD0DFD80F0EE517BBD902E1020E28
:1045400016D0D8D80F0EE417B4D902E1030E0FD05D
:10455000D1D8F00EE617ADD903E1040EE66E09D00E
:10456000C9D8E69BA6D902E1060E01D0050EE66E7B
:10457000040EBBD80B01966B120018D944E8036AED
:10458000046A0B01965153E181DA320EF1D80EEC38
:1045900027F0BED9016EF450026EF00E0B01961595
:1045A0003CE10001655121E0656B032A000E042205
:1045B00003EBE4F404EBE5F4E4C4E6FFE5C4E6FF52
:1045C00087EC28F0E552E7CFE5F4E552E7CFE4F4D5
:1045D000F3CFE6F4F4CFE7F40401F350E41902E179
:1045E000E751E51902E00B01968FAEEC2AF00009C5
:1045F00002E10B01968B8FEC2BF004010150F35C70
:10460000E46F0250BBD805E6D880B80EE4550B0E17
:1046100061D9C3E20B019689C0D7F3D9E00E0B0133
:10462000961503E0E66A060E60D80B01966B45E925
:10463000E7CFD9FF1200C1EC7AF0E552E5CFEFF4F5
:10464000E5CFEEF4E5CFEDF4E7CFECF40401EC5167
:10465000E85DE46FED51E959E56FEE51EA59E66F17
:10466000EF51EB59E76F1200E66EBCEC3BF042E90C
:1046700012000024E96E000E0120EA6E120077DAC3
:10468000EECFE4F4EFCFE5F412507BDAEF501200F6
:10469000125077DAEF50E66FE76BB7EF25F092DA5A
:1046A0000B0112000401E651075CE46FE751085862
:1046B000E56FE4C4E6FFE66E65EC7BF0D9DA0E6EDA
:1046C000E7500D6E07500D5C08500E58120005247F
:1046D000E46F000E0620E56FE45112001250EA6A02
:1046E0000B0FE96E0F0EEA221200E66EFDEC42F0AF
:1046F00042E9120004CEE4F405CEE5F406CEE6F479
:1047000007CEE7F412000F5082DAEA221200040109
:10471000EA6BEB6B640E3DEF26F0EA6A470FE96E39
:10472000000EEA2212005BDA025CE7510358120025
:10473000E56F00DAE451116E1200EECFE8F4EFCF2E
:10474000E9F40401040EEA6FEA51E8C4E6F4E9C4AE
:10475000E7F4120007DAD9500F0FE66EDACFE6FF62
:1047600009EBE6FF0AEBE6FFD2EC1DF044E912008C
:10477000E66EE66A9AEC2BF042E91200F458E56F17
:10478000E66BE76BE735000EE7191200040EE86FE1
:10479000E851E6C4E4F4E7C4E5F412002CCFE6FFE8
:1047A0002BCFE6FF8EEC3BF042E91200D9CFE6FFBB
:1047B000E1CFD9FF81E912000F0134510401012436
:1047C000E46F000E0220E56F00011F510401E45D5B
:1047D000000120510401E55912000F013451040178
:1047E0000324E66F000E0420E76F0001235104014B
:1047F000E65D000124510401E759120002EBE6FFD7
:1048000014EC3CF041E90426000E0522012A1200B6
:104810000850065CF06F09500758F16FF0C4E6FFCE
:10482000E66E1200076E086A0BEBE6FF0CEBE6FF84
:10483000640EE66EE66A120000013451275D040141
:10484000E46F0001355128590401E56F0950E45D1A
:104850000A50E55912000001275134250401E46F84
:104860000001285135210401E56FE451095CE5514F
:104870000A581200040104380F0BE46F0538F00BDE
:10488000E41305380F0BE56F0250EA6A1200C80EF8
:10489000E66E600EC8D997CBE6FF1FEC64F041E9E5
:1048A0001200AAD91BC0EFFF102A00012D51105C85
:1048B0001200E451E511E611E7111200E552E5CFCF
:1048C000E7F4E5CFE6F4E5CFE5F4E7CFE4F404015F
:1048D000E4511200E555000EE655000EE7551200B2
:1048E00056D9F458E56FE451120025C0E4F426C00F
:1048F000E5F40401D890E437E537E4510B181200D1
:10490000BCD907CFE6FF08CFE6FFE66AE66A1200E9
:1049100003CFE6FF04CFE6FF52EC2AF042E98FEC2A
:104920002BF0F35012008FEC2BF0F350046EF45088
:10493000056E12000D50075C096E0E5008580A6E85
:10494000120000011F51012620510222235103268B
:1049500024510422120007500B5C096E085082D1CA
:10496000F0EC66F017EC67F0C6EC67F035EF68F036
:1049700025C0E6FF26C0E6FF1200EECFE6F4EFCF3B
:10498000E7F41200D890E533E433E80412000B2A70
:10499000000E0C2287EC28F0F3500B1812000401D3
:1049A000E66FE76BE451E65DE551E7591200016EF1
:1049B000E551026EE651036EE751046E120002509B
:1049C000C1EF25F0056A066A076A086A0B6A0C6A75
:1049D0001200EF500401E46FE56BFF0EE4191200C2
:1049E000E66FE76BE651E45DE751E5591200D890B8
:1049F000E733E633E80412002D5100010F6F106B0E
:104A00001200000EE66EE66A52EC2AF042E9E66A0F
:104A1000E66A8EEC3BF042E942EF26F0A9DF01EBBB
:104A2000E6FF02EBE6FF24D9026EE750016EA0DF3D
:104A300003EBE6FF04EBE6FF1BD9046EE750036EC1
:104A40002EDE020E1200096E0A6A07EBE8F408EB8C
:104A5000E9F45DDE0BEBE6FF0CEBE6FF0950075CCB
:104A6000F06F0A500858F16FF0C4E6FFE66E26EFCB
:104A700026F0020EFEDD00011B51EE261C51ED2238
:104A8000040EF7DD1D51EE261E51120087DE0CCFFD
:104A9000E6FF010EE9DD0ECFE6FFFCD80FCFE6FF03
:104AA000040EE2DD10CFE6FFF2D0086E096AD4D81A
:104AB0005F0EE3D8ADDEE66AE66A99EC7BF01BEFA9
:104AC00023F0020EBFD8040E22EF26F0E1DDE651FE
:104AD000EE5CE46FE751EE582BDE640EE46FFEDD12
:104AE000EF50E45D115C1200640EE66ED3D8640EE4
:104AF000E66E040EB9DD640EE66EC9D0C9DDEE5077
:104B0000E65DE46FEE50E75913DEE8DDEF50115C2F
:104B10001200E66A020E75EF23F0D9DD025CE55162
:104B200003581200E4C41CFF040EA3DD26DF0401B9
:104B3000C6EF23F0D890E533E433D890E533E4337F
:104B400012000B01010E956FE66A080ECEDDBDEF77
:104B500028F08FEC2BF004010D50F35CE46F0E5045
:104B6000BEEF23F005500B5C096E06507BD0EA6A5D
:104B70001234FE0BE96EEA36190EE926000EEA221F
:104B80001200EA6A230FE96E0F0EEA2212008FEC80
:104B90002BF004010450F35CE46F055012008BEB22
:104BA00005F08CEB06F07BDD030E12008BEB07F0BB
:104BB0008CEB08F074DD040E1200020E5ADDDDDE0F
:104BC000C6EF23F08FEC2BF0F3500D6EF4500E6E09
:104BD0001200D880D00EE455070E6AEF24F00524A9
:104BE000E66F000E0620E76FE651120042DDEECFC1
:104BF000E4F4EFCFE5F412001050EA6A880FE96E92
:104C0000000EEA221200E66E010E34EF23F0EA6A8B
:104C1000430FE96E000E120076DDEFCFE4F41200D0
:104C200028DD9DEF23F0E66EF4EC4BF042E9120034
:104C30004EDD02181200E66A2DD8E66A040E14DD75
:104C4000E66A25D016DDEE6AED6A120065EC7BF0AF
:104C5000E66AE66A1BEF23F006EBE8F407EBE9F4FB
:104C600087EF23F00C580A6E092A000E0A22120060
:104C700085EC7AF0E552E5501200E66EE66AE66AE7
:104C8000E66A1200E66A010EEFDC1BEF26F0050E65
:0A4C900034EF23F0030E34EF23F09D
:064C9A0053EC2EF082E94C
:104CA00043E800502BE078EC2EF0EECFE4F4EFCFA9
:104CB000E5F404010A0EE8EC2FF06BE28450040BDB
:104CC00001E0010E026E02500001DE5D62E002EBC7
:104CD000DEF002505EE078EC2EF0EE2A000EED22BF
:104CE000EECFE4F4EDCFE5F404010A0EE8EC2FF08A
:104CF00050E3E8EC2EF0010EEF6E4BD0DF0EA3EC8C
:104D00002FF028EC5AF00009FCE10AEC5AF070ECA4
:104D10002FF003502F08020E045407E2AB0E035C81
:104D2000020E045802E2026A09D03E0E035C000E35
:104D3000045802E2020E01D0010E026E0250000180
:104D4000DF5D0AE002EBDFF0A9EC2FF078EC2EF04B
:104D5000F3CFEEFFE5C4EDFFE8EC2EF0EF50025C80
:104D600018E08FEC2BF078EC2EF0EE500401F35CA1
:104D7000E46FEE50F458E56FE451D008070EE555A6
:104D800008E2E8EC2EF002EBEFFF78EC2EF0EE6A92
:104D9000ED6AE8EC2EF0EF5044E9E7CFD9FF1200BE
:104DA000700ED3129B8C020EE66EFAEC59F041E9BC
:104DB000FC0ED316E66AF00EE66E040EE66EEB0EFF
:104DC000E66E93EC57F044E9170EE66EACEC59F042
:104DD00041E9C50EE66E6CEC59F041E9040EE66E51
:104DE000C7EC59F041E99380958E8484978C848632
:104DF00096968490969084929692829694969F80AE
:104E0000D08EF28EF28C98820F01140E5F6F0B0120
:104E10009C6B0B019D6B0B019E6B12000F013F51B0
:104E200001E11200000160AF859C12008350800BED
:104E300002E0800E01D0000E0001606F60AF02D072
:104E4000978C02D0979C859CDA6BDB6B460EDC6FEF
:104E5000050EDD6FD96B010ED86FDE6BDF691200B6
:104E600020EC30F041E8016A010EE66E080EE66EB5
:104E7000BCEC3BF042E98496190E0BEC2FF0A2EC4F
:104E80004CF000090CE1012A030E015C08E2B0ECD1
:104E90002FF0190EE66EE66A9AEC2BF0EBD7030EB4
:104EA000015C02E3000E01D0010E42E9E7CFD9FF19
:104EB0001200B0EC2FF0E66A080EE66EBCEC3BF098
:104EC00042E9190E0BEF2FF020EC30F046E8016AB2
:104ED0000F013F5102E1000E7BD08350046E04505D
:104EE00000016019800B0EE0010ED86F800E0414D3
:104EF000606F04AE02D0978C01D0979CDA6BDB6BAD
:104F0000010E016E04AE22D0E66AC7DE41E9036EEF
:104F10000001DE6BD96B0B019A6B9B6B020E035C7D
:104F200005E1000160B553D060850DD0000160A59A
:104F300004D0FA0E6017010E016E035048E1010E15
:104F4000601545E16081010E016E41D0010EE66EF3
:104F5000A4DE41E9026E020407E1020E00016015C1
:104F600003E16083010E016E0001DA51DB1106E1FD
:104F7000D6DBF3CFDAF0F4CFDBF029D02CEC2FF036
:104F8000DA0EE96E000EEA6E0401EE50055CE46F85
:104F9000ED500658E56FE4510001DC5D0401E55178
:104FA0000001DD5914E205EBDAF006EBDBF0460E0A
:104FB000DC1908E1050EDD1905E11E0EDC6FDD6B65
:104FC000858C05D0460EDC6F050EDD6F859C01508B
:104FD00075EF2FF06EDFF29EF29CF19CF292F29848
:104FE000F198F08EF092F098A198D38E0300F250D1
:104FF000020B06E1F050020B03E1A150100B01E09F
:1050000002D062DFF3D7D39EA098F098F298F28E88
:10501000F28C26DF12008292949286949894978460
:10502000C088C18EC0980001616B770EE66EF9EC06
:1050300057F041E9F86AB7EF2FF0A19CA09C720EDF
:10504000E66E060EE66E01CFE8F402CFE9F4040145
:10505000390EE85F030EE95B040EE8C4E6F4E9C428
:10506000E7F4000A06E00401D890E637E737E804E1
:10507000FBE1E6C4E6FFE7C4E6FF85EC7AF010EC5E
:105080002FF0E4C462F000016229636F240ED16E38
:10509000C088800E6311776EC09883EC2FF0666B2A
:1050A000676B686B696B6A6B6B6BBEEF2FF0868406
:1050B000BC0ED16E8BEC2FF00BEC2FF06AA204D05B
:1050C0008BEC2FF0646F07D0C088800E0001631155
:1050D000776EC098646B83EC2FF0F29ED6CF66F0AB
:1050E000D7CF67F0F28E66C068F067C069F066C01F
:1050F0006AF067C06BF0BEEC2FF0A19CA28CA08C74
:105100001200240ED16EA19CA09C8694120020EC6B
:1051100030F042E8F29E00017651016E7751026E46
:10512000F28ED1EF2EF023EC30F0F29E00EB76F011
:1051300001EB77F0F28E41E9E7CFD9FF120020ECC6
:1051400030F042E8DEDFC088C19EC0988684020E3F
:105150000BEC2FF0BF0EA3EC2FF028EC5AF0000957
:10516000FCE10AEC5AF0F350016EF450026EC08874
:10517000C18EC0988694D1EF2EF020EC30F064E818
:10518000026A0001070E626FE828636FC2EC2EF01E
:10519000216A226A236A246A1D6A1E6A1F6A206ABB
:1051A0002CEC2FF070EC2FF039DE2C0EE66E010E99
:1051B000E66E78D942E9025001E01AD1000165514A
:1051C00001E114D1656BF29E6451016E010406E1A8
:1051D0006A51685D0B6E69516B5505D068516A5D07
:1051E0000B6E6B5169550C6EF28E36EC2FF0E4515C
:1051F000FA08000EE55513E2010409E193EC2FF0E3
:10520000190FF3EC2EF0092A000E0A2208D093ECB5
:105210002FF0150FF3EC2EF0072A000E08227FDA8C
:1052200004010550F35CE46F0650F458E56FE45157
:10523000E808030EE55502E2020E026E075032083E
:10524000000E085406E309503208000E0A5401E328
:10525000CDD02CEC2FF007EBE6FF08EBE6FF16ECC9
:105260002FF040EC30F0186EE550176EE550166EDA
:10527000E750156E09EBE6FF0AEBE6FF21EC2FF095
:1052800040EC30F01C6EE5501B6EE5501A6EE75096
:10529000196E26EC30F016EC2FF099EC7BF0FCEC5C
:1052A0002FF00D6EE5510E6EE6510F6EE751106E48
:1052B00026EC30F021EC2FF099EC7BF0FCEC2FF099
:1052C000116EE551126EE651136EE751146E9DEBAF
:1052D00021F09EEB22F09FEB23F0A0EB24F00DEBEE
:1052E000E8F40EEBE9F40FEBEAF410EBEBF4D95031
:1052F000110FE96EDACFEAFFEE50E85DE46FEE5091
:10530000E9599BEC2FF0E4511D6EE5511E6EE651FC
:105310001F6EE751206EC2EC2EF0203431E2D6EC45
:105320002EF02EE2243408E20F0E0001635D5CE2F1
:10533000F29E622B632B32D0243406E2DFEC2EF097
:1053400003E24CEC2FF002D0ECEC2FF0203406E21C
:10535000D6EC2EF003E255EC2FF002D08BEC2EF0C1
:105360000401EB35E751EB1902E65EEC2FF03CE26D
:105370000F0E0001635D38E2F29E622B632B33D087
:10538000203432E3243402E2DFEC2EF009E30001A2
:105390006251000829E2F29E62076307F28E26D06E
:1053A000243406E2DFEC2EF003E24CEC2FF002D0C6
:1053B000ECEC2FF0203406E2D6EC2EF003E255ECB4
:1053C0002FF002D08BEC2EF00401EB35E751EB19F6
:1053D00002E65EEC2FF008E200016351000804E2EF
:1053E000F29E62076307F28E010E026EB7D8E3D613
:1053F000000EE66EE66A56D842E902042CE104018A
:10540000390EE46F030EE56FE66BE76B0001635145
:105410006225B3EC2EF0390EE66E030EE66E32EC2A
:105420002FF00DEC30F0040E0401D890EB33EA338A
:10543000E933E833E806F9E10401E851E427E951EA
:10544000E523EA51E623EB51E723E4C401FFE5C479
:1054500002FF010E01D0000E65E9E7CFD9FF12006F
:1054600053EC2EF082E942E80050640802E2640E38
:10547000006E190EE66EE66A0050E66EE66A2DECE6
:1054800030F0036EE750026E02EBE6FF03EBE6FF3F
:10549000BBEC58F042E945EF30F080C0F3FF81C02B
:1054A000F4FF120023EC30F000EBE4F401EBE5F440
:1054B0000401E66BE76BE735000EE71909E6D880D3
:1054C000EE0EE455020EE555000EE655000EE755CA
:1054D00004E2EE0E006E020E016E00EBE4F401EB4E
:1054E000E5F4E66BE76BD890E751000A07E6FA0EA1
:1054F000E8EC2FF0000EE659000EE75926E3000114
:1055000061511CE1D4DD0001806B816B826B836B88
:10551000846B856B866B876B02D9F3CF7CF0F4CFFD
:105520007DF00001640E7C5F000E7D5B6C6B6D6B2B
:10553000706B716B6E6B6F6B726B736B00EB7EF0ED
:1055400001EB7FF0010E616F05D0DBDDB7EC2FF0D2
:105550000001616B41E9E7CFD9FF120020EC30F088
:105560004FE80D6A0001615101E1D0D0D8D8F35065
:10557000096EF4500A6E7C0EE96E000E67EC2FF097
:10558000020EE8EC2FF001E2C1D009EB7CF00AEB4F
:105590007DF0F29E00016651056E6751066E7451F2
:1055A000016E7551026E7651036E7751046ED650BE
:1055B0000E6ED7500F6EF28E610506E109EB7AF0A0
:1055C0000AEB7BF0020E616F03500208000E0454D8
:1055D00020E2015002101DE005500E5C076E0650DF
:1055E0000F58086E0750015C0850025804E287EB20
:1055F00001F088EB02F01BEC30F01B0EE66EB70EEC
:10560000E66E85EC7AF0E552E5CF81F0E7CF80F0E9
:1056100002D0806B816B020E0001D89081BF03D055
:10562000805D000E81590CE27A0EE96E000E67EC87
:105630002FF0E451FA08000EE55502E2010E0D6E5E
:10564000000180517E5D826F81517F59836F82C0DE
:10565000E6FFE66E0A0EC3DBE3DB84C0E6FF85C02F
:10566000E6FF040EBCDBE552E5CFE7F4E7CFE6F456
:105670000401E451E6250001866F0401E551E721AC
:105680000001876F200EC5EC2FF03DEC7AF0E5525B
:10569000E5CF87F0E7CF86F00001873508E2865135
:1056A0006408000E875503E2640E866F03D08735C9
:1056B00003E3866B876B1BD082518427835185233C
:1056C000853509E28451E808030E855504E2E80EA9
:1056D000846F030E856FD880855104E7180E845DB2
:1056E000FC0E855904E2180E846FFC0E856F190EAE
:1056F000C5EC2FF02DEC30F00C6EE7500B6E0BEB81
:10570000E6FF0CEBE6FFBBEC58F042E90D5002E07F
:10571000000E01D0010E50E9E7CFD9FF120020ECB6
:1057200030F042E8F29E0B019351016E9451026EEB
:10573000F28E37D323EC30F044E8A9EC2FF00401CB
:10574000CFDB056A066AEBDFF3CFE8F4F4CFE9F4C8
:105750000401EA6BEB6BD950030FE96EDACFEAFF75
:10576000EE50F35CE46FEE50F458E5DB00EBECF444
:1057700001EBEDF4EE6BEF6BEC51E45DED51E559AF
:10578000EE51E659EF51E75906E2010EE66EFAECEA
:1057900059F041E9D8D749EF30F023EC30F046E832
:1057A000BEDF9EDBCCEC2FF085EB07F086EB08F03C
:1057B0005DDB0050E45D0150E55913E2EDDB07507D
:1057C000055CE46F08500658E56F060EE8EC2FF014
:1057D000EFE3827685EB07F086EB08F0C0EC47F04C
:1057E000E7D783D323EC30F044E8050EBCDADBDBEB
:1057F00002EF30F023EC30F044E8D5DB140EB3DADE
:1058000002EF30F023EC30F046E8046A100E056E2B
:10581000270E066E880E076E000E086E08EC30F03C
:10582000EF5004E0072A000E0822F8D701340EE3F7
:105830009FDA2D0EEF6EE668E6685CEC30F065EC02
:105840007BF0E552E550016EE750006E0550061002
:1058500031E04FDB5CEC30F034EC30F0036E49DBD0
:105860000350BDDAFE0EE350005E41E9E550015AF7
:10587000035005E1640E051804E1065002E1010E33
:10588000046E045003E0300E0324F4DB640E0518AC
:1058900005E1065003E16CDA2E0EEF6E0A0EE66E9D
:1058A000E66A27DB3DEC7AF0E552E550066EE750FC
:1058B000056ECCD7ADDBEF6A18D3F5D984E946E89D
:1058C000056A100E066E270E076E880E086E000E13
:1058D000096EE3DBEF5004E0082A000E0922F9D735
:1058E00002340EE34ADA2D0EEF6EE668E668A3DBBB
:1058F00065EC7BF0E552E550026EE750016E05D095
:10590000005003E03ADA200EEF6E0650071030E048
:10591000C9DB91DBA9DB046EC5DB045060DAFE0E47
:10592000E350015E41E9E550025A045005E1010EE1
:10593000061804E1075002E1010E056E055007E06C
:10594000300E0424E66E19DAE552E75004D0005018
:1059500003E013DA200EEF6E0A0EE66EE66AA2DBB3
:105960003DEC7AF0E552E550076EE750066ECDD774
:1059700094DBEF6ABAD297D989E944E80A6A880EBB
:105980000B6E000E0C6EBADAEF5004E00B2A000E1C
:105990000C22F9D7005001100210031034E0DDD9B9
:1059A00004EBE6FFA6DA07EBE6FF26DB096ED5D9A6
:1059B00009EBE6FFE66A56DA6CD9D950040FE96EB6
:1059C0001EDA095002E0010E0A6E0A500AE0300E9B
:1059D0000924E66E93DA0B2A000E0C22E552E750FA
:1059E00005D08CDA0B2A000E0C225F0EEF6E0A0E29
:1059F000BAD9B3D945DB036EE550026EE550016EAE
:105A0000E750006EC7D77ADAEF6A43D34CD985E9FD
:105A100048E8066A880E076E000E086EF9DAEF5045
:105A200004E0072A000E0822F9D7010E096E0A6A5F
:105A30000B6A0C6AFCDA99EC7BF041E9E73403501D
:105A4000E7180BE6FD0EE350005CFE0EE350015834
:105A5000FF0EE3500258E750035843E905E3E7DA45
:105A600099EC7BF00CDAE6D709500A100B100C10F9
:105A700015E048D972D9C0DA056E44D905EBE6FFC6
:105A8000E66AF0D906D9D9CFE9FFB9D9300E052495
:105A9000F1DACDDAC1EC7AF0F2D9E6D7B9DAEF6A09
:105AA00049E9E7CFD9FF1200FED884DA8ADA02E0AA
:105AB00042D9FCD7EED1F7D87DDAF9DAEF5004E01D
:105AC000032A000E0422F9D77CDA02E034D9FCD78D
:105AD000E0D1DACFE4FFE2CFDAFFE652D9CFE6FF3A
:105AE000E1CFD9FF81E944E89EA00AD09E90D10E73
:105AF000CF6E390ECE6E0B01932B000E94230AD07D
:105B00000000000000000000000000000000000095
:105B100000000000A150400B01E1B4D0A050400BA8
:105B200001E1B0D0D6CF66F0D7CF67F00001645165
:105B300055E1000168510001665D016E6751000189
:105B40006955026E00016A510001665D036E67517E
:105B500000016B55046E01502E08000E02543DE208
:105B600003501708000E045438E2C088800E00016C
:105B70006211776EC0980001010E646F0001010E82
:105B8000656F0001762B000E77236CC070F06DC03E
:105B900071F093CB6CF094CB6DF00001705100016B
:105BA0006C5D00015E6F0001715100016D590001D3
:105BB0005F6F0001E80E5E5D030E5F5905E201EBC9
:105BC00074F002EB75F005D00001C10E746FB60ED3
:105BD000756F66C068F067C069F053D000016A5104
:105BE0000001665D016E675100016B55026E000198
:105BF00068510001665D036E675100016955046ECE
:105C000001502E08000E02543CE203501708000E0B
:105C1000045437E2C088800E00016311776EC0988B
:105C20000001646B0001010E656F0001762B000E10
:105C300077236EC072F06FC073F093CB6EF094CB8D
:105C40006FF00001725100016E5D00015E6F000196
:105C5000735100016F5900015F6F0001E80E5E5D36
:105C6000030E5F5905E201EB74F002EB75F005D00D
:105C70000001C10E746FB60E756F66C06AF067C022
:105C80006BF0A19C45E9E7CFD9FFE552E5CFDAFFFC
:105C90001100E552E5CFE7F4E5CFE6F4E5CFE5F412
:105CA000E7CFE4F41200D9CFE6FFE1CFD9FF12002D
:105CB0000401E451036EE551046EE651056EE751AF
:105CC000066E03EBE4F404EBE5F405EBE6F406EB17
:105CD000E7F4E42B000EE523E623E723D890E7332F
:105CE000E633E533E433E4C4F3FFE5C4F4FFD1D194
:105CF000EA6A0034FE0BE96EEA36980EE9260B0ECE
:105D0000EA22120009EBE6FF0AEBE6FF0BEBE6FFE7
:105D10000CEBE6FF1200E668E668E668E6681DEB55
:105D2000E6FF1EEBE6FF1FEBE6FF20EBE6FF99EC3C
:105D30007BF00DEF30F000EBF6FF01EBF7FF002AF0
:105D4000000E01220800F550E66EB1D9032A000EBC
:105D50000422E552E750EF6E120000EBE6FF6BD92C
:105D600003EBE6FF1200E66EE66AE66AE66A1200F8
:105D70004FD9072A000E082212008FD9082A000ED8
:105D800009221200196A1A6A1B6A1C6A156A166AC5
:105D9000176A186A096A0A6A89EB07F08AEB08F041
:105DA000120001EBF3FF02EBF4FF6FD11D5000086E
:105DB000000E1E54000E1F54000E205412002150DD
:105DC0000008000E2254000E2354000E245412002A
:105DD0000050EA6AD80FE96E000EEA221200E66E61
:105DE000E66A65EF7BF0E96EDACFEAFFE451EE2672
:105DF000E551EE22E651EE22E751EE221200DACF13
:105E0000EAFF0401E451EE5EE551EE5AE651EE5A26
:105E1000E751EE5A1200E66EE66A8CDC42E91200A7
:105E2000E552E5CFE5F4E7CFE4F41200E66AE66A6E
:105E300015EBE6FF16EBE6FF17EBE6FF18EBE6FFC8
:105E40001200E66AE66A19EBE6FF1AEBE6FF1BEBC7
:105E5000E6FF1CEBE6FF120062DCF350056EF45027
:105E6000066E1200E66AE66A99EF7BF058DC0401E0
:105E70000350F35CE46F0450F458E56F1200E552F0
:105E8000E5500C6EE5500B6EE5500A6EE750096E5A
:105E900012000DD9EF6AF9D021EBE4F422EBE5F41E
:105EA00023EBE6F424EBE7F412001DEBE8F41EEB21
:105EB000E9F41FEBEAF420EBEBF41200E851E45DA7
:105EC000E951E559EA51E659EB51E7591200EA6EFA
:105ED0000401EE50095CE46FED500A58E56F1200C2
:105EE000F350036EF450046E120047E9E7CFD9FF78
:105EF000120005EBE6FF06EBE6FF12000BEBE9FFF5
:105F00000CEBEAFF12000F0EE66E16EC5AF041E9B8
:105F10000001656B1200C088800E00016211776E6F
:105F2000C098010E12000BEBE4F40CEBE5F4E66B09
:105F3000E76BD9501200E56FEE50EA59E66FEE506C
:105F4000EB59E76F1200E66EE1EC59F041E92EEFF4
:105F50005AF08FEC2BF0F3CFE4F4F4CFE5F4120019
:105F60008486958C958A95880F0E95121200000EE6
:105F7000E66EE66ABBEC58F042E91200766B776B8E
:105F8000746B756B786B796B1200E66EE66A86C08F
:105F9000E6FF87C0E6FF1200F29ED650056ED7508E
:105FA000066EF28E120005CFE6FF06CFE6FFE66A28
:105FB000E66A120083E942E8880E036E000E046E62
:105FC000120000EBF6FF01EBF7FF0800F55012009E
:105FD000E45D000EE5591200E668E668E668E668EA
:105FE00021EBE6FF22EBE6FF23EBE6FF24EBE6FFE7
:105FF00099EC7BF049EF2EF0C1EC7AF04ADE040117
:10600000E451120059D82EDF1FEC7BF042DE50D64F
:1060100007EBE9FF08EBEAFF1200E552E5CFEBF4EE
:10602000E5CFEAF4E5CFE9F4E7CFE8F412000A0E91
:106030009ADE82EF2EF001EBE6FF02EBE6FF1200A4
:1060400032DE81E912002FDE83E91200640E8BDE5E
:10605000550EE66E080EE66E1200780EC0DE85EC78
:106060007AF0E552E55012003DEC7AF0D9DE0401F9
:10607000E4511200E66E7CDEE552E750EF6E12004E
:10608000C1EC7AF0E552E550120043E9E7CFD9FFC1
:10609000120045E9E7CFD9FF120008EBE9FF09EB51
:1060A000EAFF120006EBE6FF07EBE6FF120003EB48
:1060B000E9FF04EBEAFF120000EBE6FF01EBE6FF6D
:0260C0001200CC
:0E60C2003E000D0A3E000D0A006F6F006F20B9
:1060D000002073006E0046554C4C005245504C4118
:1060E00059204555520045555200082008002042CD
:1060F000504D3A4641494C002042504D3A474F4F8F
:10610000440020424154454E3A0020733D00206E29
:106110003D002053554D454E3A00204348474354D7
:10612000524C3A0020504C55473A00204241544CC2
:1061300045563A0020535442454E3A002073002001
:1061400053544442593A00205265706F72744C6542
:1061500076656C3A00202D20496E74656E73697403
:1061600079204D696E202D3E2000202D20496E742F
:10617000656E73697479204D6178202D3E20002072
:106180002D205769647468204D696E202D3E2000D3
:10619000202D205769647468204D6178202D3E20A1
:1061A00000202D20506F736974696F6E204D696EE9
:1061B000202D3E2000202D20506F736974696F6E72
:1061C000204D6178202D3E2000204D61676E657462
:1061D0006963205468726561643A0D0A0020547244
:1061E000616E73702E205468726561643A0D0A0006
:1061F00020486F6C6F6772616D3A0D0A002049523A
:10620000205A6F6E653A0D0A000D0A203530302095
:106210004555524F000D0A20323030204555524F1F
:10622000000D0A20313030204555524F000D0A2014
:106230003530204555524F000D0A2032302045554B
:10624000524F000D0A203130204555524F000D0AA3
:106250002035204555524F0020496E76616C6964A7
:106260002066656174757265002053656C656374A2
:10627000202D3E2000202D20284D29204D61676EC5
:1062800065746963205468726561640D0A00202D8D
:1062900020285429205472616E73702E2054687225
:1062A0006561640D0A00202D2028482920486F6C64
:1062B0006F6772616D0D0A00202D20284929204941
:1062C00052205A6F6E650D0A002046656174757222
:1062D00065733A0D0A0020496E76616C696420622C
:1062E000616E6B6E6F74652064656E6F6D696E6153
:1062F00074696F6E0020496E736572742062616EFE
:106300006B6E6F74652064656E6F6D696E61746924
:106310006F6E2028352F31302F32302F35302F310E
:1063200030302F3230302F35303029202D3E2000B4
:106330000D0A204E6F7465496E323A20000D0A2016
:106340004E6F7465496E313A20000A2042616C61DB
:106350006E63696E672056616C75653A2000205245
:1063600065666C322042616C616E63696E672053B2
:1063700063616C65203A000A205265666C312042E8
:10638000616C616E63696E67205363616C65203A6E
:10639000002050574D203A00204D696E203A0020D1
:1063A0004D6178203A002053656E733A00205365A2
:1063B0006E736F72205265706F72740D0A0A000D51
:1063C0000A20536176652028592F4E293F2000204E
:1063D00050524F43455353494E47204F5054494F15
:1063E0004E53203A0D0D0A002054687265616420F6
:1063F00069732076616C6964207768656E20542E1D
:10640000546872656164206F72204D2E5468726505
:1064100061642069732076616C6964203A200020F1
:106420004D2E5468726561642069732076616C69D1
:1064300064207768656E206F6E6C792031207065FE
:10644000616B20697320666F756E64202E2E2E2E70
:106450002E2E203A200020542E546872656164204C
:1064600069732076616C6964207768656E20726557
:10647000636F676E697A6564206279203220736584
:106480006E736F72206F6E2033203A200046414CAD
:1064900053450D0A00545255450D0A0020486F6CB3
:1064A0006F6772616D2069732076616C6964207713
:1064B00068656E207265636F676E697A65642062D5
:1064C0007920322073656E736F72206F6E203320D7
:1064D0003A2000204F50543A002054464F4C443A42
:1064E00000205442433A0020544243503A00205482
:1064F0004C454E3A0020545452414E3A00205452DA
:1065000045464C3A002054534B45573A00205254CC
:106510003A002052523A00206D6D0020524C3A0051
:10652000204D433A00202500204D656469756D506B
:10653000574D3A00206D6D2F730D0A00204D656494
:1065400069756D53706565643A002050756C7365AC
:106550004C57696474683A002075730D0A00205026
:10656000756C73654857696474683A00206D6D2FC7
:106570007300204D533A0020456E636F64657220AE
:1065800063616C6962726174696F6E204641494C47
:10659000454400205468726573686F6C644D61787F
:1065A0003A00205468726573686F6C644D696E3A86
:1065B00000206D560D0A00205468726573686F6C78
:1065C000644C6576656C3A002050574D3A00204483
:1065D0006174613A0D0A00204D61676E65746963EC
:1065E000205369676E616C2061742000204E6F201B
:1065F0006461746120617661696C61626C65002C14
:10660000204F50543A002C0031312F31322F31308D
:106610002030303332004669726D77617265203503
:106620002E30362E30330050686F746F4575726FA0
:1066300020342E30000D0A200050484F544F564F42
:106640005820732E722E6C2E0020003E000D0A0082
:1066500020496E76616C696420636F6D6D616E6454
:1066600000434C423A202020004255524E2D494EC4
:1066700000434C423A20204552524F52004552525C
:106680004F5200434C423A20204641494C45440079
:10669000534B455700434C423A2020535543434502
:1066A000535300434C423A2020454E434F444552F9
:1066B00000434C423A00202020205665726946690A
:1066C00076652020202000204552524F523A204625
:1066D0006F6C6465642062616E6B6E6F74650D0A29
:1066E00000204552524F523A20496E76616C6964DF
:1066F00020626172636F64650D0A00204552524F3B
:10670000523A20496E76616C6964206D61676E65EE
:10671000746963207369676E616C0D0A00204552CD
:10672000524F523A204D2E54687265616420696E52
:1067300074656E73697479206E6F742076616C690C
:10674000640D0A00204552524F523A204D2E546893
:1067500072656164207769647468206E6F74207656
:10676000616C69640D0A00204552524F523A204D27
:106770002E54687265616420706F736974696F6EFE
:10678000206E6F742076616C69640D0A002045529A
:10679000524F523A20542E54687265616420696EDB
:1067A00074656E73697479206E6F742076616C699C
:1067B000640D0A00204552524F523A20542E54681C
:1067C00072656164207769647468206E6F742076E6
:1067D000616C69640D0A00204552524F523A2054B0
:1067E0002E54687265616420706F736974696F6E8E
:1067F000206E6F742076616C69640D0A002045522A
:10680000524F523A20486F6C6F67616D20696E7409
:10681000656E73697479206E6F742076616C69643B
:106820000D0A00204552524F523A20486F6C6F6754
:10683000616D207769647468206E6F742076616C76
:1068400069640D0A00204552524F523A20486F6C3D
:106850006F67616D20706F736974696F6E206E6F02
:10686000742076616C69640D0A00204552524F52C3
:106870003A204952207A6F6E6520696E74656E7396
:10688000697479206E6F742076616C69640D0A00FA
:10689000204552524F523A204952207A6F6E65205D
:1068A0007769647468206E6F742076616C69640D1A
:1068B0000A00204552524F523A204952207A6F6EB8
:1068C0006520706F736974696F6E206E6F742076C7
:1068D000616C69640D0A00204552524F523A2049BA
:1068E0006E76616C696420666F726D61740D0A006A
:1068F000204552524F523A20496E76616C696420AD
:106900006C656E6774680D0A00204552524F523A0A
:1069100020496E76616C696420736B65770D0A009F
:10692000204552524F523A20496E76616C6964207C
:106930006163717569736974696F6E0D0A00206D0A
:106940006D2C20496E74656E736974793A00206D00
:106950006D2C2057696474683A002061742000200F
:106960006D6D0D0A002C204C656E6774683A002C22
:1069700020456E64506F733A002C2053746172741A
:10698000506F733A002053656E733A0020466F6C67
:106990006420426F74746F6D202020200020466FA9
:1069A0006C6420546F702020202020202000204D77
:1069B00061676E6574696320546872656164002064
:1069C00052696768742020542E54687265616400AF
:1069D0002043656E74657220542E5468726561643C
:1069E00000204C656674202020542E546872656126
:1069F00064002052696768742020486F6C6F67726A
:106A0000616D002043656E74657220486F6C6F671E
:106A100072616D00204C656674202020486F6C6F99
:106A20006772616D0020496E667261526564205A1A
:106A30006F6E65202000206D6D2C20536B65774FA5
:106A400075743A0020536B6577496E3A00204469AB
:106A500072656374696F6E3A554E4B4E4F574E0DCB
:106A60000A0020446972656374696F6E3A424F543C
:106A7000544F4D2D4241434B0D0A0020446972652D
:106A80006374696F6E3A544F502D4241434B0D0A67
:106A90000020446972656374696F6E3A424F5454C2
:106AA0004F4D2D46524F4E540D0A002044697265D9
:106AB0006374696F6E3A544F502D46524F4E540DC9
:106AC0000A00206D6D200D0A00204C656E67746809
:106AD0003A002042616E6B6E6F74653A20554E4BE2
:106AE0004E4F574E0D0A00206E6F742076616C6910
:106AF000640D0A000D0A00205245504C41590D0A00
:106B0000002043414C4942524154494F4E20534882
:106B10004545540020353030204555524F00203235
:106B20003030204555524F002031303020455552ED
:106B30004F00203530204555524F0020323020453F
:106B400055524F00203130204555524F00203520FE
:106B50004555524F002042616E6B6E6F74653A006E
:106B60000D0A00206D6D2C20496E74656E7369747A
:106B7000793A004555524F20426172636F64652037
:106B8000617420002C20496E74656E736974793AC3
:106B9000002C2057696474683A00207065616B208E
:106BA000617420004E4547415449564500504F53AB
:106BB000495449564500204D61676E6574696320EC
:046BC000000D0A00BA
:0C6BC4001DDB42E8026A016A0C0E015C55
:106BD00044E20150A3DAEF503EE0025006E1010E1C
:106BE000026EC10EE66E6B0E1DDBB60EE66E6B0E10
:106BF00019DB015093DAEF0404E1AD0EE66E6B0E83
:106C000003D0A40EE66E6B0E0DDB7FEC4BF09A0EFC
:106C1000E66E6B0EE66E54EC2DF042E9E66A01502A
:106C200061DBDCDA910EE66E6B0E46DBC6DAD6DA95
:106C3000840EE66E6B0E40DB10DBD0DAC10EE66E22
:106C40006B0EF5DA880EE66E000EE66ECAEC4BF0BF
:106C500042E97FEC4BF0012AB9D743E9E7CFD9FFEE
:106C60001200CEDA46E801CEE5F40401E46B010E31
:106C7000E517E66BE76BE451E511E611E71165E016
:106C800068D80E0109B107D0EDDAE45D016E41E983
:106C9000E550E55906D0E6DAE425016E41E9E55014
:106CA000E521026E120EE96E0E0EEA6EEE50012420
:106CB000E46FED500220E56F140EE45D036E000EEC
:106CC000E559046E0E0112510124056E1351022084
:106CD000066E140E0526000E062205EBE6FF06EBF7
:106CE000E6FF03EBE6FF04EBE6FFC4D844E9000946
:106CF00028E00E0109A106D060510A5D606F615164
:106D00000B59616F030EE66E5F0EE66E0E0EE66EB9
:106D10008BEC6CF043E9FCC0E4F4FDC0E5F4FEC08C
:106D2000E6F4FFC0E7F4040EE96E0E0EEA6E04010D
:106D3000E451EE12E551EE12E651EE12E751EE1279
:106D400002D00E0106870E01018347E9E7CFD9FF84
:106D5000120056DA49E8076A086A0E0109B116D02E
:106D6000020E00DA0E01FE0EE3501225036E41E919
:106D7000E5501321046E0A0E0326000E0422200E95
:106D80000324056E000E0420066E1ED0020EEAD902
:106D9000E552E5CFE7F4E7CFE6F40401E6510E0152
:106DA0001E5D0401E46FE7510E011F590401E56FF8
:106DB0000A0EE45D056E000EE559066E200E055CB8
:106DC000036E000E0658046E03EBE4F404EBE5F4E6
:106DD0000401D0D903E00401FAD9FEE10401E45131
:106DE000036EE551046E05EBE4F406EBE5F4C2D95D
:106DF00003E00401ECD9FEE10401E451056EE55124
:106E0000066E0001406B800E406F426983EB01F01B
:106E100084EB02F00550015C065002581AE2015062
:106E20003C25E96E02503D21EA6EEF50096E095093
:106E30000726000E08224251095C02E209EB42F0EB
:106E40000950405D02E209EB40F0012A000E0222E7
:106E5000E1D7040107EBE4F408EBE5F4060ED89063
:106E6000E533E433E804FBE1E4C441F04AE9E7CF69
:106E7000D9FF1200D9CFE6FFE1CFD9FF85E948E875
:106E8000096A0A6A0E015F6B606B616B626B636B10
:106E9000646B656B0A6A096A056A066ACDD90FE2F6
:106EA00047D9EF6A45D9EE52EE6AED6A0ADAEE6A20
:106EB000ED6A15DAEE6AED6A052A0622EFD702EBD3
:106EC000E4F403EBE5F4040155D903E004017FD9B0
:106ED000FEE10401E451026EE551036E00EBE4F4BF
:106EE00001EBE5F447D903E0040171D9FEE10401A7
:106EF000E451006EE551016E82EB05F083EB06F084
:106F00000050055C0150065839E20A500AE1DCD90C
:106F100005E2B8D99BD9D8804155BCD9D8D92AE245
:106F20000AD00A0412E1D0D91FE3092A0C0E095C29
:106F300025E0CDD908E2020E0A6ED7D9020EEF6E17
:106F4000D4D964D907D00A6A15D0020E0A5C12E1BE
:106F5000BED903E27BD9415D0AD0092A0C0E095C37
:106F60000DE0B2D906E28ED971D9D880415592D9B7
:106F700001D00A6A052A000E0622C2D7056A066AEF
:106F80005BD91EE2D5D8EF5017E09BD91BD959D950
:106F9000CFD8EE52E451EE26E551ED2292D99AD99E
:106FA0009ED9EECFE6FFEFCFE6FF85EC7AF0E55213
:106FB000E5CFEDFFE7CFEFFF052A000E0622E0D771
:106FC0000C68FF0E0B6E056A066A36D91EE2B0D851
:106FD000EF040BE1FF0E0B5C06E081D9F3D80B50F8
:106FE0009DD8D3D802E285EB0BF0A2D8EF5002086F
:106FF00008E1FF0E0C5C03E072D959D902E285EB7F
:107000000CF0052A000E0622E0D7FF0E0B5C3EE0D6
:10701000FF0E0C5C3BE00B5065D95CD90C5062D97B
:10702000FE0EE350EE24076E41E9E550ED20086EB8
:10703000D890083207320401D8900830E56F073045
:10704000E46FAED80B501BD90C504CD9EECFE6F400
:10705000EFCFE7F4E451E65DE551E75904E20B5068
:107060000ED90C5003D00C500AD90B503BD9EE501E
:10707000E45D0E01626FEE500401E5590E01636F8D
:107080000B504CD8EAD813D90EE319D00F0139A50B
:107090001ED0FF0E0B5C09E0FF0E0C5C06E10B50EE
:1070A00027D90B50FDD80B500BD0FF0E0B5C0FE116
:1070B000FF0E0C5C0CE00C501BD90C50F1D80C509E
:1070C0002DD8CBD8EECF64FEEDCF65FE02D0000EFA
:1070D00021D0E66A60CEE4F461CEE5F4E407E55B36
:1070E000E4C4E6FFE5C4E6FFEAEC71F043E9F3CF60
:1070F00060FEF4CF61FE190EE66EE66A62CEE6FF30
:1071000063CEE6FF65EC7BF0E552E5CF63FEE7CFAB
:1071100062FE010E49E9E7CFD9FF1200070DF3CF58
:10712000E9FFF4CFEAFF740EE9260E0EEA22120000
:1071300005EBE9FF06EBEAFF070EEA02F3CFEAFFF1
:10714000E902F3CFE9FFF450EA26740EE9260E0EA9
:10715000EA221200000105503C25E96E06503D214F
:10716000EA6E1200E66EE66A0CCEE6FF0DCEE6FF92
:1071700085EF7AF0E66BE76B5A0EE45F000EE55B95
:10718000E65BE75B010E1F0B120067D8EECFE6F45B
:10719000EFCFE7F40401E451E65DE551E759120051
:1071A000E66BE76B5A0EE427000EE523E623E723A0
:1071B000E4C460FEE5C461FE1200030EE926000E81
:1071C000EA221200EECFE4F4EFCFE5F41200D890FB
:1071D000E437E537E637E737E80612007BD85DECA1
:1071E0002CF043E91200EFCFE4F440510401D880C1
:1071F000E455120032D8E451EE26E551ED2212009A
:10720000D9CFE6FFE1CFD9FF81E91200EE5205EBBD
:10721000EEFF06EBEDFF1200EFCFE4F44251040164
:10722000E45D1200E66EF4EC4BF042E91200E66E0B
:107230005BEC2DF042E912000C0E055C000E0658C6
:1072400012000401D890E533E43312004ED8B5DFC4
:10725000EE2AEF227FDFEF501200050EE926000E26
:10726000EA221200020E7EDFE552E5CFE5F4E7CF19
:10727000E4F4160E77DF0401FE0EE350120032D85C
:10728000E2EF38F0010E0A6E30D8010EEF6E2DD805
:1072900006EF39F00401E46FE56B27D8FAEF38F018
:1072A0003DDF8BDFEECF62FEEDCF63FE12008ADFA3
:1072B0000C5034DFC5EF38F0BADFE66A01508EEFCC
:1072C00038F036DFDDEF38F045DFF3EF38F042DF3E
:1072D0000CEF39F0EECFE6FFEECFE6FF120028DF2D
:1072E0002DEF39F01BDFEE52120009508EEF38F00F
:0872F000C6DFA7DFD0EF38F084
:0872F800819893989382819A1A
:10730000939A938482949494770EE66E07EC59F0E6
:1073100014DBE1EC58F042E9978A86989898770E4A
:10732000E66E2AEC59F009DB49EC58F042E9928408
:1073300086969896770EE66E4BEC59F0FEDA6FEC77
:1073400058F042E9928286909890770EE66E8CEC27
:1073500059F0F3DA95EC58F042E984989698849ABB
:10736000969A849C969C849E969E92869286B9EF6D
:1073700039F0C6DA81E941E80001006B0D6B0E6B54
:107380000F6B106B116B126B136B146B156B166B11
:10739000176B186B000E016F050E026F000E036F66
:1073A000010E046F800E056F020E066F800E076FD0
:1073B000060E086F000E096F080E0A6F800E0B6F25
:1073C000090E0C6F000E3C6F050E3D6F3E6B3F6B60
:1073D000406B800E406F4269016A040E015C10E24E
:1073E0000150EA6A430FE96E000EEA22EF6A01508B
:1073F000EA6A470FE96E000EEA22EF6A012AEDD72A
:1074000042E9E7CFD9FF12007BDA81E942E8F40EC6
:10741000E66E010EC0DAF3CF25F0F4CF26F0100EA1
:10742000E66E270EB8DAF3CF27F0F4CF28F0A00EDF
:10743000E66E0F0EB0DAF3CF34F0F4CF35F0000182
:10744000F3502525366FF4502621376F8E0EE66EE9
:10745000170E2CDA0001296F26510401E5590001AD
:107460002A6F7DDA2B6FED5002202C6F2A0EE66E0C
:10747000120E1CDA0001306F26510401E55900019B
:10748000316F6DDA326FED500220336F800EE66E91
:107490000C0E90DA0001345125250401E66F00013D
:1074A000355126210401E76F0150E65DE46F02507B
:1074B000E759E56FE4C42DF0250EE96E000EEA6E83
:1074C0000001EE5001242E6FED5002202F6F25C0D9
:1074D00038F026C039F03807000E395B2551345D8D
:1074E0003A6F265135593B6F3A07000E3B5B43E933
:1074F000E7CFD9FF120004DA81E948E8E8D9010EA4
:10750000016E060E015C43E2010E01EBF3FF015236
:1075100004E0D890E836F306FCE1026E0250000168
:10752000001533E0FAD90150DFD928EC5AF00009F0
:10753000FCE1B5D935DAEF50E66EEA6A013407DAD4
:10754000EECFE4F4EFCFE5F4EA6A0134DED9E4519A
:10755000EE24E76EE551EE20EA6EE7CFE9FFE55253
:10756000E750EF6EEA6A0134D0D9EE2A000EED2220
:10757000EECFE4F4EDCFE5F4800EE41906E1010E60
:10758000E51903E1021C00010017012ABAD749E9F5
:10759000E7CFD9FF1200B4D982E9000100A144D09D
:1075A000870EE66EE1EC59F041E92EEC5AF028EC3A
:1075B0005AF00009FCE10AEC5AF0F3CF19F0F4CFCD
:1075C0001AF00001D8901A331933D8901A331933AE
:1075D00000500AE00D2B000E0E23800E0D1904E161
:1075E000010E0E1901E100910DC0E4F40EC0E5F4A6
:1075F000BDD901E699D918E30001800E3E5D010E68
:107600003F5912E23EC0E4F43FC0E5F43E2B000EC9
:107610003F233C510401E425E96E00013D51040182
:10762000E521EA6E19C0EFFF41E9E7CFD9FF12006B
:1076300067D981E948E8010E026E49D9016A060E50
:10764000015C10E202500001001508E066D901500B
:107650004BD928EC5AF00009FCE121D9029E0246E0
:10766000012AEDD749E9E7CFD9FF120049D984E9CA
:1076700043E8046A05680668060E025C4AE2EA6AA4
:10768000023443D9EE50005CED50015842E2025002
:1076900033E100EBE4F401EBE5F468D901E644D909
:1076A0001CE300EBE4F401EBE5F4E66BE76B5A0E48
:1076B000E45F000EE55BE65BE75B010E1F0B08E095
:1076C0000401D890E437E537E637E737E806F9E113
:1076D0000401E451056EE551066E00013E51055C62
:1076E0003F51065807E205503C25E96E06503D2102
:1076F000EA6E0DD0800E0CD0EA6A023428D9EE5022
:107700000024E76EED500120EA6EE7CFE9FFEF506D
:10771000046E045044E9E7CFD9FF1200F1D883E9A1
:10772000020E011402E1000E01D0010EE8B08488BF
:10773000E8A08498010E011402E1000E01D0010EB0
:10774000E8B0848AE8A0849A020E001402E1000ED8
:1077500001D0010EE8B0848CE8A0849C010E0014D6
:1077600002E1000E01D0010EE8B0848EE8A0849EF4
:1077700041E9E7CFD9FF1200C3D883E942E80050BE
:10778000640802E2640E006E190EE66EE66A0050AE
:10779000E66EE66A780EE66EE66A65EC7BF085ECEE
:1077A0007AF0E552E550046EE750036E0150090A85
:1077B0002EE0010A21E00F0A1AE0010A14E0030A90
:1077C00016E0010A0CE0070A0EE0020A04E0030AD0
:1077D00002E0020A25D0B6D895EC58F00BD0B2D80A
:1077E000E1EC58F007D0AED849EC58F003D0AAD855
:1077F0006FEC58F042E914D0005002E1000E01D0C5
:10780000010EE8B08188E8B00BD0819809D0005013
:1078100002E1000E01D0010EE8B0818AE8A0819A51
:1078200043E9E7CFD9FF12006BD882E949E8026A41
:107830004ED8970E096E8F0E0A6E080E005C0AE293
:107840006CD8005051D828EC5AF00009FCE195D8CA
:10785000E45116D0060E005C04E18050040B10E0E9
:1078600006D0070E005C05E18050020B09E0010E16
:1078700007D0080E005C06E18150020B01E0010E0A
:10788000026E08D0090E005C05E18150040B01E096
:10789000010E026E02504AE9E7CFD9FF12006DD8FF
:1078A0007FD8E4C4EEFFE5C4EDFF120083D8340EA8
:1078B000E96E000EEA6E0401EE50015CE46FED50DB
:1078C0000258E56F000125510401E45D1200870EA6
:1078D000036E9F0E046EA70E056E970E066ED70EF2
:1078E000076E8F0E086E1200EA6AE425E96EDA5020
:1078F000EA22EFCFE6FFE1EC59F041E92EEF5AF032
:10790000D9CFE6FFE1CFD9FF1200FE0BE96EEA36D0
:107910000D0EE926000EEA2212000401D950030FD1
:10792000E46FDACFE5F412005A0EE45D000EE5597B
:10793000000EE659000EE759120041E9000EE66E0E
:10794000E66A120003EBE6FF04EBE6FF1200FE0B13
:10795000E96EEA36010EE926000EEA221200250E33
:10796000E96E000EEA6EEE50012412000401E66B8F
:10797000E76BD890E751000A12000AEC5AF0F3CFF7
:10798000E4F4F4CFE5F40401D890E533E433D8907F
:10799000E533E4331200E66EFAEC2BF042E9120014
:1079A000EA6A0134FE0BE96EEA36190EE926000E8A
:1079B000EA221200F0DFF350016EF450026E120062
:1079C00001CEE5F40401E46B040EE517E66BE76B0A
:1079D000E451E511E611E71150E00ACECFFE0BCEDF
:1079E000D0FE0E01D16BD26BD36BD46BD66BD76B41
:1079F000D86BD96BDA6BDB6B030E085D27E308519C
:107A0000060824E3095103E0030E095D02E1030EB9
:107A1000CE6F090503E0020E095D02E1050ECE6F8F
:107A2000CE0EE66E0E0EE66E010E091502E0000E99
:107A300001D0010E32DA0E01D3510401E45D0E01D2
:107A4000D4510401E55902E20E01068B0E01040E29
:107A5000D56FD50EE66E0E0EE66E010E09151DDA17
:107A60000E01DA510401E45D0E01DB510401E55918
:107A700002E20E01068B0E0101871200D9CFE6FF4C
:107A8000E1CFD9FF84E951E837DAEF500C6E77DAAD
:107A9000010EE926000EEA22EE500A6EED500B6E42
:107AA0002BDAEE5206EBEEFF07EBEDFF25DA030EC5
:107AB000EB6A040EEB6A20DA050EEB6A060EEB6A3F
:107AC000116AFC0E126E025001E18ED0CFD9030E66
:107AD000E503F3CFE5F4E403F450E52792D9EE5043
:107AE000F324066EED50E521076EE0D9EECFE4F405
:107AF000EFCFE5F4040EE45F000EE55B050EE45DF8
:107B0000086E000EE559096E86EB04F087EB05F070
:107B10000450085C055009584AE347DA090E35DA83
:107B2000EF50E66EE66A030E045CE56F000E055842
:107B3000A9D9045CE76F000E055869D926DAEFCFA2
:107B4000E8F40F0E045CEB6F000E05587AD9045C64
:107B5000ED6F000E05583ED9E9D9030E38DA04E27C
:107B600080D902E2DED901D02FD9ECD9040EDED9BA
:107B7000040E2DDA04E275D902E2D3D901D024D95A
:107B8000E1D9050ED3D9050E22DA04E26AD902E260
:107B9000C8D901D019D9E4510F5EE5518DD901E65C
:107BA00090D901E2DED9042A000E0522B1D788EB74
:107BB00004F089EB05F07AD90450EE5C0550ED58DD
:107BC00001E294D0F2D9030E9CD9105A040E99D92F
:107BD000105A050E96D970D901E673D901E2C1D9C0
:107BE000042A000E0522E7D741D90BD9EE50E4252F
:107BF000066EED50E521076E04D9040EEE24086EE2
:107C0000000EED20096E050E0826000E092286EBF7
:107C100004F087EB05F00850045C095005584AE36E
:107C2000CDD9090EB8D9EF50E66EE66A030E0424EA
:107C3000E56F000E052026D90424E76F000E05200D
:107C4000E6D8A9D9EFCFE8F40F0E0424EB6F000EAD
:107C50000520F7D80424ED6F000E0520BBD86CD9A1
:107C6000030EB8D904E2FDD802E25BD901D0ACD84A
:107C700069D9040E61D9040EADD904E2F2D802E24A
:107C800050D901D0A1D85ED9050E56D9050EA2D97A
:107C900004E2E7D802E245D901D096D8E4510F5E5C
:107CA000E5510AD901E60DD901E262D90406000EB8
:107CB000055AB1D788EB04F089EB05F0A2D8EE5055
:107CC000045CED50055812E379D9030E22D9105AFD
:107CD000040E1FD9105A050E1CD9EED801E6F1D8B2
:107CE00001E246D90406000E055AE8D7123402E331
:107CF000116A126A0CEBE6FFFFD8EE52EECFE6FFF8
:107D0000EECFE6FFEAEC71F0E6D8EE52F3CFEEFFED
:107D1000E5C4EDFF0E0109A103D0EED818D94CD867
:107D2000010E0E010915025C07E1E6D8EE52EECF16
:107D3000E4F4EFCFE5F403D0DFD809D9E56FDCD860
:107D4000030EE926000EEA22E4C4EEFFE5C4EDFFCF
:107D50000CEBE6FF030EE66EE66A11EBE6FF12EBB4
:107D6000E6FF3DEC7AF036EC72F0B5D8050EE92668
:107D7000000EEA22F3CFEEFFE5C4EDFF52E9E7CFB4
:107D8000D9FF1200E56FE4510A24E96EE551D1EF05
:107D90003FF0E76FE6510A24E96EE75102D9E66E3B
:107DA000E66A12000D6E0E6AFE0EE3500D5E41E9AA
:107DB000E5500E5A0E341200E56F9ED8EE52E4C420
:107DC000EEFFE5C4EDFF1200ACD8E46DE51F000E38
:107DD000E5231200EE6FED510A24E96EEE51E1D871
:107DE000E625E46F000EE721E56FE4511326E55127
:107DF0001422D8901430E56F1330E46FA3D8030E2B
:107E00001200BDD8120EE9260E0EEA221200E86F0B
:107E1000E7510A24E96EE851C4D8E425136E146AC8
:107E20001436FE0EE350132641E9E55014220C0EE1
:107E30001200EA6FE9510A24E96EEA510B20EA6E5A
:107E40001200EC6FEB510A24E96EEC51AAD8E82538
:107E5000E66FE76BE737120E12000F26000E1022B6
:107E600012000D500008000E0E5412000CCEE4F467
:107E70000DCEE5F40401D890E533E433D890E53332
:107E8000E4331200E66FE5510A24E96EE6510B2057
:107E9000EA6EEFCFE4F4060E1200E66EEFDD43E982
:107EA0000F0138510401E46FE56B120068D81E0E13
:107EB000E9260E0EEA221200105A10341250101841
:107EC00012000F50115C1050125812008FEB11F07D
:107ED00090EB12F0120043E9F4CFE5F47CEF3FF0B1
:107EE0000424E46F000E0520C2EF3EF0045CE46F52
:107EF000000E0558C2EF3EF000EBE9FF01EBEAFF90
:107F00001200085CE46F000E09583CDF0F5E000EA3
:107F100012000824E46F000E092034DF0F5E000E0B
:107F200012000DEBE4F40EEBE5F412000824E66F0A
:107F3000000E0920C9EF3EF0085CE66F000E0958FC
:107F4000C9EF3EF0E4510F5EE551105A1200EE52B7
:107F5000EE500A5D0401E46FEE500E010B5904016E
:107F60001200B4DF0428E46F000E0520DCEF3EF0C1
:107F7000ADDF0404E46F000E0558DCEF3EF0EA6A62
:107F80000C34FE0BE96EEA361200045CE96F000E59
:107F9000055819EF3FF00424E96F000E052019EF92
:107FA0003FF00B20EA6EEF5012000F6A106A030ECA
:107FB00014D8040E12D8050EEDEF3FF00F6A106AC8
:107FC000030E0ED8040E0CD8050EF0EF3FF088DF3C
:107FD000D2EF3EF08BDFD2EF3EF082DF2DEF3FF0AD
:067FE00085DF2DEF3FF0EC
:0A7FE60036DA83E97FEC4BF016DA7F
:107FF000060D35DAB80E0401E427FB0EE523E4C4D0
:10800000E6FFE5C4E6FF54EC2DF042E9730EE66EA0
:108010006B0E16DABBD919DA02EC2CF042E9630ECA
:10802000E66E6B0E0DDAE66AF3D90FDA5DEC2CF032
:1080300043E9600EE66E6B0E03DA880EE66E000E04
:10804000E66ECAEC4BF042E97FEC4BF041E9E7CF3A
:10805000D9FF1200FFD981E949E801CEE5F4040116
:10806000E46B020EE517E66BE76BE451E511E611F0
:10807000E71158E00E010851020802E3026A03D03A
:10808000020E085D026E040E085D02E3060E02D0C9
:10809000020E0825036ECC6BCD6B040E046E016AD4
:1080A000015006082CE30250015C27E30150035CF9
:1080B00024E381EB05F0D950040FE66EDACFE6FF3A
:1080C00035D842E90E010851015C06E1CC51085C4B
:1080D000CD51095812E305D00850CC5D0950CD5957
:1080E0000CE204EBC8FE05EBC9FE06EBCAFE07EB8B
:1080F000CBFE08EBCCFE09EBCDFE012AD1D70E0159
:108100000851C95D0DE10F0135510401E46FE56BC4
:10811000E4510E01CC5D0401E5510E01CD5901E29F
:10812000068901854AE9E7CFD9FF120093D983E98F
:1081300056E89FD9EF50036E71D9046E59D9010EDC
:10814000E926000EEA22EE50136EED50146E06CEB4
:10815000E6F40401E46BE56B0F0EE617E76BE45100
:10816000E511E611E71105E10E0160510B6E615159
:1081700004D00E0152510B6E53510C6E156AFC0E59
:10818000166E88D9EECFE4F4EFCFE5F477D971D944
:10819000040EEB6A050EEB6A31D90B500900F55C51
:1081A0000C500A00F55801E3BCD028D9040109009D
:1081B000F5500B5CE46F0A00F5500C58E56FE4C411
:1081C000E6FFE66EFAEC2BF042E9F350096EF4504C
:1081D0000A6E36CFE6FF37CFE6FFFAEC2BF042E926
:1081E000F3500D6EF4500E6E0E0109A153D04CD910
:1081F000040118D9E4510D24056EE5510E20066ED8
:1082000043D910D90D50E45D076E0E50E559086E44
:1082100085EB0FF086EB10F007500F5C08501058FC
:1082200001E27FD0176A186A116A126A280E115C7F
:10823000000E12580EE2B0D8E6BFE769E6C4E6FFCA
:10824000E7C4E6FF11500F5CE46F12501058BAD823
:10825000EDD718341650181804E61750155C18504E
:10826000165814E297EB15F098EB16F0C1D80D0EE6
:10827000E926000EEA2204010F50EE5CE46F105074
:10828000ED58E56FE407000EE55BF8D80F06000E29
:10829000105AC2D7FFD80401CCD80D50E45D056E4A
:1082A0000E50E559066EF6D8C4D8E4510D24076E79
:1082B000E5510E20086E85EB0FF086EB10F00F50A5
:1082C000075C105008582DE3176A186A116A126A81
:1082D000280E115C000E12580EE25ED8E6BFE76968
:1082E000E6C4E6FFE7C4E6FF0F501124E46F105028
:1082F000122068D8EDD718341650181804E6175015
:10830000155C1850165809E297EB15F098EB16F02B
:108310003DD80FEBEEFF10EBEDFF0F2A000E102201
:10832000CED7163402E3156A166A03EBE6FF2ED8A1
:108330008CD8EAEC71F043E992D828D8F3CFEEFF5D
:10834000E5C4EDFF03EBE6FFF76A0434FE0BF66EBF
:10835000F736AA0EF626FB0EF7220900F5CFE6FF48
:108360000900F5CFE6FF15EBE6FF16EBE6FF3DEC67
:108370007AF036EC72F043E972D84AD8F3CFEEFFC8
:10838000E5C4EDFF57E9E7CFD9FF120072D8020E1E
:10839000E926000EEA2212000450280DF3CFE8F47B
:1083A000F4CFE9F4840E0401E827FA0EE923115012
:1083B000E825F66E1250E921F76E0800F5CFE6F4D5
:1083C000E76B1200E56FE4511324E96EE5511420C8
:1083D000EA6EEF50E66EE66A65EC7BF0FE0EE35067
:1083E000172641E9E5501822112A000E1222120028
:1083F000EA6A0334FE0BE96EEA361200F76A0434C7
:10840000FE0BF66EF7369C0EF626FB0EF7221200D8
:1084100030D8040EE926000EEA2212002AD8EE52C5
:10842000EF5012000950EE5CE46F0A50ED58E56F12
:108430001200EE500924E46FED500A20E56F12009F
:10844000E66E5BEC2DF042E91200EECFE6FFEECFD8
:10845000E6FF1200D9CFE6FFE1CFD9FF1200F3CF3C
:10846000E4F4F4CFE5F41200120EE9260E0EEA222F
:10847000120000EBE9FF01EBEAFF120087DFE4C422
:10848000EEFFE5C4EDFF1200B3DF1E0EE9260E0E6F
:0A849000EA221200ADDF34EF42F0E3
:06849A000001010E556F08
:1084A000566B576B586B596B5A6B5B6B5C6B5D6BA8
:1084B00063EF42F00001010E556F63EF42F00001DF
:1084C000556B63EF42F016DA536B546B1200D9CF41
:1084D000E6FFE1CFD9FF81E943E80401D15102E190
:1084E000036A01D003688FEC2BF0F350016EF45057
:1084F000026ED40EE96E040EEA6E0401EE50015CC9
:10850000E46FED500258E56FE4510508000EE555A3
:108510006FE201EBD4F402EBD5F481B040D000015E
:10852000565103E0566BDAD9CEDF0401D15110E188
:108530009CD9040EE4195CE1E5515AE1E65158E199
:10854000E75156E1F6D90401010ED16FBCDF50D0DE
:10855000D10510E18AD9900EE4194AE1010EE5191E
:1085600047E1E65145E1E75143E1E3D96FD9040121
:10857000020E13D0020ED15D3BE177D9B00EE419A3
:1085800037E1040EE51934E1E65132E1E75130E11B
:10859000D0D95CD95BD90401030ED16F29D0040175
:1085A000D2510408000ED35503E2040ED26FD36BF0
:1085B000D2510008000ED35513E2D207000ED35B50
:1085C000D251D3110DE1D10507E10B01955104E121
:1085D000E66A20EC0FF041E90401D151036ED16B42
:1085E0000B01955105E10001575102E0576B76D917
:1085F000035044E9E7CFD9FF1200D9CFE6FFE1CF1E
:10860000D9FF83E971D9849084928CD901500C0AE6
:1086100001E1A2D00A0A01E183D00D0A01E180D074
:108620000E0A6BE00F0A69E0030A60E0010A54E0F9
:108630000F0A4DE0030A3EE0070A13E0010A0EE0CC
:10864000030A01E093D0B60EE66E660E07D900016C
:10865000D00E4D6F070E4E6F65D982D0E3EC50F00F
:1086600085D000EBE6FF4DEC50F041E922D901E165
:108670002DD90F013E5101E179D00E010851E96E6B
:10868000EA6AD890E936EA36D60EE926040EEA22DE
:10869000EECFE4F4EFCFE5F40401E45100015827F4
:1086A0000401E55100015923000E5A235B235C2B82
:1086B0005D235CD000EBE6FFA7EC50F041E9E0D889
:1086C0000F013C0501E102D90E0108694FD0B10E3E
:1086D000E66E660EC3D84AD0A30EE66E660EBED80E
:1086E0000001E20E4D6F040E4E6F40D0950EE66E07
:1086F000660EB4D8DED83AE12AD0050E015C04E15A
:10870000900EE66E660EFED80A0E015C04E1830E42
:10871000E66E660EA3D8B4D80F013C0527E117D04A
:10872000060E015C04E17D0EE66E660EEBD80B0EC4
:10873000015C04E1710EE66E660E90D8A1D8C6D831
:10874000900EE66E010EE66E81EC47F042E9E80E0F
:10875000E66E030EE66E07D0DDD833EC4DF044E94B
:10876000640EE66EE66ACDEC2BF042E941E9E7CF14
:10877000D9FF120000014D514E1121E08CD80001AB
:108780004D5D0401E55100014E5919E24D6B4E6BF0
:10879000ABD80B01955103E1E3EC50F010D09505F7
:1087A00007E1610EE66E660EE66EE66AE66A04D0E2
:1087B000020E955D04E1AED833EC4DF044E90001C2
:1087C0004F5150110CE067D800014F5D0401E55195
:1087D0000001505904E24F6B506B849284900B015E
:1087E000955133E10001550530E18FEC2BF000018C
:1087F0005151F35C0401E46F00015251F45804013B
:10880000E56FE80EE45D030EE5591FE373D8532BC3
:10881000000E54230F013A510001535D0F013B51EB
:108820000001545912E3536B546B0E0108690F0198
:108830003D5107E084928490EAEC27F04FD863EF33
:1088400042F052D80001010E566F1200320EE66E51
:10885000E66A81EC47F042E999EF44F0E66EE66A99
:10886000E66A33EC4DF044E91200D22B000ED3231C
:10887000D2C4E4F4D3C4E5F40401E66BE76B120060
:108880000001D00E4D6F070E4E6F8482D00E4F6FD9
:10889000070E506F12008FEC2BF000014B51F35C70
:1088A0000401E46F00014C51F4580401E56FE451F8
:1088B00012000001E20E4D6F040E4E6F8480E20E36
:1088C0004F6F040E506F0F013C511200E80EE66E20
:1088D000030EE66ECDEC2BF042E91200E66A020EC2
:1088E000E66E8BDE42E91200010EE66E6CEC4DF096
:1088F00041E912008FEC2BF0F3CF51F0F4CF52F09E
:1089000000011200E66EE66A060EE66E33EC4DF0EC
:1089100044E91200690EE66E660EE66EE66A050E22
:10892000E66E12008FEC2BF0F3CF4BF0F4CF4CF04F
:108930001200640EE66EE66ACDEC2BF042E91200FE
:1089400004D804EC3AF01DEF28F00CDA81E943E892
:10895000026A036AFCD9F4EC48F046E901CFE4F47A
:1089600002CFE5F40401CFD904E6390EE45D030E2D
:10897000D0D90CE301CFE8F402CFE9F4D0D905E671
:10898000D880400EE855090ED0D902E2010E036EE0
:1089900005CFE4F406CFE5F4B6D902E6640EE7D9D4
:1089A0000CE305CFE8F406CFE9F4B9D905E6D880A1
:1089B000E80EE855030EB9D902E2010E036E016A12
:1089C000080E015C0DE20150EA6A0B0FE96E0F0E12
:1089D000EA22EF50640802E2010E036E012AF0D78A
:1089E0000F012B51030803E32C51030802E2010E8F
:1089F000036E320E2D1901E12E5102E0010E026EBE
:108A000003CFE4F404CFE5F404017DD902E6FA0EC5
:108A1000AED90CE303CFE8F404CFE9F480D905E63E
:108A2000D880EE0EE855020E80D902E2010E026EE9
:108A300007CFE4F408CFE5F466D904E6100EE45D50
:108A4000270E67D90CE307CFE8F408CFE9F467D91C
:108A500005E6D880500EE855460E67D902E2010EB1
:108A6000026E09CFE4F4E56B4ED902E6010E7FD920
:108A700007E309CFE8F4E96B52D901E67CD902E2B9
:108A8000010E026E0ACFE4F4E56B3DD902E6010E59
:108A90006ED907E30ACFE8F4E96B41D901E66BD957
:108AA00002E2010E026E0F01C80E2F5D000E30595A
:108AB00005E32F51C208010E305502E2010E026E8D
:108AC000640E315D000E325905E331512C08010E60
:108AD000325502E2010E026E140E335D03E3335190
:108AE000640802E2010E026E040E345D03E33451A9
:108AF000140802E2010E026E0A0E355D0BE33551D9
:108B00000401E46FE56BE53507E2E451FF08000E70
:108B1000E55502E2010E026E36CFE4F437CFE5F4FC
:108B20000401F1D804E62C0EE45D010EF2D80CE34A
:108B300036CFE8F437CFE9F4F2D805E6D880580EFE
:108B4000E855020EF2D802E2010E026E280E0F0165
:108B5000385D03E338515A0802E2010E026E3ACF43
:108B6000E4F43BCFE5F40401CED802E6010EFFD8D1
:108B70000CE33ACFE8F43BCFE9F4D1D805E6D8804E
:108B80002C0EE855010ED1D802E2010E026E0F0143
:108B90003C5104E03C0502E0010E026EF00E391576
:108BA00002E0010E026E3D5104E03D0502E0010EBF
:108BB000026E035038E0010E006F710E016F060E59
:108BC000026FF40E056F010E066F640E0B6F320E0E
:108BD0000C6F0D6F0E6F0F6F106F080E116F126F0D
:108BE000640E136F146F2B6B2C6B016A080E015C03
:108BF00018E20150EA6A130FE96E0F0EEA22EF68DD
:108C00000150EA6A1B0FE96E0F0EEA22EF6A01506B
:108C1000EA6A230FE96E0F0EEA22800EEF6E012A38
:108C2000E5D7010E026E02503AE0320E0F012D6FB1
:108C30002E6B120E036F020E046F980E076F3A0E22
:108C4000086F5A0E096F3C0E0A6F900E2F6F010EBF
:108C5000306F2C0E316F010E326F320E336F080EF3
:108C6000346F140E356FF40E366F010E376F460EEB
:108C7000386F3C0E3A6F3B6B010E3D6F3C6F030E3D
:108C8000396F3E6B010E3F6F8480640EE66EE66ABC
:108C90009AEC2BF042E9849007D8000E01D0010E27
:108CA00044E9E7CFD9FF12005DD881E941E80B0123
:108CB0005A0EA56F4CD804EC4AF046E9016E0B0140
:108CC000A56B015042E9E7CFD9FF12004BD883E9E9
:108CD00032D8F4EC48F046E9010E41E9E7CFD9FF7C
:108CE000120040D883E941E80B015A0EA56F23D842
:108CF00004EC4AF046E9036E0B01A56B035042E910
:108D0000E7CFD9FF1200E66BE76BD890E751000A76
:108D10001200E559000EE659000EE7591200EA6B01
:108D2000EB6BEB35000EEB191200E955000EEA551E
:108D3000000EEB551200180EE66E010EE66E00EB0B
:108D4000E6FF01EBE6FFE66A040EE66E1200400E57
:108D5000E66EE66A000EE66E0F0EE66E000EE66E3A
:108D6000E66A1200D9CFE6FFE1CFD9FF1200E45D39
:108D7000000E89EF46F0D880640EE855000E95EF9E
:028D800046F0BB
:0E8D8200EBD981E941E80E01F06BF16B0B01BA
:108D9000A46B016A020E015C04E2F0D9EF6A012AB9
:108DA000F9D70E01020EDC6FDF6B0D0EE06FE16B89
:108DB00042E9E7CFD9FF1200D0D988E942E8020E94
:108DC000045C08E20250031005E0200E005C000E77
:108DD000015802E2000E35D00450AED9010EEF6EFC
:108DE0000450AAD9030EBED902EBEEFF03EBEDFF50
:108DF0000450A2D9050EB6D900EBEFFF82EB08F0C4
:108E000083EB09F0A3D9EF68B5D9EF6A040103EB4E
:108E1000E4F4E56B9BD9E4C4EFFFACD905EBEFFFBD
:108E200095D906EBEFFF92D907EBEFFF8FD9010E33
:108E3000EF6E045081D9EE5208EBEEFF09EBEDFF27
:108E4000010E94D18AD981E941E80B01A46B016A32
:108E5000020E015C16E292D9EF0403E18FD9020EF3
:108E6000EF6E8CD9EF50020808E088D9EF50040863
:108E700004E084D9EF50050802E10B01A42B012A7C
:108E8000E7D70B01A451010801E27AD842E9E7CF04
:108E9000D9FF120062D982E9020E005C0CE271D99E
:108EA000EF0404E06ED9EF50030805E16AD9020E21
:108EB000EF6E0B01A42B41E9E7CFD9FF12004DD98A
:108EC00082E9020E005C19E25CD9EF50030808E069
:108ED00058D9EF5005E055D9030EEF6E0B01A407EA
:108EE0000B01A45105E1010EA46F0E01020EDC6F0F
:108EF0000E01F051005C01E143D841E9E7CFD9FF11
:108F000012002BD983E942E80B01A4511EE00E01A7
:108F1000F05112D9040EEF6E8FEC2BF0F3CFE4F486
:108F2000F4CFE5F40E01F05107D9060E1BD9E4C4C5
:108F3000EEFFE5C4EDFFF051FFD8080E13D900EBAA
:108F4000EEFF01EBEDFF1CD81AD08FEC2BF0F350A5
:108F5000036EF450046E8FEC2BF004010350F35CAD
:108F6000E46F0450F458E56F0050E45D0150E5599A
:108F700006E2010EE66E16EC5AF041E9ECD7F6D0A7
:108F8000ECD881E942E80B01A45138E00E01F05120
:108F9000016E012A020E015C01E1016AEFD8EF5077
:108FA000026E040E025C20E18FEC2BF0F3CFE6F4AE
:108FB000F4CFE7F4E3D8060ED5D8EE500401E65D11
:108FC000E46FEE50E759E56FD9D8080ECBD8EECF55
:108FD000E8F4EFCFE9F4E851E45DE951E55904E341
:108FE000CDD8020EEF6E03D0020E025CD2E101EB8F
:108FF000F1FE0E01F051F15D01E001D8B7D0F29E13
:10900000F29CD8CFE4FFE0CFE4FFE46EE9CFE4FFC9
:10901000EACFE4FFE652D9CFE6FFDACFE6FFF6CF9C
:10902000E6FFF7CFE6FFF8CFE6FFF3CFE6FFF4CF9A
:10903000E6FFE96A1F0EFC1409E0FDCFE6FFFECF54
:10904000E6FFFFCFE6FF0600E92AF4D7E9CFE6FF07
:10905000FC5001E0FC6AE1CFF2FEE2CFF3FE0B012F
:10906000A45140E00E01F0510A0DF3CFE9FFF4CF17
:10907000EAFFDC0EE9260E0EEA22EE52F2CEEFFFF8
:109080000E01F0510A0DF3CFE9FFF4CFEAFFDC0E39
:10909000E9260E0EEA22EE52E92A000EEA22F3CE6B
:1090A000EFFFF1CEF0FE0E01F0510A0DF3CFE9FF14
:1090B000F4CFEAFFDC0EE9260E0EEA22EE52EFCFE5
:1090C000F2FE0E01F0510A0DF3CFE9FFF4CFEAFFF3
:1090D000DC0EE9260E0EEA22EE52E92A000EEA2202
:1090E000EFCFF3FEF2CEE1FFF3CEE2FFE552E55023
:1090F000E96E0500E550FF6EE550FE6EE550FD6E31
:10910000E906F7E1E5CFF4FFE5CFF3FFE5CFF8FFA0
:10911000E5CFF7FFE5CFF6FFE5CFDAFFE7CFD9FFE1
:10912000E552E5CFEAFFE5CFE9FFE550E5CFE0FF07
:10913000E5CFD8FF100012000A0DF3CFE9FFF4CFFE
:10914000EAFFDC0EE9260E0EEA22120008EBE9FF28
:1091500009EBEAFF082A09221200D9CFE6FFE1CF86
:10916000D9FF1200E926000EEA22120043E9E7CFF8
:10917000D9FF120009D8EF6AC4EF48F001509CEF04
:1091800048F000509CEF48F0E1DFEF6ADFDFEF6A64
:04919000A6EF48F00E
:0C919400D9CFE6FFE1CFD9FF83E941E825
:1091A000F2AE03D0010E036E01D0036A000E00265A
:1091B000C00E0122F86A040101EBE4F4E56BE4C49B
:1091C000F7FF00EBF6FFA684A688F29E550EA76E69
:1091D000AA0EA76EA682035001E0F28EA694A6986E
:1091E00042E9E7CFD9FF1200D9CFE6FFE1CFD9FF9F
:1091F00087E942E804EBE4F405EBE5F40401E66BEF
:10920000E76BD8900401E751000A08E6000EE45D20
:10921000080EE559000EE659000EE75964E2040114
:1092200004500024E46F05500120E56F0401E66B53
:10923000E76B0401E735000EE71909E6D880000E58
:10924000E455080EE555000EE655000EE7552AE2F6
:109250000401E86B080EE96FEA6BEB6B04EBECF4CE
:1092600005EBEDF40401EE6BEF6B0401EC5104012E
:10927000E85D0401E46F0401ED510401E9590401C2
:10928000E56F0401EE510401EA590401E66F04019F
:10929000EF510401EB590401E76F0401E451006E42
:1092A000E551016E000E0426C00E0522F86A040185
:1092B00005EBE4F4E56BE4C4F7FF04EBF6FF076AA3
:1092C000086A0050075C015008580DE2090002507E
:1092D0000724E96E03500820EA6EF5CFEFFF072A56
:1092E000000E0822EED743E9E7CFD9FF1200D9CF0D
:1092F000E6FFE1CFD9FF87E943E8096A04EBE4F42C
:1093000005EBE5F40401E66BE76BD8900401E75147
:10931000000A08E6000EE45D080EE559000EE65965
:10932000000EE75967E2040104500024E46F055081
:109330000120E56F0401E66BE76B0401E735000EE1
:10934000E71909E6D880000EE455080EE555000E31
:10935000E655000EE7552AE20401E86B080EE96FB6
:10936000EA6BEB6B04EBECF405EBEDF40401EE6B54
:10937000EF6B0401EC510401E85D0401E46F0401AA
:10938000ED510401E9590401E56F0401EE510401B6
:10939000EA590401E66F0401EF510401EB5904019D
:1093A000E76F0401E451006EE551016E000E0426E2
:1093B000C00E0522F86A040105EBE4F4E56BE4C491
:1093C000F7FF04EBF6FF076A086A0050075C0150DC
:1093D000085810E2090002500724E96E03500820E3
:1093E000EA6EEF50F55C02E0010E096E072A000EEE
:1093F0000822EBD7095002E0000E01D0010E00D088
:1094000044E9E7CFD9FF1200D9CFE6FFE1CFD9FF7A
:1094100087E946E8096A0A6A5A0E0B01A55D23E14D
:10942000C00E0416FF0E051684EB07F085EB08F05E
:1094300082EB0BF083EB0CF0040104500024E46F8A
:1094400005500120E56FE66BE76BE735000EE71985
:1094500009E6D880000EE455080EE555000EE655E5
:10946000000EE75502E2000E30D004EBE6FF05EBFC
:10947000E6FF90DE42E90050095C01500A5817E20D
:109480000BEBE6FF0CEBE6FF07EBE6FF08EBE6FF76
:1094900020D844E9400E0726000E0822400E0B2675
:1094A000000E0C22400E0926000E0A22E4D700EB23
:1094B000E6FF01EBE6FF02EBE6FF03EBE6FF04EB62
:1094C000E6FF05EBE6FF13DF46E947E9E7CFD9FF03
:1094D0001200D9CFE6FFE1CFD9FF85E942E8C00EFF
:1094E0000216FF0E031602EBE4F403EBE5F40401AD
:1094F000E66BE76B0401E735000EE71909E6D88053
:10950000C00EE455070EE555000EE655000EE75572
:1095100030E3000E0226C00E0322F86A040103EBBA
:10952000E4F4E56BE4C4F7FF02EBF6FF0A00056A1A
:10953000400E055C0BE205500024E96E000E012090
:10954000EA6EEF50F56E0F00052AF2D7F2AE03D0A7
:10955000010E066E01D0066AA69AA684A698F29E0F
:10956000550EA76EAA0EA76EA682065001E0F28ED7
:0A957000A69443E9E7CFD9FF1200EB
:06957A00040120511F0B4B
:10958000010801E012002051600BE842E842E84285
:10959000E842E842010801E01200245103E02405FA
:1095A00001E012002151230A39E0010A33E0030AE5
:1095B00025E0010A1CE0240A31E0070A2FE0010A35
:1095C0002DE0030A0EE0010A01E01200B7D90B01F9
:1095D000C80E8C6F040E8D6F0B019D930B01080E4E
:1095E00017D0ACD90B01C80E8E6F040E05D0A6D9CA
:1095F0000B01C00E8E6F040E8F6F12009FD90B01EE
:10960000C00E8C6F040E8D6F0B019D930B01070E26
:10961000906F120093D922C4C7F412001200040103
:10962000C06BC20EC16F010EC26FC36BC46BC56B42
:10963000080EC66FB96BB86B0F011A0E4E6F1E0E77
:109640004F6F0401300E166F040E176F400E146F2B
:109650000401196F380E1A6F040E1B6F880E186FF5
:109660000401780E1E6F040E1F6F400E1C6F120057
:1096700045D984E90401B86B040118BF19D0005022
:10968000195D02E21951006E0401B86B0050B85D1B
:109690000EE2B8514CD9E66EB8510124E96E000EC5
:1096A0000220EA6EE552E750EF6EB82BEFD737D9BC
:1096B0000401B85141E9E7CFD9FF12001FD981E970
:1096C00042E801680268040118BF11D01951040171
:1096D000B85D05E2B851B82B2AD9016E026A0401BF
:1096E00019510401B85D03E31AD90401B86B01EB09
:1096F000F3FF02EBF4FF43E9E7CFD9FF1200FED8F6
:1097000081E943E8060E0B019C5D3CE10401B9517F
:1097100002E1D06B13D0D05104E0036AC0EC47F0F3
:1097200034D08FEC2BF0F350016EF450026E060E25
:109730000B019C5D29E10401B95103E1010E036EA7
:1097400024D08FEC2BF004010150F35CE46F025045
:10975000F458E56FE66BE76BE735000EE71909E6AD
:10976000D880640EE455000EE555000EE655000E57
:10977000E75505E2036A0401010ED06F06D0C0EC84
:1097800047F0D5D70401D06B036A035044E9E7CF13
:10979000D9FF1200B3D883E942E8B1DF000920E025
:1097A000046A04500401E46FE56BE53504E2E4511A
:1097B000FF08000EE5550AE304500024E96E000E90
:1097C0000120EA6EEF5002E0042AEBD700EBBAF476
:1097D00001EBBBF404EBBEF40401BF6B010EB96FE7
:1097E00043E9E7CFD9FF120089D883E941E887DF51
:1097F000000921E0036A03500401E46FE56BE535DD
:1098000004E2E451FF08000EE5550BE30350002489
:10981000F66E000E0120F76E0800F55002E0032AF4
:10982000EAD700EBBAF401EBBBF403EBBEF404019E
:10983000010EBF6FB96F42E9E7CFD9FF12005ED8C2
:1098400081E941E804011CBF55D0030E0401B95D54
:1098500001E1B96BB9514EE0020EB95D03E10401BB
:109860001D6B3FD0B90540E1BE510401E46FE56BCB
:10987000E4514008000EE55502E2400E02D004011A
:10988000BE51016E01EB1DF401500401BE5DBE6FBF
:10989000780EBC6F040EBD6FBF050AE1015011E0E8
:1098A000BAC4F6FFBBC4F7FF0800F5502CD8F6D7B2
:1098B000015007E0BAC4E9FFBBC4EAFFEF5023D868
:1098C000F7D70401BE5110E104011D510401E46FFA
:1098D000E56B400EE41905E1E55103E10401020ED8
:1098E00002D00401030EB96F400E04011C171C7D49
:1098F000880E1C1342E9E7CFD9FF1200D9CFE6FF4B
:10990000E1CFD9FF1200BCC4E9FFBDC4EAFFEF6E8E
:10991000BC2B000EBD23BA2BBB2301061200040191
:10992000400E196F1817187D880E18131200EA6A76
:10993000380FE96E040EEA22EF5012000B01030EFD
:049940008B6F120017
:0C9944009ED9010E016E959C959A959895
:10995000F00E9516839C839A8398949A828A0A0EB5
:1099600031D9829A020E2ED9828A320E2BD94CD945
:10997000030E28D949D972D947D970D9200EE66E7D
:10998000EFD841E96BD9290E1AD901E1016A66D9EC
:10999000180E15D901E1016A61D97F0E10D901E1D4
:1099A000016A5CD9570E0BD901E1016A57D9690EDA
:1099B00006D901E1016AFA0E05D9280E00D901E1A4
:1099C000016A4CD90C0EFBD801E1016A47D9010E9E
:1099D000F6D801E1016A42D9060EF1D801E1016A27
:1099E000050EF0D801500CD1E5D883E9100E015CCA
:1099F0000AE2020E005C07E2005002E1800E01D094
:109A0000C00E01242ED9E4D0D5D882E900EBE6FFC0
:109A100074D841E9DDD0CED883E937D9EF5003E0DF
:109A2000E7D841E9FAD7D4D0C5D883E9F7D803E01D
:109A3000D3D841E9FBD7CCD0BDD885E9100E035C63
:109A400011E2020E025C0EE2025002E1800E01D031
:109A5000C00E0324E66E40D841E917D9EF5002E06A
:109A6000C7D8FAD7B5D0A6D885E9100E035C10E2A6
:109A7000020E025C0DE2025002E1800E01D0C00E27
:109A80000324E66E29D841E9C9D802E0A5D8FBD75E
:109A90009FD090D884E942E841D8056E070E0214A1
:109AA000080DF3504009DDD8046A080E045C0DE28D
:109AB00004500024F66E000E0120F76E0800F5CF6A
:109AC000E6FF1BD841E9042AF0D7800E0510C9D85B
:109AD00043E9E7CFD9FF1200C8D856D8000909E0FA
:109AE00002500206000902E1000E06D00A0E5DD8FF
:109AF000F4D7C1D8839CD3D883D0B7D845D8000930
:109B000009E002500206000902E1000E06D00A0E2A
:109B10004CD8F4D7B0D8838CC2D872D0B2D8016AEE
:109B2000C8D8839C8FD8019E01506AD043D881E960
:109B300042E8016AFA0E026E27D8000909E00250D5
:109B40000206000902E1000E07D00A0E2ED8F4D753
:109B5000B0D8838C77D8015043E9E7CFD9FF120002
:109B600029D882E900380F0B006E839C839A0A0E75
:109B70001CD88388140E19D8F00E83140010836E3D
:109B80008398140E12D824D07CD893D8839C010ECD
:109B900081D8080E8314016E8398020E8ED801506E
:109BA00002E1000E01D0010E2BD0E66E16EC5AF049
:109BB00041E91200D9CFE6FFE1CFD9FF120051D819
:109BC00000091200E66EE66A9AEC2BF042E91200F8
:109BD00041E9E7CFD9FF120000EBF6FF01EBF7FFF9
:109BE000002A000E01220800F5CFE6FF7DEF4DF0C0
:109BF0004CD8002A000E0122EFCFE6FF7DEF4DF09A
:109C000042E9E7CFD9FF1200300EE66EA9DF41E945
:109C100012000F0E831401128398120000EBF6FF5E
:109C200001EBF7FF0800F55012000F0E9512838A22
:109C300012000401E46FF00E8314E411836E010E30
:109C40005DEF4EF0010E26D8E4DF0138F00B016E17
:109C5000020E20D8DEDF010ED5EF4DF01E0ED5EF3F
:109C60004DF0E66E39DF41E91200A4DF82E941E8F8
:109C7000FA0E026E1200010E98DF839AF00E95160E
:109C8000120098DF81E941E8120000EBE9FF01EBE7
:109C9000EAFF12008ADF8388020ED5EF4DF000380C
:109CA0000F0B0F0BC6DF0F0E0014C3DFBEDF010E5C
:109CB0001200010E7ADF15EF4EF0ECDF8398010EF3
:049CC000D5EF4DF09F
:0C9CC400FF0EE3CFEAFFE552FF0EE3CFF6
:109CD000E9FFE552E66AD9CFE6FFDACFE6FFFD0EEF
:109CE000E124D96EFF0EE220DA6EE66AE66A200E03
:109CF000EF5C06E0090EEF5C03E0EF6603D02CD0CA
:109D0000EE50F5D72D0EEF5C03E1FF0EE32A03D0F2
:109D10002B0EEF5C01E1EE502F0EEF6416D03A0EE1
:109D2000EF6013D0D890FB0EE336FE0EDFCFE3FFDB
:109D3000D890FB0EE336D890FB0EE336FE0EE350D0
:109D4000DF26300EEE5CDF26E7D7FF0EE3CFE8FF1D
:109D5000E85202E0DF1EDF2AE552E552FF0EE3CFB4
:109D6000DAFFE552FF0EE3CFD9FFE552FF0EE3CF56
:109D7000E8FFE6521200FF0EE3CFEAFFE552FF0EC6
:109D8000E3CFE9FFE552E66AE66AD9CFE6FFDACF2C
:109D9000E6FFFC0EE124D96EFF0EE220DA6EE66AE1
:109DA000E66AE66A200EEF5C06E0090EEF5C03E06F
:109DB000EF6603D03FD0EE50F5D72D0EEF5C03E1F8
:109DC000FF0EE32A03D02B0EEF5C01E1EE502F0EC5
:109DD000EF6424D03A0EEF6021D0D890F90EE3362C
:109DE000FA0EE336FD0EDECFE3FFFE0EDDCFE3FF1E
:109DF000D890F90EE336FA0EE336D890F90EE33632
:109E0000FA0EE336FD0EE350DE26FE0EE350DD22B1
:109E1000300EEE5CDE26000EDD22D9D7FF0EE3CF3A
:109E2000E8FFE85207E0F90EE31EE32AFA0ED8B481
:109E3000E306E31EE552E552E552FF0EE3CFDAFFFB
:109E4000E552FF0EE3CFD9FFE552E1CFE9FFE2CFC4
:109E5000EAFFED52ED52EECFF3FFEFCFF4FF120029
:109E6000D9CFE6FFDACFE6FFE66AE66AE66AE66A97
:109E7000E66AE66AE66AE66AE66AE66AF20EE3CF50
:109E8000E9FFF30EE3CFEAFF200EEF5C06E0090ED8
:109E9000EF5C03E0EF6603D07BD0EE50F5D72D0EDC
:109EA000EF5C03E1FF0EE38003D02B0EEF5C01E1DA
:109EB000EE50FA0EE124D96EFF0EE220DA6E2E0E7D
:109EC000EF5C04E1FF0EE382EE52F9D72F0EEF6450
:109ED00049D03A0EEF6046D0D890FA0EE336FB0E2A
:109EE000E336FC0EE336FD0EE336F60EDECFE3FF7F
:109EF000F70EDECFE3FFF80EDECFE3FFF90EDDCF86
:109F0000E3FFDD52DD52D890FA0EE336FB0EE33666
:109F1000FC0EE336FD0EE336D890FA0EE336FB0E68
:109F2000E336FC0EE336FD0EE336F60EE350DE2696
:109F3000F70EE350DE22F80EE350DE22F90EE35076
:109F4000DD22DD52DD52300EEE5CDE26000EDE221A
:109F5000DE22DD22DD52DD52FF0EE3A2B0D7FE0E7F
:109F6000E306ADD7FF0EE3A013D0FA0EE31EFB0EFF
:109F7000E31EFC0EE31EFD0EE31EFA0EE32A08E1CB
:109F8000FB0EE32A05E1FC0EE32A02E1FD0EE32AC3
:109F9000F20EE9CFE3FFF30EEACFE3FFEE0EE3CFDD
:109FA000D9FFEF0EE3CFDAFFFA0EE3CFDEFFFB0EB1
:109FB000E3CFDEFFFC0EE3CFDEFFFD0EE3CFDDFFE0
:109FC000DD52DD52F00EE3CFD9FFF10EE3CFDAFF21
:109FD000FE0EE3CFDFFFF20EE124E96EFF0EE2207A
:109FE000EA6EF60EE126FF0EE222FF0EE3CFDAFF65
:109FF000E552FF0EE3CFD9FFE552EECFF3FFEFCFEF
:04A00000F4FF120057
:0CA004006C0EE66EAC0EE66EE66A49ECEF
:10A010004DF043E9740EE66EAC0EE66E010E5ED9AD
:10A020007C0EE66EAC0EE66E020E58D9840EE66E1D
:10A03000AC0EE66E030E6EEF51F08C0EE66EAC0EBB
:10A040006ED9940EE66EAC0E6ED99C0EE66EAC0E1A
:10A050006ED9A40EE66EAC0E5ED1AC0EE66EAC0E02
:10A060005ED9B40EE66EAC0E5ED9BC0EE66EAC0EDA
:10A070005ED9C40EE66EAC0E4ED1CC0EE66EAC0EC2
:10A080004ED9D40EE66EAC0E4ED9DC0EE66EAC0E9A
:10A090004ED9E40EE66EAC0E3ED1D9CFE6FFE1CF4D
:10A0A000D9FF82E944E8AEDF000403E0040E005C5F
:10A0B00002E1C3DF09D0020E005C03E0050E005C84
:10A0C00002E1CBDF01D0D9DF0050040A14E0010A1D
:10A0D00012E0030A10E0070A0AE0030A08E0010A96
:10A0E00006E0030A0DE1EC0E026EAC0E07D0F80E8E
:10A0F000026EAC0E03D0040E026EAD0E036E02D0E3
:10A10000026A036A025003101DE0E66A060EE66E5C
:10A11000F4EC4CF042E9046A056A060E045C000E99
:10A12000055802E2E0D8F9D7010EE66E060EE66E9B
:10A13000F4EC4CF042E90C0E045C000E055802E20F
:10A14000D2D8F9D7E0D845E9E7CFD9FF1200D9CF67
:10A15000E6FFE1CFD9FF82E945E8660E026E720E96
:10A16000036E300E046E056E066A640E005C14E227
:10A170000A0EE66E00EBE6FF0FEC7AF041E9E750DD
:10A18000300F046E0A0EE66E00EBE6FF12EC7AF07A
:10A1900041E9E750300F056EDB0EE66E600EE66EAD
:10A1A000E66A060EC8D8D950020FE66EDACFE6FF8F
:10A1B000010EE66E060EE66E1CEC4DF044E946E933
:10A1C000E7CFD9FF12000F013E516BE04C0E0001AA
:10A1D000585D400E59590F0E5A59000E5B5920E236
:10A1E0000E0108510CE0010A0AE0030A08E0010A26
:10A1F00006E0070A04E0010A02E0030A18E1085138
:10A20000E96EEA6AD890E936EA36F20EE926040EDB
:10A21000EA22EECFE6FFEECFE6FFE66A090E06D0B1
:10A22000D60EE66E600EE66EE66A060E84D8D40E92
:10A23000E66E600EE66E54EC2DF042E9E80EE66E36
:10A24000030EE66EE66AE66A5CC0E6FF5DC0E6FF06
:10A25000E66AE66ABBEC2CF048E9D10EE66E600EC9
:10A26000E66E5BEC2DF042E9400EE66E420EE66EC5
:10A270000F0EE66EE66A58C0E6FF59C0E6FF5AC008
:10A28000E6FF5BC0E6FFBBEC2CF048E9880EE66E0B
:10A29000000EE66E010EE66E020EE66E1CEC4DF050
:10A2A00044E90F013F5118E0040E0001601514E16C
:10A2B00060BF03D060B307D002D060A104D0CB0E42
:10A2C000E66E600E03D0CE0EE66E600EE66EE66AB7
:10A2D000E66A33EC4DF044E983EF51F0E66E49EC69
:10A2E0004DF043E9120002500424F66E035005209D
:10A2F000F76E0800F5CFE6FF04EC4DF041E9042AC3
:10A30000000E05221200E60EE66E600EE66EE66AAC
:10A310000D0E9BEF51F0E66E070E6EEF51F0E66EFC
:10A32000040E6EEF51F0E66E050E6EEF51F0E66E24
:10A33000060E6EEF51F0E66E33EC4DF044E912007C
:10A34000645007E162966AD902E10AD8010C37D855
:10A35000010C040E645C03E1629640D8010C000C11
:10A3600057D941E8040104BF046B0B01926B8A6B5F
:10A370008B6B906B916B24EC53F0016A010E55D9F5
:10A3800019E20B018B5116E1F76A0134FE0BF66EF0
:10A39000F736850EF626AE0EF7220900F5CFE4F467
:10A3A0000800F5CFE5F4E5C4FAFF0401E451140018
:10A3B000012AE4D7A6D842E9E7CFD9FF1200020E5E
:10A3C0000B018A5D09E173D8040100BD02D0C80EFB
:10A3D00001D0880E006F1200BAEF52F0040E0B018C
:10A3E0009C5D0CE122C45EFF0F015E51000803E298
:10A3F0000B01050E02D00B01030E9C6F0B018A05A9
:10A4000010E111D8020E0B01925D03E10401840EEC
:10A4100006D0040104BD02D0C80E01D0880E046F1E
:10A420001200BAEF52F0F4D842E80B01080E905D2A
:10A43000000E91590DE29051016E9151026E9251B0
:10A4400002E1010E03D0920506E1020E926F03D0E5
:10A45000080E016E026A0401049304910250041371
:10A4600001EB05F401500B01905F0250915B280E47
:10A470008E6F040E8F6F0B019DA30BD00150021045
:10A4800012E08CCBF6FF8DCBF7FF0800F550B0D86B
:10A49000F5D70150021007E08CCBE9FF8DCBEAFF26
:10A4A000EF50A6D8F6D743E9E7CFD9FF1200B0D8CE
:10A4B00042E8030E04010015026E0151016E900E78
:10A4C000E96E0B0EEA6E0B01EE500124906FED5019
:10A4D0000220916F280E8C6F040E8D6F01500210B8
:10A4E0000CE08CCBE9FF8DCBEAFFEF508ECBE9FF80
:10A4F0008FCBEAFFEF6EA0D8F1D743E9E7CFD9FFC2
:10A50000120065980B018B5105E17AD8840E006F1B
:10A5100004011DD0040120AF1CD00B019051040197
:10A52000265D0B0191510401275904E226C490FBDA
:10A5300027C491FB78DF0B01010E8A6F61D8800E72
:10A54000006F0401280E066F040E076FC80E046F1B
:10A5500012000B01020E8A6F0401056BC80E046F16
:10A560000401080E016F280E026F040E036FC80E5F
:10A57000006F12004DD841E8020E0B018A5D2DE1FB
:10A580006550100B2AE0040101510401E46FE56BF2
:10A59000080EE41922E1E55120E140D81EE1005106
:10A5A000800B1BE1200E026F040E036F016A080E80
:10A5B0003CD81AE20150EA6A280FE96E040EEA223A
:10A5C000EF50E66E0150EA6A200FE96E040EEA22AF
:10A5D000E552E750EF6E012AEAD70B018A6B10D8DB
:10A5E0008C0E006F0401046B42E9E7CFD9FF120023
:10A5F0008ECBE9FF8FCBEAFFEF6E0B011CEF53F020
:10A600000401080E016F200E026F040E036F12008A
:10A61000D9CFE6FFE1CFD9FF81E912000401005153
:10A620003C0BE842E8420D081200F36EF46AF35066
:10A63000015C000EF45412008E2B000E8F238C2B25
:08A640008D230106025A1200ED
:08A6480004012051600BE842FF
:10A65000E842E842E842E842000901E012002151E4
:10A66000070A3FE00B0A3DE0070A32E0010A23E057
:10A670000B0A1FE0020A1DE0030A19E0080A10E0B5
:10A68000010A0CE00F0A08E0030A01E0120015D9E4
:10A690000B01040E9C6F120072EF53F0A9EF53F000
:10A6A0000CD90B019E0E8C6F0B0E8D6F0BD0CAEF69
:10A6B00053F0FCEF53F005D90B018D6B9F0F8C6F9E
:10A6C0000B0E8D230B019D930B01010E906F120059
:10A6D000F8D8EA6A9F0FE96E0B0EEA2222C4EFFF58
:10A6E00012001200800E0401205D32E12351030AA2
:10A6F0001FE0010A0AE0030A29E1DFD80B01E60E98
:10A700008C6FAD0E8D6F120E1ED0C1D87B0EF6264B
:10A71000AE0EC6D8020E0B01F76A8C25F66E8D516F
:10A72000F7220900F5CF90FB0A00F5CF91FB0ED080
:10A73000AED87F0EF626AE0EB3D88CCBF6FF8DCBFF
:10A74000F7FF0800F5500B01906F916B0B019D8393
:10A750001200B3D80F0EE66E4D0EE66E0F0EE66ECB
:10A760003CEC55F043E9010EE66E9F0EE66E0B0ED3
:10A77000E66E3CEC55F043E922C49EFB04012251F5
:10A7800004E10B01050E9C6F12000B01060E9C6F7D
:10A790000FEF4BF00401286B296B040120511F0BB4
:10A7A000020A0FE0030A0BE0010A18E186D804014F
:10A7B00028810B019DA112D0040128830FD07DD8E0
:10A7C0000DD04BD801E0010E56D88ECBE9FFEA6ED2
:10A7D000EF50040B03E00401010E286F0B018B0501
:10A7E0000AE10B01280E8C6F040E8D6F0B019D93F7
:10A7F0000B01020E906F1200040122050EE12051A0
:10A800001F0B00090AE159D8030E0401215D03E181
:10A810000B019D8102D00B019D91040122511CE18D
:10A8200020511F0B020818E124510F0B000914E0FE
:10A8300014D801E0010E1FD8030E0401215D04E1CC
:10A84000840E36D8EF6E120024AF03D031D8EF6AF1
:10A850001200880E2DD8EF6E120033D80F0B080DA2
:10A86000F3500401E56B000FE46F040EE5230401CF
:10A870002451800B1200040DF3500401E4250B0158
:10A880008E6F000E0401E5210B018F6F120015D8A9
:10A8900004012251F66EF76AD890F636F7361200A8
:10A8A000F7220900F5CF8CFB0A00F5CF8DFB1200D3
:10A8B0008ECBE9FF8FCBEAFF12000B01010E8B6FED
:0AA8C0001200FBDF04012451120016
:06A8CA0086A204D065B671
:10A8D00004D011D802D065B616D80B019C050AE148
:10A8E00065BA08D0626A0F015C6B5C815C890B0100
:10A8F000020E9C6F1200656A0F015C6B65860B018E
:10A90000010E9C6F1200656A0F015C6B0B019C6B62
:10A91000120083EF54F00B019C5101E112006250D0
:10A92000040B05E00F015C51040B01E04AD865B24D
:10A9300012006250010B05E00F015C51010B01E0B8
:10A9400071D86250100B05E00F015C51100B01E053
:10A9500032D86250400B05E00F015C51400B01E022
:10A960004BD86250200B05E00F015C51200B01E039
:10A9700045D86250020B05E00F015C51020B01E06B
:10A980004FD8030E0B019C5D01E212000B01A06B7E
:10A99000040EA05D0FE26250080B0CE00F015C5149
:10A9A000080B08E0A0EC51F0000901E162960B01F0
:10A9B000A02BEED712000F015C85629865825AEFDA
:10A9C00042F065920F015C9562A402D06294FCD7BC
:10A9D0005FEF42F00B019DA10ED0659265840B01E3
:10A9E000080EA16F070EA26FA107000EA25BA15176
:10A9F000A211FAE165941200629C12000F014CA1B1
:10AA00000DD0800E0401005D07E1840E0401045D99
:10AA100003E104018C0E006F0F014C91629A120049
:10AA2000636A1200636A626A0F019F0E5D6F0F0115
:10AA30007B0E5C6F0F015E6B0F0EE66E4D0EE66EC9
:10AA40000F0EE66E19D843E90F01160E4C6F62A681
:10AA500008D0629600000000000000000000000026
:10AA6000F6D76598BAEC52F00B019D910B019E6BE5
:10AA70000B01030E9C6F1200D9CFE6FFE1CFD9FF87
:10AA800084E901EBE9FF02EBEAFF005003E0EE6A24
:0CAA90000006FBD741E9E7CFD9FF120018
:04AA9C00D9CFE6FF29
:10AAA000DACFE6FFE1CFD9FFE2CFDAFF84E950E861
:10AAB000136AD950060FE66E000EDA20E66ED95002
:10AAC0000A0FE66E000EDA20E66E00EBE6FF01EB01
:10AAD000E6FF30EC4FF046E9F350046EF450056E9B
:10AAE00004EBE9FF05EBEAFFEF50DF0B45080CE153
:10AAF000042A000E052204EBE6FF05EBE6FFBBECA3
:10AB00004EF042E9F3500A2606EBE6FF07EBE6FFBC
:10AB100008EBE6FF09EBE6FFC0EC7CF07FD80A50BB
:10AB200062E00A3406E3010E136EFF0E0A02F350D0
:10AB30000A6E0F6A106A800E116E3F0E126ED89068
:10AB40000A5002E6140E0A5C0AE3EC0EE66E780E7A
:10AB5000E66EAD0EE66E600E54D8140E0A5ED89006
:10AB60000A5002E60A0E0A5C0AE3F90EE66E020ECD
:10AB7000E66E150EE66E500E44D80A0E0A5ED890A8
:10AB80000A5002E6050E0A5C09E3E66A500EE66E1C
:10AB9000C30EE66E470E35D8050E0A5ED8900A50F1
:10ABA00002E6020E0A5C08E3E66AE66AC80EE66E92
:10ABB000420E27D8020EF1D7D8900A5002E6010EB5
:10ABC0000A5C07E3E66AE66A200EE66E410E19D8D3
:10ABD0000A06135004E02BD8E5EC7CF003D027D80C
:10ABE000EAEC7BF01BD80BEBFCF00CEBFDF00DEB73
:10ABF000FEF00EEBFFF051E9E5CFDAFFE7CFD9FF2A
:10AC00001200E66E2AD8EAEC7BF01BD80F6EE551F5
:10AC1000106EE651116EE751126E120012D80B6ED3
:10AC2000E5510C6EE6510D6EE7510E6E120015D80F
:10AC30000BEBE6FF0CEBE6FF0DEBE6FF0EEBE6FFA2
:10AC40001200E552E5CFE7F4E5CFE6F4E5CFE5F411
:10AC5000E7CFE4F40401E45112000FEBE6FF10EB40
:0CAC6000E6FF11EBE6FF12EBE6FF12002E
:04AC6C00070F1C189A
:10AC7000181818181C1E070B0B1313131919191A7F
:10AC80001A1C0F070303030303071E1C0000000028
:10AC900000000000060E1E1E06060606000000004C
:10ACA000000000000606060606060F0F070F1C1818
:10ACB000180000001C1E0703070E1C1803070E1CBB
:10ACC00018181F1F0000000000001F1F1F1F18186A
:10ACD00018181F1F1E1E00000000181C0000000096
:10ACE000181C0F070703030303071E1C2020202046
:10ACF0000405202020200607202004050001202034
:10AD0000060702030405000100010607020302030F
:10AD10002020350020313000203230002035300036
:0CAD20003130300032303000353030006F
:04AD2C0056003E3E51
:10AD30003E3E45003E3E3E3E52003E3E3E3E5300BD
:10AD40003E3E3E3E44003E3E3E3E4D003E3E3E3E8A
:10AD500050574D007878454E4300787843454E4330
:10AD600000014D53000000004D54000000004D4311
:10AD700000000000524C0000000052520000000091
:10AD800052540000000054534B455700544C454E5C
:10AD90000001545245464C00545452414E00544216
:10ADA0004350000154424300080854464F4C4400AD
:10ADB0004F505400A8A8425000000000524C455685
:10ADC000000153544442590042504D007878535486
:10ADD00042454E0053554D007878424154454E004F
:06ADE00052444241540000
:0AADE6001201000202000008741CB4
:10ADF000C80001000102000109024300020100C075
:10AE000032090400000102020100052400100104BF
:10AE10002402020524060001052401000107058221
:10AE20000308000209040100020A000000070503EC
:10AE300002400000070583024000000403090420CB
:10AE400003500048004F0054004F0056004F005878
:10AE500000200073002E0072002E006C002E001CDB
:10AE600003500068006F0074006F004500750072A9
:10AE7000006F00200034002E003000F8ADF8AD3B2C
:07AE8000AE3FAE5FAE7A9514
:01AE870000CA
:08AE8800000EF66EC80EF76E15
:10AE9000000EF86E0B010900F550856F0900F550A2
:10AEA000866F03E1856701D03DD00900F550806FC2
:10AEB0000900F550816F0900F550826F0900090003
:10AEC000F550E96E0900F550EA6E09000900090025
:10AED000F550836F0900F550846F09000900F6CF23
:10AEE00087FBF7CF88FBF8CF89FB80CBF6FF81CBC0
:10AEF000F7FF82CBF8FF0B01835302E1845307E095
:10AF00000900F550EE6E8307F8E28407F9D787CB86
:10AF1000F6FF88CBF7FF89CBF8FF0B018507000E02
:06AF2000865BBFD71200A2
:0AAF2600D9CFE6FFDACFE6FFE1CF56
:10AF3000D9FFE2CFDAFF86E9C098C26AC16A02404F
:10AF40007F0B3C0BC26E0250400DF350C00BC2127F
:10AF5000800E0314C16E03380F0B070BC112035090
:10AF6000040DF350380BC112C08800EBC1FF04017F
:10AF700001EBE4F4E56BE4C4C2FFC09802AE03D079
:10AF80009E9C9D8CF28CC28041E9E5CFDAFFE7CF31
:04AF9000D9FF1200D3
:0CAF9400D9CFE6FFDACFE6FFFA0EE3CFDC
:10AFA000D9FFFB0EE3CFDAFFFC0EE3CFE9FFFD0E86
:10AFB000E3CFEAFFE9CFF3FFEACFF4FFDECFEFFF05
:10AFC000EE66FCD7FF0EE3CFDAFFE552FF0EE3CFCC
:10AFD000D9FFE5521200FE0EE3CFE9FFFF0EE3CFEB
:10AFE000EAFFF36AF46AEE5203E0F34AF42AFBD76D
:02AFF00012004D
:0EAFF200D9CFE6FFDACFE6FFE1CFD9FFE2CFFD
:10B00000DAFF83E942E80C0EB66E050EF66EF76ABB
:10B01000300EF86E0800F550010B02E0046801D014
:10B02000046A949279B605D0CA9400EBCBFFCA8427
:10B0300004D0769400EB77FF768443E9E5CFDAFF1E
:06B04000E7CFD9FF12006A
:0AB04600F36AF46AFF0EE124E96EDC
:10B05000FF0EE220EA6EED6607D01F0EEF6404D00B
:10B060007F0EEF6001D0F32A1200FF0EE124E96E9B
:10B07000FF0EE220EA6EEDCFF4FFEFCFF3FFF466B0
:10B0800007D0600EF36404D07B0EF36001D0F39A16
:02B090001200AC
:0EB09200D9CFE6FFDACFE6FFE1CFD9FFE2CF5C
:10B0A000DAFF84E942E880EB04F081EB05F0060E5C
:10B0B000D89004360536E804FBE105EB71FF044047
:10B0C000E8423F0B300B0401E46FCF0E7014E41123
:0EB0D000706E43E9E5CFDAFFE7CFD9FF12003B
:02B0DE00D9CFC8
:10B0E000E6FFDACFE6FFE1CFD9FFE2CFDAFF84E96E
:10B0F00042E880EB04F081EB05F0060ED8900436B0
:10B100000536E804FBE105EB74FF0440E8423F0B21
:10B11000300B0401E46FCF0E7314E411736E43E936
:0AB12000E5CFDAFFE7CFD9FF1200F8
:06B12A00D9CFE6FFDACFE9
:10B13000E6FFE1CFD9FFE2CFDAFF84E942E880EB16
:10B1400004F081EB05F0060ED89004360536E804CD
:10B15000FBE105EBB2FF0440E8423F0B300B04017A
:10B16000E46FCF0EB114E411B16E43E9E5CFDAFF1D
:06B17000E7CFD9FF120039
:0AB17600D9CFE6FFDACFE6FFE1CF04
:10B18000D9FFE2CFDAFF84E942E880EB04F081EBFB
:10B1900005F0060ED89004360536E804FBE105EB11
:10B1A000B7FF0440E8423F0B300B0401E46FCF0EC1
:10B1B000B614E411B66E43E9E5CFDAFFE7CFD9FF65
:02B1C00012007B
:0EB1C200D9CFE6FFDACFE6FFE1CFD9FFE2CF2B
:10B1D000DAFF84E942E880EB04F081EB05F0060E2B
:10B1E000D89004360536E804FBE105EBBCFF0440CB
:10B1F000E8423F0B300B0401E46FCF0EBB14E411A7
:0EB20000BB6E43E9E5CFDAFFE7CFD9FF1200BE
:02B20E00D9CF96
:10B21000E6FFDACFE6FFE1CFD9FFE2CFDAFF83E93D
:10B220000C0EBB1294947950400B08E07950080B37
:10B2300005E0769400EB77FF768404D0CA9400EBA7
:10B24000CBFFCA8441E9E5CFDAFFE7CFD9FF12008F
:04B2500094941200C0
:0CB25400D9CFE6FFDACFE6FFE1CFD9FF4B
:10B26000E2CFDAFF83E90C0E706E7950400B08E1F3
:10B270007950080B05E1CA9400EBCBFFCA8404D0D7
:10B28000769400EB77FF7684989841E9E5CFDAFF72
:06B29000E7CFD9FF120018
:0AB29600D9CFE6FFDACFE6FFE1CFE3
:10B2A000D9FFE2CFDAFF83E90C0E736E98967950DE
:10B2B000400B08E17950080B05E1CA9400EBCBFF85
:10B2C000CA8404D0769400EB77FF768441E9E5CF19
:08B2D000DAFFE7CFD9FF1200FD
:08B2D800D9CFE6FFDACFE6FF53
:10B2E000E1CFD9FFE2CFDAFF83E97E0E0014CD6E05
:10B2F00000AC02D0CD8E01D0CD9ECF6ACE6A9E909A
:10B3000000AE02D09D8001D09D90CD8041E9E5CF77
:08B31000DAFFE7CFD9FF1200BC
:08B31800D9CFE6FFDACFE6FF12
:10B32000E1CFD9FFE2CFDAFF83E90C0EB16E79509D
:10B33000400B08E17950080B05E1CA9400EBCBFF04
:10B34000CA8404D0769400EB77FF768441E9E5CF98
:08B35000DAFFE7CFD9FF12007C
:08B35800D9CFE6FFDACFE6FFD2
:10B36000E1CFD9FFE2CFDAFF83E97F0E0014D56E7B
:10B37000D76AD66AF29400AE02D0F28A01D0F29A6D
:0EB38000D58E41E9E5CFDAFFE7CFD9FF120005
:02B38E00D9CF15
:10B39000E6FFDACFE6FFE1CFD9FFE2CFDAFF83E9BC
:10B3A000FB0E0014CA6ECC6A9E9200AE02D09D8243
:10B3B00001D09D92CA8441E9E5CFDAFFE7CFD9FFFA
:02B3C000120079
:0EB3C200D9CFE6FFDACFE6FFE1CFD9FFE2CF29
:10B3D000DAFF83E9C098C30EC2140401E46F004091
:10B3E0007F0B3C0BE411C26E41E9E5CFDAFFE7CFFA
:04B3F000D9FF12006F
:0CB3F400FF0EE3500B01A36F480E01D0C8
:10B400004C0EE76EE72EFED7E76AE72EFED7A32F96
:04B41000F7D7120058
:0CB41400C4CFE6F4E6C4E7F40401E66BE4
:0CB42000C350E611F36EE7C4F4FF120005
:04B42C00FF0EE350DC
:10B43000E84E1200000000D000D000D0E82EFAD76D
:02B440001200F8
:0EB4420000EE00F00F0EEE6AEA62FDD7120077
:0CB45000C098C250020B01E0010E120077
:04B45C00C098C28250
:02B460001200D8
:0EB46200000000000005000A00140032006423
:05B4700000C800F4011A
:09B47500000000000000000000CE
:02B47E0010AD0F
:0CB4800014AD18AD1CAD20AD24AD28ADFE
:10C000000000000000000000000000000000000030
:10C010000000000000000000000000000000000020
:10C020000000000000000000000000000000000010
:10C030000000000000000000000000000000000000
:10C400001027C422280A1405FF32EC2C942A840336
:10C41000F401FF46A816C0122C016400FF1EA816E6
:10C42000C012C8004B00FF056829E42540068403BC
:10C43000FF280C30502D8403F401FF469C18B414DF
:10C440002C016400FF1E9C18B414AF004B00FF05C4
:10C45000242C3C28D007B004FF46C832A82FE8039C
:10C460005802FF466419E0152C016400FF1E641990
:10C47000E015AF004B00FF05502D302A8403F40176
:10C48000FF3C903338314006E803FF46F41A761635
:10C490002C016400FF1EF41A7616AF004B00FF0556
:10C4A000502D302AD0071405FF464C369033A40691
:10C4B000E803FF46201C38182C016400FF1E201CD6
:10C4C0003818AF004B00FF05442F242C9808A40611
:10C4D000FF46A438E835A406E803FF464C1D64195E
:10C4E0002C016400FF1E4C1D6419AF004B00FF05BA
:10C4F0003831182E280A0807FF46983A40386C074A
:10C50000B004FF46781EC8192C016400FF1E781E77
:10C51000C819AF004B00FF0500000000000000003C
:10C52000000000000000000000000000000000000B
:10C5300000000000000000000000000000000000FB
:10C5400000000000000000000000000000000000EB
:10C5500000000000000000000000000000000000DB
:10C800000500FEFB0000A50B0000010000007EB447
:10C810000000F20400000E00000087AE0000A40B30
:10C8200000000100000075B40000930B0000090037
:0EC83000000062B40000D104000013000000FC
:02C83E0068ECA4
:10C8400073F082E943E800CEE4F4080EB9EC72F02C
:10C8500053E0550EE66E6B0E23EC73F00E0108519B
:10C86000070A2AE0010A24E0030A1EE0010A18E090
:10C87000070A12E0010A0CE0030A06E0010A20E1BF
:10C880004D0EE66E6B0E1FD0440EE66E6B0E1BD087
:10C890003B0EE66E6B0E17D0320EE66E6B0E13D0AB
:10C8A000280EE66E6B0E0FD01E0EE66E6B0E0BD0D2
:10C8B000140EE66E6B0E07D0010EE66E6B0E03D003
:10C8C000F70EE66E6A0E23EC73F0000E0E01085DA3
:10C8D00018E30851070815E3D0EC6BF0FFEC73F098
:10C8E0000401F350F41004E0F40EE66E6A0E07D073
:10C8F000E70EE66E6A0E03D0D20EE66E6A0E23ECE9
:10C9000073F0005001E1EED0FEEC72F0040EB9ECD1
:10C9100072F00DE07FEC4BF0C90EE66E6A0E5FEC34
:10C9200075F00ACEE6FF0BCEE6FF7BEC77F0FEEC6F
:10C9300072F0100EB9EC72F01FE00E010951030AFB
:10C9400012E0010A0CE0030A06E0010A10E1AB0E56
:10C95000E66E6A0E0FD0910EE66E6A0E0BD07B0E5D
:10C96000E66E6A0E07D0620EE66E6A0E03D04D0EBA
:10C97000E66E6A0E23EC73F0FEEC72F0020EB9EC78
:10C9800072F018E07FEC4BF0440EE66E6A0E5FEC3E
:10C9900075F00ECEE6FF0FCEE6FF88EC75F0360E92
:10C9A000E66E6A0E2AEC77F010CEE6FF11CEE6FFB7
:10C9B0007BEC77F0FEEC72F0200EB9EC72F009E03F
:10C9C000250EE66E6A0EE66E2E0EE66E0E0E3BEC41
:10C9D00074F0FEEC72F0400EB9EC72F024E0000E40
:10C9E0000E01085D17E30851020814E3140EE66E09
:10C9F0006A0EE66E350EE66E0E0E3BEC74F0030E1C
:10CA0000E66E6A0EE66E3C0EE66E0E0E3BEC74F0C1
:10CA100034EC77F0030E0E01085D05E308510608BB
:10CA200002E334EC77F0FEEC72F0800EB9EC72F0B9
:10CA30001BE0E10EE66E690EE66E4A0EE66E0E0E25
:10CA40003BEC74F0D00EE66E690EE66E510EE66EAB
:10CA50000E0E3BEC74F0BF0EE66E690EE66E580EDD
:10CA6000E66E0E0E3BEC74F06BEC77F0010E34ECDE
:10CA700073F009E0AE0EE66E690EE66E5F0EE66ECE
:10CA80000E0E3BEC74F0005001082CE26BEC77F0DA
:10CA9000040E34EC73F019E0030E0E01085D0CE394
:10CAA0000851060809E39D0EE66E690EE66ECE0E8D
:10CAB000E66E0E0E3BEC74F08C0EE66E690EE66EC2
:10CAC000D50EE66E0E0E3BEC74F06BEC77F0020EBA
:10CAD00034EC73F007E0C80EE66E0E0EE66EF3EC73
:10CAE0003FF042E90050020808E26BEC77F0010EDB
:10CAF00034EC73F002E0E2EC35F00050030851E250
:10CB0000FEEC72F0010EB9EC72F04BE0F40EE66E42
:10CB10006A0E23EC73F0026A0250050842E3EA6AE7
:10CB2000023481EC77F00234E4EC72F09FEC74F0A4
:10CB3000036EF450046E7FEC4BF0850EE66E690ECA
:10CB40005FEC75F0E66A0250E66EE66A5DEC2CF08A
:10CB500043E9790EE66E690E56EC75F0EA6A023426
:10CB6000E4EC72F05BEC77F06F0EE66E690E56EC5B
:10CB700075F0EA6A023417EC73F05BEC77F0650E3F
:10CB8000E66E690E2AEC77F003EBE6FF04EBE6FFB6
:10CB900088EC75F05F0EE66E690E9EEC73F0022A6B
:10CBA000BBD7005001E03BD844E9E7CFD9FF1200E2
:10CBB00068EC73F085E900EBE6FF01EBE6FFF4ECCF
:10CBC0004BF042E95A0EE66E690E5FEC75F0A1EC8F
:10CBD00075F0EE52C5EC73F088EC75F04E0EE66E13
:10CBE000690E2AEC77F0A1EC75F0F9EC72F0C5EC67
:10CBF00073F088EC75F03E0EE66E690E56EC75F03B
:10CC0000A1EC75F0BCEC76F05BEC77F0F40EE66E20
:10CC10006A0E9EEC73F041E9E7CFD9FF12000E01D6
:10CC200064EC75F001E1D6D0F40EE66E6A0E23ECEA
:10CC300073F004CEE4F4010EB9EC72F005E0200EBE
:10CC4000E66E690E23EC73F004CEE4F4020EB9EC48
:10CC500072F005E0090EE66E690E23EC73F004CE67
:10CC6000E4F4040EB9EC72F005E0F00EE66E680E26
:10CC700023EC73F004CEE4F4080EB9EC72F005E096
:10CC8000D70EE66E680E23EC73F004CEE4F4100EBB
:10CC9000B9EC72F005E0B20EE66E680E23EC73F0AC
:10CCA00004CEE4F4200EB9EC72F005E0900EE66ECE
:10CCB000680E23EC73F004CEE4F4400EB9EC72F08D
:10CCC00005E06A0EE66E680E23EC73F0FCEC74F07F
:10CCD000010E34EC73F005E0450EE66E680E23ECB1
:10CCE00073F0FCEC74F0020E34EC73F005E0230EEC
:10CCF000E66E680E23EC73F0FCEC74F0040E34EC7A
:10CD000073F005E0FD0EE66E670E23EC73F0FCECAD
:10CD100074F0100E34EC73F005E0D70EE66E670E7B
:10CD200023EC73F0FCEC74F0200E34EC73F005E0AF
:10CD3000B40EE66E670E23EC73F0FCEC74F0400E5C
:10CD400034EC73F005E08D0EE66E670E23EC73F0A5
:10CD50008BEC74F0010E31EC74F005E0670EE66EBA
:10CD6000670E23EC73F08BEC74F0020E31EC74F070
:10CD700005E0440EE66E670E23EC73F08BEC74F066
:10CD8000040E31EC74F005E01D0EE66E670E23EC28
:10CD900073F08BEC74F0080E31EC74F005E0FB0ED0
:10CDA000E66E660E23EC73F08BEC74F0100E31EC33
:10CDB00074F005E0E10EE66E660E23EC73F08BEC8A
:10CDC00074F0200E31EC74F005E0C70EE66E660ECE
:10CDD00023EC73F012000E010869006B80EF75F010
:10CDE0003AEC77F041E80E010869010E006F80EC23
:10CDF00075F0016A0C0E015C16E2EDEC73F0EF6A5F
:10CE0000EDEC73F0EE52EE6AED6AEDEC73F0F9ECD6
:10CE100072F0EE6AED6AEDEC73F0BCEC76F0EE6A5F
:10CE2000ED6A012AE7D742E9E7CFD9FF12003AECD1
:10CE300077F047E800CEE4F4010EB9EC72F001E1BE
:10CE4000A1D0010E016E0150020832E379EC74F0BA
:10CE500000012551065C2651075805E2D9EC72F015
:10CE60008CEC75F0F5D74BEC76F00450065C055071
:10CE700007580CE2D9EC72F0A7EC74F003E2AAECCC
:10CE800077F004D0062A000E0722EFD78BEC76F05D
:10CE900007340CE2D9EC72F0A7EC74F003E2ADECCD
:10CEA00077F004D00606000E075AF2D7012ACBD736
:10CEB000030E016E015005084EE379EC74F0000199
:10CEC0002551065C2651075805E2D9EC72F08CEC2E
:10CED00075F0F5D74BEC76F00450065C055007581A
:10CEE0000CE2D9EC72F0B6EC74F003E2AAEC77F045
:10CEF00004D0062A000E0722EFD78BEC76F0073419
:10CF00000CE2D9EC72F0B6EC74F003E2ADEC77F021
:10CF100004D00606000E075AF2D7030E015C03E0A8
:10CF2000050E015C16E1B6EC78F0EE50ED100FE066
:10CF3000EA6A0134CDEC76F00404E66F000E055881
:10CF4000E76FE651E41905E1E751E51902E10E0149
:10CF50000481012AAFD70E0118511C25126F1951F7
:10CF60001D21136FD89013331233245128251E6FBF
:10CF7000255129211F6FD8901F331E3364EC75F0A3
:10CF800001E1008348E9E7CFD9FF12003AEC77F0DE
:10CF900046E800CEE4F4020EB9EC72F064E00E0153
:10CFA00018511C5D0E6F19511D590F6F2451285DCA
:10CFB000106F25512959116F320EE66EE66A0ECEBA
:10CFC000E6FF0FCEE6FF65EC7BF0E552E5CF0FFE06
:10CFD000E7CF0EFE320EE66EE66A10CEE6FF11CE09
:10CFE000E6FF65EC7BF0E552E5CF11FEE7CF10FEE2
:10CFF0000F012F51016E3051026EE668E668ABEC0E
:10D0000075F065EC7BF0E552E550046EE750036E79
:10D010000E010F3502500F1904E60E51015C0F513D
:10D02000025809E304340F51041804E603500E5D5E
:10D0300004500F5901E2048311350250111904E61E
:10D040001051015C1151025809E3043411510418C4
:10D0500004E60350105D0450115901E2048364ECAE
:10D0600075F001E10085B0EF75F03AEC77F044E837
:10D0700000CEE4F4040EB9EC72F04FE00E0118514A
:10D08000245D016E25511955026E1C51285D036EF9
:10D0900029511D55046ED8800F5104E7FF0E0E5D17
:10D0A000FF0E0F5916E30F3504E20E510108000E72
:10D0B0000F550FE3D880115104E7FF0E105DFF0EEE
:10D0C000115907E3113513E210510108000E1155F3
:10D0D0000EE20F350F51111904E60E51105D0F517C
:10D0E000115905E203EB0CFE04EB0DFE09D00150D3
:10D0F00003240C6F025004200D6FD8900D330C33B5
:10D100000CCEE6FF0DCEE6FFF2EC2BF042E9F3CFBA
:10D110000AFEF4CF0BFE0E01008745E9E7CFD9FFE9
:10D1200012003AEC77F046E80E01086900CEE4F40C
:10D13000080EB9EC72F001E194D00E0100890A5199
:10D14000016E0B51026E31CFE4F432CFE5F40401ED
:10D15000E66BE76BE00EE4272E0E7BEC73F0E00E3F
:10D16000E86F2E0E9BEC72F006E3CEEC74F003E356
:10D170000E01086B76D034EC74F09C0EE427310E6F
:10D180007BEC73F09C0EE86F310E9BEC72F006E3C3
:10D19000CEEC74F003E30E01010E5ED034EC74F0BB
:10D1A000F40EE427330E7BEC73F0F40EE86F330ECD
:10D1B0009BEC72F006E3CEEC74F003E30E01020E7A
:10D1C0004BD034EC74F0B00EE427360E7BEC73F0E9
:10D1D000B00EE86F360E9BEC72F006E3CEEC74F006
:10D1E00003E30E01030E38D034EC74F06C0EE42728
:10D1F000390E7BEC73F06C0EE86F390E9BEC72F01D
:10D2000006E3CEEC74F003E30E01040E25D034ECFB
:10D2100074F0C40EE4273B0E7BEC73F0C40EE86F91
:10D220003B0E9BEC72F006E3CEEC74F003E30E01D0
:10D23000050E12D034EC74F0800EE4273E0E7BEC29
:10D2400073F0800EE86F3E0E9BEC72F007E3CEECBD
:10D2500074F004E30E01060E086F03D00E0100996E
:10D260000487B0EF75F03AEC77F064E80E01096BD3
:10D27000640EE66EE66A250E1CEC77F065EC7BF03A
:10D28000A6EC75F01E6EE7501D6E00CEE4F4100E95
:10D29000B9EC72F001E100D1010E016E086E020ED0
:10D2A0000F6E166E0E01080503E0020E085D23E105
:10D2B000D950010F4BEC74F01A0E0BEC73F0CBEC61
:10D2C0006DF046E9D950AAEC76F01A0E1BEC74F01A
:10D2D000CBEC6DF006EC75F01A0E40EC74F0CBEC74
:10D2E0006DF046E9D950B3EC76F01A0EACEC73F061
:10D2F000CBEC6DF046E9030E0E01085D1FE1D9503D
:10D30000010F4BEC74F00E0E0BEC73F0C9DB46E929
:10D31000D950AAEC76F00E0E1BEC74F0C1DB06ECD3
:10D3200075F00E0E40EC74F0BBDB46E9D950B3EC5F
:10D3300076F00E0EACEC73F0B3DB46E90E0108514B
:10D3400009E0040E085D06E0050E085D03E0060E28
:10D35000085D16E1D950010F86EC77F0AAEC76F063
:10D36000230E1BEC74F0B4EC75F00F0F86EC77F025
:10D37000B3EC76F0230EACEC73F054EC6EF046E9AF
:10D380000E01096B09500A5D096E0A500B590A6EAD
:10D3900017500A5D176E18500B59186E246A1F6AD1
:10D3A000040E1F5C24E2E66AB9EC75F0DACFE9F40A
:10D3B0001F50070DE851F324E66FDA50F420E76FB1
:10D3C000E6C4E6FFE66E10DA43E9E66E0401CAEC55
:10D3D00073F0E552E750EF6ECAEC73F0EF50245C47
:10D3E00004E2CAEC73F0EF50246E1F2AD9D71F6AEB
:10D3F000040E1F5C2BE20401CAEC73F0EF50245CB6
:10D4000023E1D950010FE66FDACFE7F41F50070D83
:10D41000E6512CEC75F0BAEC78F0D950010FEA6FB8
:10D42000DACFEBF40E010951070D0401EA512CEC9F
:10D4300075F0EECFE8F4EFCFE9F4E451E85DE551A3
:10D44000E95902E21FEB09FE1F2AD2D70401D95085
:10D45000010FE46FDACFE5F40E010951070D040165
:10D46000E45160EC77F0EECF2EFEEECF2FFEEECF44
:10D4700030FEEECF31FEEECF32FEEECF33FEEFCFF9
:10D4800034FEE66A2E0EE66E0E0E8CEC77F0C5ECDE
:10D4900074F0600E0E01001365E9E7CFD9FF1200AA
:10D4A0003AEC77F050E8106A00CEE4F4400EB9ECA4
:10D4B00072F001E1B8D0000E0E01085D01E281D0EA
:10D4C0000851020801E27DD00951030A0BE0010A6C
:10D4D00005E0030A03E0010A09E104D0050E0D6E20
:10D4E000030E03D0030E0D6E050E0E6E0DEB35FE12
:10D4F000040E3C6F0EEB43FE350EE66E0E0EE66E2E
:10D50000EA6A0D34CDEC76F091EC74F0EA6A0D34F1
:10D51000E5EC76F03C0EE66E0E0EE66E22CEE4F4FE
:10D5200023CEE5F491EC74F00C0EACEC73F0E6EC69
:10D530006EF046E97AEC78F091EC74F0EA6A0E3419
:10D54000E5EC76F00E0109A10ED036510A5D366F7A
:10D5500037510B59376F3D510A5D3D6F3E510B59A5
:10D560003E6F93EC75F0010EE66E350EE66E0E0E14
:10D57000ECEC72F02FEC75F0010EE66E3C0EE66EF0
:10D580000E0EECEC72F039EC75F0010EBFEC78F099
:10D59000ECEC72F012EC75F039A110D00F6A030EAA
:10D5A0000F5C09E2B9EC75F00F505DEC74F001E12D
:10D5B000102A0F2AF4D7020E105C33E23DEC73F010
:10D5C0002ED00951030A0AE0010A06E0030A04E02A
:10D5D000010A06E1050E03D0040E01D0050E0E6E01
:10D5E0000EEB43FE7AEC78F00401160E9BEC76F01D
:10D5F000EA6A0E34E4EC72F061EC78F0160EE6277D
:10D6000072EC74F071EC6FF046E90E0109A102D0E2
:10D6100093EC75F0010EBFEC78F08CEC77F0C5EC74
:10D6200074F00E01008F51E9E7CFD9FF12003AECF8
:10D6300077F056E8166A00CEE4F4800EB9EC72F08A
:10D6400001E1AAD00E010951030A19E0010A0CE018
:10D65000030A06E0010A1EE1030E136E050E07D051
:10D66000050E136E030E0ED0050E136E030ED6ECD0
:10D6700073F0E45D0D6E41E9E550E5590AD0030E03
:10D68000136E050ED6EC73F0E4250D6E41E9E550FE
:10D69000E5210E6E13EB4AFE0E01040E516F14EBE2
:10D6A00058FEEA6A1334E4EC72F004EC74F0EA6AAF
:10D6B000133401EC77F04A0EE66E0E0E24EC74F093
:10D6C0001A0EE96E0E0EEA6E04EC74F00E011A5199
:10D6D0000D24116E1B510E20126E140ECFEC72F041
:10D6E000510EE66E0E0E24EC74F0EA6A1434E4EC8B
:10D6F00072F004EC74F0EA6A143401EC77F0580E1E
:10D70000E66E0E0E24EC74F00E0109A112D04B51FE
:10D710000A5D4B6F4C510B594C6F52510A5D526F61
:10D7200053510B59536F59510A5D596F5A510B5947
:10D730005A6F020EE66E4A0EE66E0E0EECEC72F0BA
:10D740002FEC75F0020EE66E510EE66E0E0EECEC4E
:10D7500072F039EC75F0020EE66E580EE66E0E0EA3
:10D76000ECEC72F012EC75F039A310D0156A030ED0
:10D77000155C09E2B9EC75F015505DEC74F001E14F
:10D78000162A152AF4D7020E165C04E23DEC73F05B
:10D79000C5EC74F00E01018157E9E7CFD9FF120003
:10D7A00000CEE4F4800EB9EC72F01AE00E0164ECE5
:10D7B00075F012E00F0139A711D04DEC75F00F0E86
:10D7C0000401E517FCEC76F007E04DEC75F0F00E87
:10D7D000E617FCEC76F002E1010E03D0000E01D05A
:10D7E000000EF36EF46A120068EC73F084E94DE801
:10D7F000046A0050030A42E0010A2DE0030A18E01F
:10D80000010A02E0000E83D03DEC77F00900F550EC
:10D810009BEC78F0020E5DEC76F0040E64EC76F092
:10D82000060E6BEC76F0080ED0EC76F0090E38D0D0
:10D830003DEC77F00A0EC1EC76F00C0E5DEC76F064
:10D840000E0E64EC76F0100E6BEC76F0120ED0EC4F
:10D8500076F0130E25D03DEC77F0140EC1EC76F087
:10D86000160E5DEC76F0180E64EC76F01A0E6BEC8A
:10D8700076F01C0ED0EC76F01D0E12D03DEC77F059
:10D880001E0EC1EC76F0200E5DEC76F0220E64ECFC
:10D8900076F0240E6BEC76F0260ED0EC76F0270EA8
:10D8A00087EC73F00F6E106A12EC74F0EE520750B2
:10D8B000EE5C0850ED580AE312EC74F0EE52EE50B4
:10D8C000055CED50065802E32D0E042670EC77F04F
:10D8D0000B50EE5C0C50ED5809E370EC77F0EE5015
:10D8E000095CED500A5802E3160E042685EC78F028
:10D8F0000F50EE5C1050ED5809E385EC78F0EE50D7
:10D900000D5CED500E5802E3210E042604504EE942
:10D91000E7CFD9FF120068EC73F084E951E8046A9C
:10D92000056A066A076A146A0050030A4FE0010A92
:10D9300037E0030A1FE0010A06E00001FC6BFD6B03
:10D94000FE6BFF6BA9D03DEC77F00900F550A1EC20
:10D9500078F0020E72EC76F0040E79EC76F0060E9A
:10D9600080EC76F0080ED5EC76F0090E73EC77F0CB
:10D97000040E41D03DEC77F00A0EC4EC76F00C0EAC
:10D9800072EC76F00E0E79EC76F0100E80EC76F0FC
:10D99000120ED5EC76F0130E73EC77F0080E2BD048
:10D9A0003DEC77F0140EC4EC76F0160E72EC76F0C7
:10D9B000180E79EC76F01A0E80EC76F01C0ED5EC91
:10D9C00076F01D0E73EC77F00C0E15D03DEC77F071
:10D9D0001E0EC4EC76F0200E72EC76F0220E79EC7E
:10D9E00076F0240E80EC76F0260ED5EC76F0270E3D
:10D9F00073EC77F0100E146E12EC74F0EE520A50C5
:10DA0000EE5C0B50ED5808E312EC74F0EE52EE5061
:10DA1000085CED50095803E259EC75F0EE8070ECAB
:10DA200077F00E50EE5C0F50ED5807E370EC77F096
:10DA3000EE500C5CED500D5803E259EC75F0EE829F
:10DA400085EC78F01250EE5C1350ED5807E385EC4E
:10DA500078F0EE50105CED50115803E259EC75F07F
:10DA6000EE8404EBE4F405EBE5F406EBE6F407EBF7
:10DA7000E7F414501F0B08E00401D890E437E537B1
:10DA8000E637E737E806F9E1E4C4FCF0E5C4FDF069
:10DA9000E6C4FEF0E7C4FFF052E9E7CFD9FF120079
:10DAA00023EC78F0D3EC74F02CE3116A126A0401D1
:10DAB00009EC78F00E0E1DEC78F00D0E1DEC78F0F0
:10DAC0000C0E1DEC78F00B0E1DEC78F00A0E1DEC20
:10DAD00078F00A0E2AEC78F00B0E2AEC78F00C0E97
:10DAE0002AEC78F00D0E2AEC78F00E0EC4EC78F0EB
:10DAF00002E6BEEC75F002E2C7EC76F07CEC75F065
:10DB0000D1D7143446E2C3EC75F043E2F7EC76F07B
:10DB100009EC78F00D0ED0EC78F00C0ED0EC78F02B
:10DB20000B0E89EC78F089EC78F0CDEC78F00B0EE8
:10DB3000CDEC78F082EC78F00D0E93EC78F038ECC8
:10DB400076F00E0EB5EC73F00DE39BEC77F007E387
:10DB500087EC76F00F5C03E36EEC75F003D03BECE2
:10DB600076F0EDD7E1EC76F038EC76F00E0EBDEC09
:10DB700073F00DE39BEC77F007E389EC76F00F5C34
:10DB800003E373EC75F003D03EEC76F0EDD714ECC4
:10DB900076F059EF78F023EC78F0D3EC74F032E3C0
:10DBA000116A126A04010A0ECDEC77F0CFEC72F024
:10DBB000090E44EC78F01A0E1DEC78F0190E1DECED
:10DBC00078F0180E1DEC78F0170E1DEC78F0160E9C
:10DBD0001DEC78F0160E2AEC78F0170E2AEC78F08F
:10DBE000180E2AEC78F0190E2AEC78F01A0EC4EC14
:10DBF00078F002E6BEEC75F002E2C7EC76F07CEC61
:10DC000075F0CBD714344EE2C3EC75F04BE2F7EC71
:10DC100076F00A0ECDEC77F077EC77F044EC78F004
:10DC2000190ED0EC78F0180ED0EC78F0170ED0EC7E
:10DC300078F0160ED0EC78F0160ECDEC78F0170ECA
:10DC4000CDEC78F0180ECDEC78F0190E93EC78F05E
:10DC500038EC76F01A0EB5EC73F00DE39BEC77F030
:10DC600007E387EC76F00F5C03E36EEC75F003D00E
:10DC70003BEC76F0EDD7E1EC76F038EC76F01A0E6E
:10DC8000BDEC73F00DE39BEC77F007E389EC76F0E5
:10DC90000F5C03E373EC75F003D03EEC76F0EDD748
:10DCA00014EC76F059EF78F023EC78F0D3EC74F0C4
:10DCB00031E3116A126A0401D9EC78F01DEC78F0B6
:10DCC0001F0E1DEC78F0200E1DEC78F0210E1DECDF
:10DCD00078F0220E1DEC78F0230E1DEC78F01E0E6D
:10DCE0002AEC78F01F0E2AEC78F0200E2AEC78F05F
:10DCF000210E2AEC78F0220E2AEC78F0230EC4ECE8
:10DD000078F002E6BEEC75F002E2C7EC76F07CEC4F
:10DD100075F0CCD7143451E2C3EC75F04EE2F7EC59
:10DD200076F0D9EC78F0D0EC78F01F0ED0EC78F0EB
:10DD3000200ED0EC78F0210ED0EC78F0220ED0EC52
:10DD400078F01E0ECDEC78F01F0ECDEC78F0200EA2
:10DD5000CDEC78F0210ECDEC78F0220ECDEC78F001
:10DD6000160E01EC76F038EC76F0230EB5EC73F07D
:10DD70000DE39BEC77F007E387EC76F00F5C03E3B1
:10DD80006EEC75F003D03BEC76F0EDD7E1EC76F07D
:10DD900038EC76F0230EBDEC73F00DE39BEC77F0DE
:10DDA00007E389EC76F00F5C03E373EC75F003D0C6
:10DDB0003EEC76F0EDD714EC76F024EC79F00C0E16
:10DDC000DAEC76F0F8EC75F078EF75F068EC73F05B
:10DDD00087E94AE838EC78F0BFEC77F00D6A0E6A14
:10DDE000C4EC77F0D3EC74F02AE30F6A106AF7EC16
:10DDF00077F017EC74F00B0E1BEC79F00A0E6AEC5E
:10DE000078F0090E48EC78F00A0E48EC78F00B0E2A
:10DE100048EC78F00C0E48EC78F010340E501018E6
:10DE200004E60F500D5C10500E5806E28FEB0DF01B
:10DE300090EB0EF08CEC78F07CEC75F0D3D70E34D0
:10DE40003BE276EC73F038E20F6A106AEEEC78F0A1
:10DE5000F7EC77F0F4DB0B0EE8EC78F00A0EE8EC68
:10DE600078F0090EE8EC78F0090EEBEC78F00A0E89
:10DE7000EBEC78F00B0ED5EC75F0C9EC77F097EC85
:10DE800078F038EC76F00C0EB5EC73F006E3A3EC0A
:10DE900077F003E23BEC76F0F4D7E1EC76F038EC87
:10DEA00076F004010C0EBDEC73F006E3A3EC77F002
:10DEB00003E23EEC76F0F3D70BEBE6FFE1EC75F016
:10DEC0002FEC77F00BEBE6FF080EE66EE66A0DEB43
:10DED000E6FF0EEBE6FFF8EC75F04BE9E7CFD9FF74
:10DEE0001200A3EC76F00F6EEA6A0F341EEC79F0A4
:10DEF0006DEC74F0D3EC74F039E3136A146ADBEC64
:10DF000077F0F0EC74F0150EF2EC78F0140EF2EC01
:10DF100078F0130EF2EC78F0120EF2EC78F0110EAD
:10DF2000F2EC78F0110E5EEC78F0120E5EEC78F008
:10DF3000130E5EEC78F0140E5EEC78F0150E5EECCD
:10DF400078F0160E5EEC78F014341250141804E6D3
:10DF50001350115C1450125806E293EB11F094EB3D
:10DF600012F08CEC78F07CEC75F0C4D7123450E2EF
:10DF7000C8EC75F04DE2136A146AEEEC78F0DBEC55
:10DF800077F0D8DB150ED6EC78F0140ED6EC78F0DE
:10DF9000130ED6EC78F0120ED6EC78F0110ED6EC0B
:10DFA00078F0110ED3EC78F0120ED3EC78F0130E5B
:10DFB000D3EC78F0140ED3EC78F0150ED3EC78F0A7
:10DFC000160ED3EC78F0180EDAEC76F051DB106E0A
:10DFD0004BEC78F038EC76F0160EC7DB08E3A2DBEA
:10DFE000105C03E23BEC76F0F5D76EEC75F0E1ECFB
:10DFF00076F038EC76F0160EC0DB08E393DB105CAD
:10E0000003E23EEC76F0F5D773EC75F014EC76F0A5
:10E010000FEBE6FFE1EC75F02FEC77F00FEBE6FF8E
:10E020000C0E56EC78F078EF75F0FCEC78F0D3EC51
:10E0300074F060E30F6A106A6EEC78F023EC77F00E
:10E04000EFCFE8F4E4DAE825E66FE76BE737DFDAED
:10E050001DEC75F0E1EC78F0B3EC77F0EFCFE6F47F
:10E060000728E96F000E0820EA6FE9510924E96EDC
:10E07000EA510A20EA6EEF50E625E46FE56BE537DA
:10E08000CDEC75F0E4510F26E5511022050E1BEC86
:10E0900079F0040E29EC79F0040E48EC78F0050EC6
:10E0A000F5EC78F005E222DB03E20FEC76F001D02C
:10E0B00070DA03EC79F005E219DB03E20FEC76F09D
:10E0C00001D067DA0BEC79F005E210DB03E20FEC2C
:10E0D00076F001D05EDA21DB10341250101804E61D
:10E0E0000F50115C1050125802E24CEC77F07CECAF
:10E0F00075F09DD7123421E2C8EC75F01EE22CECCD
:10E1000076F02DEC78F0C9EC77F041EC76F038EC55
:10E1100076F0050E2ADB06E3A3EC77F003E23BEC96
:10E1200076F0F5D7E1EC76F0A7EC78F006E3A3EC17
:10E1300077F003E23EEC76F0F7D71EEC76F0060EB1
:10E140002DEF79F0FCEC78F0D3EC74F001E211D112
:10E150000F6A106A04010704E56F000E085843ECCB
:10E1600075F0B3EC77F0EF50E42501E3102A67DA9D
:10E1700023EC77F0EFCFEAF44ADAEA25E86FE96BAF
:10E18000E93745DAE825E66F000EE921E76F3FDA67
:10E190001DEC75F0E56F000E082043EC75F00728C4
:10E1A000E76F000E0820F4EC74F0EF50E42501E373
:10E1B000102AC9EC77F06AEC78F0060E29EC79F0B9
:10E1C000060E48EC78F0090E48EC78F00C0EF5ECF1
:10E1D00078F005E28BDA03E20FEC76F001D0D9D9C2
:10E1E00003EC79F005E282DA03E20FEC76F001D07D
:10E1F000D0D90BEC79F005E279DA03E20FEC76F096
:10E2000001D0C7D98ADA060E90D9060E20EC78F034
:10E2100005E26CDA03E20FEC76F001D0BAD97DDAD0
:10E22000070E83D9070E20EC78F005E25FDA03E2EF
:10E230000FEC76F001D0ADD970DA080E76D9080E61
:10E2400020EC78F005E252DA03E20FEC76F001D030
:10E25000A0D963DA090E69D9090E20EC78F005E23D
:10E2600045DA03E20FEC76F001D093D956DA0A0EC4
:10E270005CD90A0E20EC78F005E238DA03E20FEC04
:10E2800076F001D086D949DA0B0E4FD90B0E20EC6F
:10E2900078F005E22BDA03E20FEC76F001D079D9C1
:10E2A0003CDA0C0E42D90C0E20EC78F005E21EDAB6
:10E2B00003E20FEC76F001D06CD92FDA0A0E88DA7F
:10E2C000040E20EC78F005E211DA03E20FEC76F0B0
:10E2D00001D05FD922DA0A0E28D9040EC7EC78F0F3
:10E2E00005E204DA03E20FEC76F001D052D915DA38
:10E2F0000B0E6EDA050E20EC78F005E2F7D903E29A
:10E300000FEC76F001D045D908DA0B0E0ED9050EC8
:10E31000C7EC78F005E2EAD903E20FEC76F001D021
:10E3200038D9FBD90C0E54DA060E20EC78F005E251
:10E33000DDD903E20FEC76F001D02BD9EED90C0E2B
:10E34000F4D8060EC7EC78F005E2D0D903E20FEC62
:10E3500076F001D01ED9E1D910341250101804E61D
:10E360000F50115C1050125802E24CEC77F0C4DBF5
:10E37000EBD612342AE2C8EC75F027E22CEC76F0EA
:10E38000070EEBEC78F0060EE8EC78F02DEC78F068
:10E3900056D9060EEBEC78F0070E97EC78F038ECD7
:10E3A00076F0050EE2D906E3A3EC77F003E23BEC4E
:10E3B00076F0F5D7E1EC76F0A7EC78F006E3A3EC85
:10E3C00077F003E23EEC76F0F7D71EEC76F0080E1D
:10E3D0002DEF79F07DD984E946E8EA6A003481ECD2
:10E3E00077F00034F1D8ABDA046EF450056EEA6AC7
:10E3F0000034EAD80401EE50015CE46FED5002589D
:10E4000052EC77F0016EF450026E94DB020EE66E71
:10E41000E66AE66AE66A0ACEE6FF0BCEE6FFB9ECEC
:10E4200077F099EC7BF081DA066EE551076EE651E4
:10E43000086EE751096E06EBE4F407EBE5F408EB30
:10E44000E6F409EBE7F4E42B000EE523E623E723EB
:10E45000D890E733E633E533E433E451016EE55118
:10E46000026E01EBF3FF02EBF4FF7AD331D984E9BA
:10E4700042E80050EA6A130FE96E0F0EEA22EFCF6E
:10E48000E4F40050EA6A1B0FE96E0F0EEA22EF5027
:10E490000401E45D046E056A4DDBE668E66AB9ECEA
:10E4A00077F043DA016EE551026E01EBE4F402EB22
:10E4B000E5F4E66BE76BE735000EE71909E6D8806F
:10E4C000FF0EE455000EE555000EE655000EE7552B
:10E4D00002E20168026A01EBF3FF02EBF4FF43E999
:10E4E000E7CFD9FF1200E56FE4510D24E96EE55145
:10E4F0000E20EA6EEF501200E56FE4510924E96E38
:10E50000E5510A20EA6EEF5012000851280DF3CFB2
:10E51000F6FFF4CFF7FF000EF626C40EF722120026
:10E5200000EBE9FF01EBEAFF1200075CE66F000E6B
:10E5300008580CEF77F0E96FEA6BEB6B31CFECF436
:10E5400032CFEDF4EE6BEF6BEC51E85DE46FED5123
:10E55000E959E56FEE51EA59E66FEF51EB59E76F74
:10E56000E451056EE551066E0550015C06500258F7
:10E5700012000401E417E56BE66BCAEF78F00D6E4C
:10E580000E6AFE0EE3500D5E41E9E5500E5A0E3460
:10E59000120045DBE46DE51F000EE5231200112695
:10E5A000000E12221200F626000EF7220900F55086
:10E5B0001200EA6A01342ADB0624E76EED500720D8
:10E5C000EA6EE7CFE9FF1200FE0BE96EEA36120EA3
:10E5D000E9260E0EEA221200E66E8BEC6CF043E99F
:10E5E000FCC0E4F4FDC0E5F4FEC0E6F4FFC0E7F4CF
:10E5F0001200030EE926000EEA22120000CEE4F417
:10E6000001CEE5F402CEE6F403CEE7F4120023ECEB
:10E6100077F0EF5012008FDB1D500E01205D0401DA
:10E62000E66F1E500E012159040117EF77F0FE0B23
:10E63000E96EEA361E0EE9260E0EEA2212000F26B9
:10E64000000E10221200E66EF4EC4BF042E91200CC
:10E65000EA6E0401EE501D24E46FED501E20E56FBC
:10E66000E4C4E6FFE66E1200E517E66BCAEF78F049
:10E670003DEC7AF0E55294EF77F005EBE4F406EB2D
:10E68000E5F407EBE6F408EBE7F4D950010FE96E87
:10E69000DACFEAFFEE500401E413EE50E513EE503A
:10E6A000E613EE50E71309EBE8F40AEBE9F40BEBA1
:10E6B000EAF40CEBEBF4E851E413E951E513EA5109
:10E6C000E613EB51E713040EE96E0E0EEA6E12002C
:10E6D000D9CFE6FFE1CFD9FF1200EE52EE50076E20
:10E6E000ED50086E1200EE52BAEF78F00D500008AF
:10E6F000000E0E541200E523000EE623E723E4513A
:10E70000036EE551046E120037DB2FEF77F0F6262B
:10E71000000EF7220800F5501200E4510F5EE5519B
:10E72000105A12000D500724E96E0E500820EA6EB0
:10E73000EF5012001326000E142212008BDB880EFD
:10E74000E66E000EE66ECAEC4BF042E97FEF4BF04E
:10E75000115E000E125A12000E0116250401E66F1A
:10E76000000E0E011721040162D3E427000EE523F9
:10E770000750E45D0850E5591200E45F000EE55BC8
:10E78000E451075CE55108581200EECFE6FFEECFEA
:10E79000E6FF1200D950200FE46FDACFE5F41F50E6
:10E7A000EA6AE425E96EDA50EA221200146E020EDB
:10E7B00043DB85EC7AF0E552E5CFE5F4E7CFE4F40E
:10E7C000160E3ADB85EC7AF00401FE0EE3501200DF
:10E7D0000724E66F000E08201FD30150070DF3CF6A
:10E7E000E9FFF4CFEAFF740EE9260E0EEA221200CA
:10E7F000EE52EE04076E000EED58086E1200F3CFD5
:10E80000E4F4F4CFE5F412000401EE500D24E46FBB
:10E81000ED500E20E56F140EE45D0F6E000EE5590D
:10E82000106E120001EBE9FF02EBEAFF12000F5E2F
:10E83000000E105A12000E0114250401E66F000E9E
:10E840000E0115210401F3D2E66E11EBE6FF12EB87
:10E85000E6FF0FEBE6FF10EBE6FF15EC70F046E984
:10E860001200E617CAEF78F031CFE4F432CFE5F4C6
:10E87000E66BE76B1200E66ED8EC65F044E9120037
:10E880005ADA1D500E01225D0401E66F1E500E0182
:10E8900023590401CCD2E66EDACFE6FF20CEE4F4B1
:10E8A00021CEE5F404011200EE5207EBEEFF08EB77
:10E8B000EDFF1200EE522FEF77F0040DE85100DB70
:10E8C000EECFE4F4EECFE5F461EC78F0FCEF76F017
:10E8D00056DB136A146AC4EF77F051DB116A126ACF
:10E8E000C4EF77F0000EE723E6C4E6FFE7C4E6FFD7
:10E8F0001200EA6A0134FE0BE96EEA360D0EE926D3
:10E90000000EEA22EE50046EED50056E026A036AB4
:10E91000066A076A120006CEE6F40401E46BE56BB2
:10E92000120004010C0E9BEF76F099EC7BF01FECCB
:10E930007BF0E552E5CFE7F4E5CFE6F4F5D2EE5013
:10E940000401E65DE46FEE50E75952EF77F0EFCF48
:10E95000E4F40F0133510401025CE56F000E03582B
:10E96000E66FE551E45D000EE6551200EFCFE4F4EA
:10E970000F01345104010224E56F000E0320E66FFD
:10E98000E451E55D000EE6591200E451EE12E55146
:10E99000EE12E651EE12E751EE1212000150035C46
:10E9A0000250045812000750025C0850035812002D
:10E9B000EE2AEF22072A08221200EE2AEF2207068B
:10E9C000085A1200EECFE6FFEFCFE6FF65EC7BF0D2
:10E9D000E552E5CFEDFFE7CFEFFF0BEBE6FF1200CF
:10E9E000135E000E145A1200E86FE7510924E96E15
:10E9F000E8510A20EA6E120005CEE5F40401E46B4A
:10EA00001200E4C4EEFFE5C4EDFF120046E9D95060
:10EA10000F0FE66EDACFE6FF22CEE4F423CEE5F464
:10EA2000040112000401E451096EE5510A6EE65139
:10EA30000B6EE7510C6E0F011200E625E46F000E1D
:10EA4000E721E56FE4510F26E55110220728120057
:10EA500006DA10EBE6FF120033DABCEF76F00401C1
:10EA6000E451016EE551026EE651036EE751046E0A
:10EA700012000401E451056EE551066EE651076E81
:10EA8000E751086E1200E66FE5510924E96EE65180
:10EA90000A20EA6EEFCFE4F4120004CEE4F405CECF
:10EAA000E5F406CEE6F407CEE7F41200D3D9E66A21
:10EAB0001200D950040FE96EDACFEAFF1200E66EB9
:10EAC00054EC2DF042E91200045105110611071112
:10EAD000120006EBEEFF07EBEDFF120087EB0BF0E9
:10EAE00088EB0CF0120087EB09F088EB0AF01200BB
:10EAF0004FE9E7CFD9FF1200072A000E08221200C3
:10EB0000016B026B036B046B056B066B076B1200EA
:10EB100002EC2CF042E91200EF500226000E032214
:10EB2000062A0722120044510A5D446F45510B59D1
:10EB3000456F120004EBE6FF05EBE6FFE66AE66AC6
:10EB4000120002EBE9FF03EBEAFF120085EC7AF01A
:10EB5000E552E550120001EBE6FF02EBE6FF120082
:10EB600047E9E7CFD9FF120054EC6EF046E9D950DF
:10EB700012000401D950010FE86F12001150135C0C
:10EB800012501458120013500008000E14541200B2
:10EB900011500008000E12541200D890E533E433EF
:10EBA0001200075CD9D20724DCD20724E46F000EE0
:10EBB00008207CEF72F0075CE46F000E08587CEFD1
:10EBC00072F05DDBE2DD8DDA81DADFDDF2EC2BF075
:10EBD00042E915DE66EF78F052DB04EBEEFF05EB61
:10EBE000EDFF9EDC030EEB6A040EEB6A90EF72F011
:10EBF0003DEC7AF03BDC43E9F4CFE5F491DC84EFC3
:10EC000073F030DB35DD0F6E4BEF78F0FE0BE96E05
:10EC1000EA36010EE926000EEA22EE5012000DEB54
:10EC2000E4F40EEBE5F412000B500924E46F0C50F1
:10EC30000A20E56FB2DF23DB01EF75F00BEBE6FF97
:10EC40001EDB3FDA0401E62B4DDE4BDA320EE66EB8
:10EC5000E66A3CDAE2EF74F00F6A106ABFDA3EDA75
:10EC6000D6DCEDDC0728ADDAD8900F36103612006E
:10EC700057DC73EF73F02ADAD8EF74F027DADDEFA0
:10EC800074F0E66EE66A0FEBE6FF10EBE6FFF0DCF1
:10EC90000C6EEEEF78F025C0E6FF26C0E6FF02EB33
:10ECA000E6FF03EBE6FF52DF036EE750026E5EDA2B
:10ECB000EE6AED6A066A076A120075DC076E0A00E2
:10ECC000F550086E85EF72F06EDC096E0A00F550A3
:10ECD0000A6E85EF72F067DC0B6E0A00F5500C6E61
:10ECE00085EF72F060DC0A6E0A00F5500B6E85EF5E
:10ECF00072F059DC0C6E0A00F5500D6E85EF72F063
:10ED000052DC0E6E0A00F5500F6E85EF72F0072888
:10ED100028D2070421D204010404E46F000E055830
:10ED2000E56FEA6A013483DC6CDE0404066E000ED3
:10ED30000558076E1200E45F000EE55BE4C4E6FFD1
:10ED4000E5C4E6FF1200C4DC87E94EE890EC72F0FF
:10ED5000EF501200080FE66EDACFE6FF140EE96EF0
:10ED60000E0E28EF73F0160FE66EDACFE6FF160EE2
:10ED7000E96E0E0E28EF73F0050EE926000EEA226A
:10ED8000120011DC9BEF78F00EDCA1EF78F091EB34
:10ED900013F092EB14F08CEF78F049DCBAEF78F0D6
:10EDA000B6DC0D6E0E6A85EF72F0B1DC106E116A82
:10EDB00085EF72F0E66EE66A13EBE6FF14EBE6FF12
:10EDC000120090EC72F0F8EF73F0E4EC72F079D985
:10EDD0000C0EE62787DDE6EC6EF046E91200CFEC7C
:10EDE00072F0040E1200CFEC72F0020E1200116AE3
:10EDF000126AF4D904011200E451E511E611E71199
:10EE00001200E4EC72F0EE500D24116EED500E2065
:10EE1000126E140ECFEF72F0E76FE6510924E96E1F
:10EE2000E7510A20EA6EEF50E66EE66A1200E76FDD
:10EE3000E6C4E6FFE66E1200E66EE66A0CCEE6FF7A
:10EE40000DCEE6FF120009500724E96E0A50082093
:10EE5000EA6E1200E66E5BEC2DF042E91200F3CF91
:10EE6000EEFFE5C4EDFF1200F20EE66E690E87D9E3
:10EE70003BEF74F02DDC81E912000E0185EF72F09A
:10EE8000CFEC72F00A0E1200CFEC72F0060E1200F8
:10EE90001FEC73F0030E12008FEB11F090EB12F0E9
:10EEA0008CEF78F0E56FE4C4E6FFE66EF2EC2BF051
:10EEB00042E9F350120069DC5DEC2CF043E91200EA
:10EEC000F324E96EDA50F420EA6E120041DC1234C9
:10EED000145012181200FEEC72F00401E46B1200E0
:10EEE000A1DCF9EF72F013DC126E136A1200CFECA2
:10EEF00072F0080E12000CDEC20EE66E6A0E9EEF75
:10EF000073F017EC73F0DDD8EA6A1200C4DC230E4C
:10EF10000BEC73F0B4EF75F0ECEC72F0040EE96EEC
:10EF20000E0EEA6E04011200E5CFE5F4E7CFE4F43B
:10EF30000401E451120092EC73F00F5C12001FEC1C
:10EF400073F0040E120007EC73F00C5C12006FDC1F
:10EF5000030E12000BD969EF75F0EA6A013417EC61
:10EF600073F069EF75F00704E76F000E0858F4EFCF
:10EF700074F0E66AE66AEFDDE66AE66A1200050EFC
:10EF8000EB6A060EEB6A120084EB07F085EB08F0E3
:10EF900012001FEC73F00C0E120003DEA8DF01DE7E
:10EFA00073DFFFDD1CDF65D964D9FDDD18DFFBDD14
:10EFB0006BDFD3EF75F004010C0EF8D80A0EF6D80B
:10EFC000080EF4D8060EF2D8040EF0D8020EEED8D1
:10EFD000020EE9D8040EE7D8060EE5D8080EE3D8ED
:10EFE0000A0EE1D80C0EDFD8160ED1EF75F0040131
:10EFF000040E42D9EDD8020EEBD815D90728E1D876
:10F00000020ED3DD45DFD1DD9ADFCFDDC2DFDBEFDE
:10F0100075F0050EC6DDE3DEC3D8030E2AD9C0D8CD
:10F0200078DECFEC72F073DEDEDEB7D8030EBBDD28
:10F03000D6DEB3D8050ECDEF78F0B3DDA8EF73F0D0
:10F04000B4DDBFEF72F07FDE106EEA6A1034F6D8DE
:10F0500068EF74F0A8DDA8EF73F0050EACDD6FDF8C
:10F060000BD90AD9A2DD6BDFB6D8050ED5EF75F046
:10F0700090EC72F0EF500B6EEA6A0B34C7DD096E4C
:10F08000ED500A6EECEF75F08EDDFADECDEF78F024
:10F090008CDD17EF74F0F3D8EE500B6EED500C6E64
:10F0A0008BEB09F08CEB0AF0EEEF78F0DBD8F8EFA1
:10F0B00075F0CAD80A0E7EDE9BDD1AD574DDF0EF3E
:10F0C00074F0EECFE6F4EFCFE7F4120090EC72F0BC
:10F0D000F9EF72F0B0D8090E1BEF79F0040113EFCD
:10F0E00079F0EAEC71F043E9FFEC73F090EC72F028
:10F0F0005AEF74F0430EE66E0E0EE66EEA6A0E34B8
:10F10000CDEF76F00C0ECDEF78F012EC74F0BCEF92
:10F1100076F047DD40EF77F090EC72F054EF74F04A
:10F120004ADDA7EF77F039D8120E01EF76F053D809
:10F13000100E41EF76F0056E0A00F550066E85EF71
:10F1400072F0086E0A00F550096E85EF72F090DDDE
:10F150000401050EBDEF73F0E46F000E085873EF65
:10F1600072F0E46F000E082073EF72F0EA6A013467
:10F17000E4EF72F0EECFE4F4EFCFE5F41200E66EC8
:10F18000430EE66E0E0E12000EDD66EF77F013DD15
:10F19000BFEF72F0E76BFCEF76F005DDCFEF72F0BA
:10F1A00000DDCFEF72F0FFDC9AEF73F0FADC9AEF3C
:10F1B00073F00C0EAEDFF1DE9ADE66DFA3DF1E0E0B
:10F1C0001200E46F000E08207CEC72F01FEF73F069
:10F1D000F2DC1FEF73F0E9DC1FEF73F090EC72F0DC
:10F1E0006DEF73F0DEDCF0EF74F0DFDCB0DE95EC99
:10F1F00072F0030E20EF78F068EC73F087E94CE8CA
:10F2000037DF6DEF74F08DEC73F0040E95EC72F057
:10F21000040E20EF78F08DEC73F0050E95EC72F093
:10F22000050E20EF78F00704E46F000E08587CEC20
:10F2300072F01FEF73F0BFDC17EF74F0E7DC0D6EB8
:10F24000ED500E6EECEF75F010EBE6FFBADC28EF38
:10F2500075F066DF65DF48EF78F028DF4DE9E7CF2E
:10F26000D9FF1200E66EE66A11EBE6FF12EBE6FF4D
:10F27000120097DCF3EF76F09EDC48EF77F090EC2D
:06F2800072F0EE521200D4
:0AF2860045E8D9CFE6FFDACFE6FF36
:10F29000E1CFD9FFE2CFDAFF8BE9086A9EEC79F083
:10F2A00008B657EF79F008AA0ED008BC05D07F0E3B
:10F2B000016EFF0E006E23D0800E016E006A1FD01B
:10F2C000016A006A1CD008B8FBD78F0E0360EDD727
:10F2D0007E0E0364F5D78E0E035C05E0D8900232F3
:10F2E0000132032AF8D708AC06D0016C021EE86A86
:10F2F000022202AEE5D781EB00F082EB01F0E5528D
:10F30000E5CFDAFFE7CFD9FF47E912000636073627
:10F3100002E30884087E06E10880076A066A056A37
:10F32000046A1200072803E0D88006321200D89041
:10F33000063202E108821200088612000236033605
:10F3400002E3088C087E06E10888036A026A016A03
:10F35000006A1200032803E0D88002321200D8901D
:10F360000232EAE1088A120045E8D9CFE6FFDACF97
:10F37000E6FFE1CFD9FFE2CFDAFF8BE9086A9EEC26
:10F3800079F008B6C8EF79F008AA0FD008BC07D00A
:10F390007F0E036EFF0E026E016E006E2DD0800E8A
:10F3A000036E01D0036A000EF6D708B8FBD7076AD0
:10F3B0009F0E0360EBD77E0E0364F4D79E0E035CB2
:10F3C00007E0D8900232013200320732032AF6D722
:10F3D00008AC0AD0076C001E011E021EE86A00225B
:10F3E0000122022202AEDED782EB03F081EB02F0B3
:10F3F00080EB01F087EB00F0E552E5CFDAFFE7CFD5
:10F40000D9FF45E9120042E8D9CFE6FFDACFE6FF9F
:10F41000E1CFD9FFE2CFDAFF86E9036A1200F3DF1A
:10F42000038003D0F0DF01D00382026A080EE76E8A
:10F43000D890013602360050025C02E3026E012AC7
:10F44000E72EF7D703B2120003B081EB00F003A060
:10F4500082EB00F0E552E5CFDAFFE7CFD9FF43E9D1
:10F46000120043E8D9CFE6FFDACFE6FFE1CFD9FFBC
:10F47000E2CFDAFF89E9066A1200F3DF068001D0E5
:10F48000F0DF01AE4AEF7AF0006C011EE86A01225B
:10F4900006B0067E03AE52EF7AF0026C031EE86AF5
:10F4A0000322067E8AEC7AF003BE74EF7AF006AE91
:10F4B00008D0026C031EE86A0322046C051EE86A89
:10F4C000052206B006D084EB00F085EB01F006A023
:10F4D00004D082EB00F083EB01F0E552E5CFDAFFD8
:10F4E000E7CFD9FF45E9000C06BE59EF7AF0E9DF16
:10F4F000FF0C43E8D9CFE6FFDACFE6FFE1CFD9FF33
:10F50000E2CFDAFF89E9066A1200F3DF068003D052
:10F51000F0DF01D00682056A046A100EE76ED8900B
:10F5200002360336043605360050045C0150055897
:10F5300005E30050045E0150055A022AE72EF0D779
:10F5400006B2120006B006D084EB00F085EB01F0A5
:10F5500006A004D082EB00F083EB01F0E552E5CF8A
:10F56000DAFFE7CFD9FF45E9120045E8D9CFE6FF3A
:10F57000DACFE6FFE1CFD9FFE2CFDAFF8FE90C6AFD
:10F580001200F3DF0C8001D0F0DFE86A03AED2EFA7
:10F590007AF0006C011E021E031E012202220322C9
:10F5A0000CB00C7E07AEDDEF7AF0046C051E061E73
:10F5B000071E0522062207220C7E24EC7BF007BEE4
:10F5C0000EEF7BF00CAE0FD0046C051E061E071E5E
:10F5D000E86A052206220722086C091E0A1E0B1E75
:10F5E00009220A220B220CB00AD088EB00F089EB2A
:10F5F00001F08AEB02F08BEB03F00CA008D084EB57
:10F6000000F085EB01F086EB02F087EB03F0E552AA
:10F61000E5CFDAFFE7CFD9FF49E9000C0CBEE4EFF4
:10F620007AF0E1DFFF0C45E8D9CFE6FFDACFE6FF5D
:10F63000E1CFD9FFE2CFDAFF8FE90C6A1200F3DFE6
:10F640000C8003D0F0DF01D00C820B6A0A6A096AD1
:10F65000086A200EE76ED89004360536063607365F
:10F66000083609360A360B360050085C0150095836
:10F6700002500A5803500B5809E30050085E01502D
:10F68000095A02500A5A03500B5A042AE72EE4D7AB
:10F690000CB212000CB00AD088EB00F089EB01F03C
:10F6A0008AEB02F08BEB03F00CA008D084EB00F0A7
:10F6B00085EB01F086EB02F087EB03F0E552E5CF36
:10F6C000DAFFE7CFD9FF49E9120044E8D9CFE6FFD6
:10F6D000DACFE6FFE1CFD9FFE2CFDAFF8AE980EBAC
:10F6E00004F081EB05F082EB06F002500402F450C6
:10F6F000016EF350006E0350076E0502F450036E66
:10F70000F350026E07500402F3500126F450022217
:10F71000E86A032206500502F3500126F450022243
:10F72000E86A0322E552E5CFDAFFE7CFD9FF46E9E1
:10F73000000C44E8D9CFE6FFDACFE6FFE1CFD9FFEE
:10F74000E2CFDAFF8EE980EB08F081EB09F082EB83
:10F750000AF083EB0BF004500802F350006EF450F3
:10F76000016E04500902F3500126000EF420026ECF
:10F7700004500A02F3500226000EF420036E0450D7
:10F780000B02F350032605500802F3500126F450F3
:10F790000222000E032205500902F3500226F45003
:10F7A000032205500A02F350032606500802F350C4
:10F7B0000226F450032206500902F3500326075094
:10F7C0000802F3500326E552E5CFDAFFE7CFD9FF71
:10F7D00048E9000C4AE8D9CFE6FFDACFE6FFE1CFEF
:10F7E000D9FFE2CFDAFF94E9086A86EC79F09EEC63
:10F7F00079F008B6A2EF7CF008A205D008B8A2EF15
:10F800007CF0A9EF7CF008AA05D008B0A2EF7CF04C
:10F81000A9EF7CF008B002D008A802D0B5EF7CF0C8
:10F820000E6A035007240D6EE86A0E227E0E0D5EEE
:10F83000E86A0E5A096A0A6A0B6A0C6A02500602E2
:10F84000F4500C6EF3500B6E01500602F3500A2672
:10F85000F4500B22000E0C2202500502F3500A262F
:10F86000F4500B22000E0C2200500602F350092621
:10F87000F4500A22000E0B220C2201500502F35014
:10F880000926F4500A22000E0B220C220250040218
:10F89000F3500926F4500A22000E0B220C220050CD
:10F8A0000502F4500926000E0A220B220C220150F8
:10F8B0000402F4500926000E0A220B220C2261EFEA
:10F8C0007CF00C500B100A10091055E00EBE4DD004
:10F8D0000CBE0CD00D500E1048E0D89009360A36F8
:10F8E0000B360C360D06D8A00E06F2D70E5031E1BD
:10F8F0000D282FE009AE11D07F0E091402E10AA0F5
:10F900000CD00A2AE86A0B220C2207E3D8800C32BA
:10F910000B320A320D2A0D281CE00D5026E08AEB2E
:10F9200000F08BEB01F00C34026E0D30036E0232EE
:10F93000039E08BE038EE552E5CFDAFFE7CFD9FF7D
:10F940004EE912007F0E036EFF0E026E016E006E16
:10F95000F2D77F0E08BEFF0E036E02D07F0E036E3D
:10F96000800E026E016A006AE6D708AE04D0800EEF
:10F97000036E026AF7D7036A026AF4D7D89801D0F7
:10F98000D8884EE8D9CFE6FFDACFE6FFE1CFD9FF3E
:10F99000E2CFDAFF94E9089E0BE703AE09D0006CD2
:10F9A000011E021E031EE86A012202220322088EA3
:10F9B00083EB0CF082EB0BF081EB0AF080EB09F0AB
:10F9C0009E0E0D6E0E6A61EF7CF04AE8D9CFE6FF1D
:10F9D000DACFE6FFE1CFD9FFE2CFDAFF94E9086A98
:10F9E00086EC79F09EEC79F008B6A2EF7CF008A2E4
:10F9F00005D008BAA2EF7CF0A9EF7CF008BAB5EF09
:10FA00007CF008A005D008B8A2EF7CF0B5EF7CF040
:10FA100008B8A9EF7CF00E6A7F0E07240D6EE86A25
:10FA20000E2203500D5EE86A0E5A1A0E0F6E076A18
:10FA3000096A0A6A0B6A0C6A0050045E0150055A92
:10FA40000250065A000E075A09E7005004260150DA
:10FA5000052202500622000E072201D0098AD89002
:10FA60000436053606360736D89009360A360B3680
:10FA70000C360F2EE1D7065005100410D8A4098AC1
:04FA800061EF7CF0C6
:0CFA840000FFFFFF00000101010000FF77
:10FA9000FFFF000001010100000101010000FFFF64
:10FAA000FF000000000000000000000000FFFFFF5A
:10FAB000000001010100000101010000FFFFFF0043
:10FAC000000101010000FFFFFF0000000000000036
:10FAD0000000000000FFFFFF00000101010000FF27
:10FAE000FFFF00000101010000FFFFFF0000010116
:10FAF000010000FFFFFF00000101010000FFFFFF08
:10FB000000000101010000FFFFFF000001010100F2
:10FB100000FFFFFF000001010100000101010000E2
:10FB2000FFFFFF0000FFFFFF00000101010000FFD9
:10FB3000FFFF000001010100000101010000FFFFC3
:10FB4000FF00000101010000FFFFFF0000FFFFFFB9
:10FB5000000001010100000101010000FFFFFF00A2
:10FB6000000101010000FFFFFF0000010101000092
:10FB7000FFFFFF00000101010000FFFFFF00000187
:10FB800001010000FFFFFF00000101010000FFFF75
:10FB9000FF00000101010000FFFFFF009209920930
:10FBA000220BEA0B540B4E0CB20C090009000C009E
:10FBB0000C000C000C000C0020352000787820315F
:10FBC000302000012032302000012035302000019B
:10FBD00020313030200020323030200020353030CD
:02FBE000200003
:0EFBE2001DEE00F02DEE00F0F86A44EC57F036
:0CFBF000FEEC7DF058EC1BF0FBD712007F
:02FBFC001200F5
:01FBFE000006
:01FFF8006C9C
:01FFF900F710
:01FFFA000303
:01FFFB00F90C
:01FFFD00FF04
:00000001FF
